:10A22D000D0A0D0A0D0A092A2A2A2A2A2A2A2A2A59
:10A23D002A2A2A2A2A2A2A2A2A2A2A2A2A2A2A2A71
:10A24D002A2A2A2A2A2A2A2A2A2A2A2A2A2A2A0D7E
:10A25D000A00092A202020202020205472616B4200
:10A26D006F782020383043333230202076332E362D
:10A27D00306120202020202020202A0D0A00092ACC
:10A28D00202020284329204A414D5341542F4A4133
:10A29D003646544C2020205365702E3232203230F9
:10A2AD003133202020202A0D0A00092A2A2A2A2AA1
:10A2BD002A2A2A2A2A2A2A2A2A2A2A2A2A2A2A2AF1
:10A2CD002A2A2A2A2A2A2A2A2A2A2A2A2A2A2A2AE1
:10A2DD002A2A2A0D0A00205472616B426F782038A9
:10A2ED003043333230200000202076657273696F61
:10A2FD006E20332E3630612000002843294A414D0F
:10A30D005341542F4A413646544C0000594F524F39
:10A31D004E0031332F30312F30312030303A303044
:10A32D003A3030000A0D07546F6F206F6C64206552
:10A33D006C656D656E74732E0D0A000A0D07000DA8
:10A34D000A092A2A2A2020547261636B696E6720DC
:10A35D006F626A65637420736174656C6C69746592
:10A36D0020202A2A2A0D0A000D0A0D0A092A2A2A56
:10A37D00202053656C656374206F626A6563742079
:10A38D00736174656C6C69746520202A2A2A0D0A24
:10A39D000007000D0A094461746120696E20524165
:10A3AD004D20776173206C6F7374202121205365CC
:10A3BD00742064656661756C7420706172616D6581
:10A3CD00746572202120070D0A004E4F43414C4CFD
:10A3DD000000594F524F4E0000205B592F4E5D200B
:10A3ED003F20000D0A093D3D3D3D2041444320766F
:10A3FD00616C756520616E6420616E74656E6E6151
:10A40D0020646972656374696F6E203D3D3D3D202A
:10A41D000D0A0D0A000D0A20092D2D2D2D2D2D2093
:10A42D004D41494E204D454E55202D2D2D2D2D2D77
:10A43D000D0A0D0A0009312E205265616C74696D8B
:10A44D006520547261636B696E672E0D0A000932C7
:10A45D002E20446973706C6179205363686564754F
:10A46D006C652E0D0A0009332E20557064617465DC
:10A47D0020536174656C6C69746520456C656D6500
:10A48D006E74732E0D0A0009342E2055706461749C
:10A49D00652053746174696F6E20456C656D656ED2
:10A4AD0074732E0D0A0009352E2055706461746584
:10A4BD00205265616C74696D6520436C6F636B2E02
:10A4CD000D0A0009362E20436F6E6669677572613D
:10A4DD0074696F6E2E0D0A0009372E20486F737444
:10A4ED00206D6F64652E0D0A0009382E20446972A7
:10A4FD0065637420416E74656E6E6120636F6E745A
:10A50D00726F6C2E0D0A0D0A000D090953656C65ED
:10A51D006374205B312D382C532C4D5D3A20000D8A
:10A52D000A0D0A092020203D3D3D3D3D3D3D3D3D6F
:10A53D0020555044415445204D454E55203D3D3DFF
:10A54D003D3D3D3D3D0D0A0009312E204544495408
:10A55D0020203A20566965772F4564697420736110
:10A56D0074656C6C69746520456C656D656E74738E
:10A57D002062792068616E642E0D0A0009322E204A
:10A58D0053454C4543543A2053656C6563742053D1
:10A59D006174656C6C697465732066726F6D20747F
:10A5AD0068652064617461626173652E0D0A00092E
:10A5BD00332E2052454C4F41443A20436C65617215
:10A5CD002064617461626173652026207265616427
:10A5DD0020696E206E657720456C656D656E7473B0
:10A5ED002E0D0A0009342E20415050454E443A207C
:10A5FD00417070656E64206E657720456C656D6584
:06A60D006E74732E0D0AAD
:10A613000009352E204D554C544920545241434B8B
:10A623003A20436F6E666967757265206D756C7449
:10A633006920747261636B696E67207361742E2085
:10A643006E756D6265722E0D0A0D0A000D090953B0
:10A65300656C6563743A20000D0A092A2A2A2020B2
:10A6630053656C656374206F626A656374207361FC
:10A6730074656C6C69746520202A2A2A0D0A000708
:10A683000D0A0953656C6563746564206C697374A2
:10A693002077696C6C206265206C6F73742E204187
:10A6A300726520796F752073757265203F000D0AFE
:10A6B3000D0A09312E2053656C6563742020202018
:10A6C3003A2053656C65637420736174732E206242
:10A6D300792068616E642E0D0A0009322E205365BD
:10A6E3006C65637420416C6C3A2053656C656374CC
:10A6F30020616C6C20736174732E20696E20746802
:10A70300652064617461626173652E0D0A0009330B
:10A713002E2055706C6F6164202020203A205570E4
:10A723006C6F61642073656C656374696F6E20641C
:10A733006174612066696C652E0D0A0D0A00070DB0
:10A743000A0953746F726564206461746120696ED1
:10A75300206D656D6F72792077696C6C206265205E
:10A763006C6F73742E2041726520796F7520737539
:10A773007265203F00070D0A204E6F20726F6F6DC8
:10A7830020666F7220617070656E6420210D0A006F
:10A793000D0A0946696C6520666F726D6174204EFF
:10A7A30041534120284E29203A2020000D0A094810
:10A7B3006F77206D616E7920736174656C6C697459
:10A7C300657320636F6E66696775726520666F7265
:10A7D300206D756C746920747261636B696E672098
:10A7E3006D6F6465203F202832202D2035292020DD
:10A7F300000D0A094F7574206F662072616E6765DC
:10A8030020210700536F757468004E6F72746800DF
:10A8130020333030003132303000323430300034C5
:10A8230038303000393630300031393230300020A2
:10A83300202020202020202043616C6C7369676EE8
:10A84300002020202020202020204C617469747572
:10A8530064650020202020202020204C6F6E676933
:10A863007475646500202020416E74656E6E6120EE
:10A8730068656967687400526F746F7220737461DE
:10A8830072742028532F4E290020202020434F4D3F
:10A8930020706F72742062617564000D0A0D0A09DD
:10A8A3002020203D3D3D3D3D3D3D3D3D20537461D8
:10A8B30074696F6E2044617461203D3D3D3D3D3DB3
:10A8C3003D3D0D0A0009312E20454449543A2020CC
:10A8D30020566965772F45646974207374617469C0
:10A8E3006F6E20656C656D656E7473206279206888
:10A8F300616E642E0D0A0009322E2052454C4F41E1
:10A90300443A20436C6561722064617461626173CF
:10A91300652026207265616420696E206E6577204C
:10A92300646174612E0D0A0D0A000D0A0D0A093DBA
:10A933003D3D3D3D3D3D3D3D2053746174696F6E2A
:10A9430020456C656D656E7473203D3D3D3D3D3D19
:10A953003D3D0D0A0D0A00253135733A202025733C
:10A963000900253135733A2020252B352E33660017
:10A973000900253135733A202025352E326600250E
:10A983003135733A20202573092000253135733A78
:10A9930020202573000D0A09456E7465722027591E
:10A9A3002720666F72207A65726F207365632E208D
:10A9B30061646A7573746D656E74000D0A09456E82
:10A9C3007465722027512720666F72206578697439
:10A9D300000D0A09456E74657220275265742E278F
:10A9E30020666F72205265616C2054696D65204347
:06A9F3006C6F636B207322
:10A9F90065740D0A0D0A000950726573656E74203D
:10AA090054696D653A55544320002534642F253027
:10AA19003262642F25303262642025303262643A12
:10AA290025303262643A25303262640D000D0A0D18
:10AA39000A09536574207265616C74696D652043F8
:10AA49006C6F636B2E0D0A0950726573656E742005
:10AA590054696D653A55544320002534642F2530D7
:10AA69003262642F25303262642025303262643AC2
:10AA790025303262643A25303262640D0A00094594
:10AA89006E746572207769746820666F726D61747F
:10AA9900205B59592F4D4D2F44442048483A4D4D7C
:10AAA9003A53535D20000D0A095365742074696D8A
:10AAB900653A2025730D0A000D0A09202020454E0C
:10AAC900544552207768656E2072656164792E005D
:10AAD9000D0A07202120466F726D6174204572723C
:10AAE9006F7220210043415420004D69632D636C2E
:10AAF90069636B20004E6F00596573002020202088
:10AB0900202020536174656C6C69746520203A00BB
:10AB190020202045706F63682054696D652054308A
:10AB290020203A002020202045706F63682052655C
:10AB390076204B3020203A00204D65616E20416E11
:10AB49006F6D616C79204D3020203A0020204D65D1
:10AB5900616E204D6F74696F6E204E3020203A006F
:10AB69002020496E636C696E6174696F6E2049308B
:10AB790020203A0020456363656E747269636974C5
:10AB89007920453020203A002020417267207065E5
:10AB9900726967656520573020203A0020202020FF
:10ABA90020522E412E412E4E2E204F3020203A0089
:10ABB90020202020202020204465636179204E3107
:10ABC90020203A0020446F776E6C696E6B204672C4
:10ABD900712E463120203A0020202055706C696E74
:10ABE9006B204672712E463220203A0020202044E4
:10ABF9006F776E6C696E6B206D6F646520203A000B
:10AC0900202020202055706C696E6B206D6F646563
:10AC190020203A0020202045706F63682059656123
:10AC29007220593020203A00446F70706C65722090
:10AC3900636F72726563742E20203A0020204C43A2
:10AC490044204D4120646973706C617920203A0079
:10AC59002020204F666673657420666F7220463126
:10AC690020203A002020204F666673657420666FA5
:10AC79007220463220203A00202020202046312010
:10AC8900736C657728487A2920203A006E6F6E65C3
:10AC9900004C5342200055534220004357202000C6
:10ACA900464D2020000D0A0D0A09093D3D3D3D3D57
:10ACB9003D20536174656C6C6974652064617461CD
:10ACC900203D3D3D3D3D3D0D0A0009257320252DC3
:10ACD90073090900092573202564000909095930F8
:10ACE9003A000925732025362E35660009095430A6
:10ACF9003A000925732025366C640009094B303A5E
:10AD09000009094D303A0009094E303A000909494C
:10AD1900303A00090945303A00090957303A000923
:10AD2900094F303A0009257320256500094E313A4B
:10AD3900000925732025362E336600090946313A64
:10AD4900000925732025362E306600090946783A10
:10AD59000009202046314F46465345543A000925FB
:10AD6900732025362E33662025362E336620253668
:10AD79002E33662025362E33660D0A09090920204F
:10AD890020200025662025662025662025660009E5
:10AD9900202046324F46465345543A000925732030
:10ADA9002573090920202000092573202573090925
:10ADB90009202020000D0A0D0A093D3D3D3D3D3D7C
:10ADC9003D20436F6E66696775726174696F6E20A5
:06ADD9004D656E7520209F
:10ADDF003D3D3D3D3D3D0D0A0009302E2044697338
:10ADEF00706C617920616C6C20636F6E666967753A
:10ADFF007265642076616C7565730D0A0009312EDA
:10AE0F002043616C6962726174696F6E206F662096
:10AE1F00616E74656E6E61207370616E2076616C09
:10AE2F0075650D0A0009322E205365742041444385
:10AE3F00207370616E2076616C75650D0A000933A1
:10AE4F002E2053657420446561642042616E642036
:10AE5F00616E6420536B65772076616C75650D0AA2
:10AE6F000009342E2053657420616E74656E6E6117
:10AE7F00205061726B696E6720616E64204C696D42
:10AE8F00697420706F736974696F6E0D0A000935EC
:10AE9F002E204D6F6E69746F72204144432076618E
:10AEAF006C7565202620416E74656E6E6120706F23
:10AEBF00736974696F6E0D0A0009362E204469722A
:10AECF0065637420616E74656E6E6120636F6E745E
:10AEDF00726F6C0D0A0009372E20526164696F2062
:10AEEF0043415420706F727420636F6E666967758B
:10AEFF00726174696F6E0D0A0009382E204D6963F7
:10AF0F002D636C69636B20636F6E66696775726121
:10AF1F0074696F6E0D0A0009392E20536574206411
:10AF2F00656661756C7420706172616D65746572B0
:10AF3F000D0A0D0A000D0A09436F6E666967757277
:10AF4F006520796F75722073746174696F6E2065F7
:10AF5F006C656D656E7473203F205B592F4E5D20BD
:10AF6F0020000D0A0A0943415420526967204B45BE
:10AF7F004E574F4F442C59414553552C49434F4D34
:10AF8F00205B4B2F592F495D203F2020000D0A09D0
:10AF9F004973207468652043415420524947205417
:10AFAF00532D37313120262054532D383131206322
:10AFBF006F6D62696E6174696F6E203F205B592FF0
:10AFCF004E5D20000D0A092020596F75206D757395
:10AFDF00742075736520616C7465726E6174652081
:10AFEF00434F4D20706F727420666F722055706CD6
:10AFFF00696E6B20545258000D0A092020416C7461
:10B00F0065726E61746520434F4D20706F727420AE
:10B01F00697320383033312050312E352F434E3362
:10B02F002D3620000D0A0953656C65637420545248
:10B03F005820313A46542D3733362020323A465471
:10B04F002D3834372020333A4F7468657220202012
:10B05F00000D0A0953656C65637420464D4E206DD3
:10B06F006F6465203F205B592F4E5D20000D0A094C
:10B07F00456E7465722064657374696E6174696F6F
:10B08F006E204164647265737320666F722052582C
:10B09F0020282542582920002568780009456E741C
:10B0AF0065722064657374696E6174696F6E204197
:10B0BF0064647265737320666F722054582028255C
:10B0CF0042582920000953657061726174656420CC
:10B0DF00545258203F205B592F4E5D2020000D0AFF
:10B0EF0009576169742074696D6520666F722063FA
:10B0FF006F6D6D616E64205B25645D2000205B3198
:10B10F002D3235355D20000D0A09506F72742062A3
:10B11F006175642072617465203F205B313230307D
:10B12F002F323430302F343830302F393630302FF3
:10B13F0031393230305D20000D0A0955706C696E5F
:10B14F006B20446F70706C657220636F72726563F1
:10B15F0074696F6E203F205B592F4E5D2020000DCC
:10B16F000A09446F776E6C696E6B20446F70706C58
:10B17F00657220636F7272656374696F6E203F2012
:10B18F005B592F4E2F525D2020000D0A0953656C1D
:10B19F006563742046756C6C206F72626974206FE2
:10B1AF007220414F532043415420636F6E74726F6E
:06B1BF006C203F205B46FE
:10B1C5002F415D2020000D0A0D0A09203D3D3D3D22
:10B1D5003D3D3D3D3D3D205265616C74696D652089
:10B1E500547261636B696E67205B2534642F25306B
:10B1F5003262642F25303262645D203D3D3D3D3D28
:10B205003D3D3D3D0D0A000D0A2020274527546F81
:10B2150067676C6520726F746F7220636F6E7472EE
:10B225006F6C2020275027546F67676C65207072FC
:10B23500696F7269747920747261636B2027512775
:10B2450052657475726E20746F206D61696E206D24
:10B25500656E750D0A0D0A00202048483A4D4D3A95
:10B2650053532020202000252D3133730020202D1D
:10B2750020202020202020202020000D0A000D0A5B
:10B28500202027452720546F67676C6520726F74EF
:10B295006F7220636F6E74726F6C202027592720A0
:10B2A500525443207A65726F2061646A7573742005
:10B2B500202751272052657475726E20746F206D9A
:10B2C50061696E206D656E75000D0A20202749277E
:10B2D50020496E697469616C697A652074686520B6
:10B2E500545258202020202754272054756E65205D
:10B2F500545258202020275350432F4253272020B3
:10B305004E6578742F50726576696F75732E20734C
:10B3150061742E000D0A202027312F322F332F3450
:10B32500272055706C696E6B206368616E6E656C65
:10B335002020272B2F2D2F302720446F70706C6510
:10B345007220636F6D70656E736174696F6E202016
:10B35500273F27206F626A2E207361742E000D0A25
:10B365002020274E2720547261636B206E65787408
:10B3750020736174656C6C697465202027502720E3
:10B38500546F67676C65207072696F726974792094
:10B39500747261636B696E670D0A0020205B5361EF
:10B3A50074656C6C6974653A20252D39735D200DC3
:10B3B5000A00202020202055544320202020204111
:10B3C5007A696D2E202020456C65762E202020522E
:10B3D500616E6765202020202020416C742E20207E
:10B3E500204C61742E2020204C6F6E672E2020503B
:10B3F50068617365202020446F70706C65720D0A5A
:10B4050000202048483A4D4D3A535320202064658A
:10B415006720202020206465672020202020204BE5
:10B425006D20202020202020204B6D202020202052
:10B4350064656720202020206465672020203C3239
:10B4450035363E202020202020487A0D0A000D0A9E
:10B455000D0A092A2A2A202053656C656374206F1A
:10B46500626A65637420736174656C6C69746520C8
:10B47500666F72204C434420646973706C61792057
:10B485002831202D2025626429202A2A2A0D0A0028
:10B49500070D0A094F7574206F66206E756D62651C
:10B4A500722021202831202D202562642920202387
:10B4B50031207761732073656C65637465642066FC
:10B4C5006F72204C434420646973706C61790D0A76
:10B4D5000025632025303262643A25303262643AB1
:10B4E5002530326264200025352E31662F252D3614
:10B4F5002E316625362E31662F252D362E316625C1
:10B50500362E31662F252D362E316625362E31669F
:10B515002F252D362E31660025362E31662F252D09
:10B52500362E31660D0025303262643A253032629E
:10B53500643A25303262642563252D377300415AFC
:10B545002025332E316620454C25322E31662020AC
:10B555002020000D0A25730D0A00256320253032B1
:10B5650062643A25303262643A25303262640025DD
:10B57500382E326625382E326625392E3166253924
:10B585002E316625372E316625382E316625372E24
:10B595003166252B362E3066002F252D352E30664B
:06B5A500200D00412533DA
:10B5AB002E3066204525322E3066205025332E3125
:10B5BB00662020202000415A2025332E316620455D
:10B5CB004C25322E3166202020202000070D0A0D3D
:10B5DB000A20205B5072696F7220536174656C6C2A
:10B5EB0069746520252D397320697320414F535D94
:10B5FB000D0A0051525820466C69702063686563D0
:10B60B006B2E2E00070D0A0D0A09526F7461746FB1
:10B61B0072204572726F7220617420253032626421
:10B62B003A25303262643A25303262640D0A09439E
:10B63B006865636B20616E6420706F776572206F35
:10B64B006E20726573657420666F722073797374E4
:10B65B00656D207265636F766572792E0D0A0052E7
:10B66B006F7461746F72204572726F7220212000AB
:10B67B00436865636B207468652073797374656DBB
:10B68B00000709457869742066726F6D20457272E8
:10B69B006F72206D6F646520617420253032626497
:10B6AB003A25303262643A25303262640D0A0A0060
:10B6BB000D0A665F6C6F732F665F616F732F665F2A
:10B6CB00646966662F70756C73653A256C642F25FB
:10B6DB006C642F256C642F256C640D0A005550206B
:10B6EB0070756C73653A0044574E2070756C7365BA
:10B6FB003A002A005F004642253031316C753B0021
:10B70B00002530394C640000253031306C75000059
:10B71B004641253031316C753B00004443303B00D2
:10B72B004443313B004D442562643B0000464E30A0
:10B73B003B00464E313B00414F2D30370000464F0A
:10B74B002D32390000534F2D333300000D0A0D0AF3
:10B75B000009312E44697265637420726F746F72C5
:10B76B0020636F6E74726F6C2066726F6D206B65E9
:10B77B007920626F6172642E0D0A0009322E456EBC
:10B78B0074657220646972656374696F6E2076618B
:10B79B006C75652E0D0A0009332E50726573657436
:10B7AB0020436F6E74726F6C2E0D0A0D0A000D091B
:10B7BB0053656C6563745B312D332C515D3A2000FE
:10B7CB000D0A0D0A094C6566742834292C20526920
:10B7DB006768742836292C2055702838292C20446A
:10B7EB00776E2832292C2053746F70283529206FDF
:10B7FB0072205265742E0D0A0D0A000D0A0D0A09EE
:10B80B00417A696D7574683A2025322E3166000DC8
:10B81B000A09456C65766174696F6E3A2025322E84
:10B82B003166000D0A0D0A09313A25352E31662F86
:10B83B00252D342E316620323A25352E31662F25B3
:10B84B002D342E316620333A25352E31662F252D9A
:10B85B00342E316620343A25352E31662F252D3482
:10B86B002E31660020353A25352E31662F252D34A5
:10B87B002E3166000D0A0D0A0953656C6563745B06
:10B88B00312D352C532C515D3A20000D0A09507285
:10B89B006573657420706F736974696F6E202564AE
:10B8AB002020417A3A25352E3166000920202020B0
:10B8BB002020202020202020202020202020204558
:10B8CB006C3A25352E31660009415A3D25346420EA
:10B8DB002F2025332E316664656709454C3D253491
:10B8EB0064202F2025332E31666465672E2020209F
:10B8FB00200D000D0A0D0A0954686973206D656EE1
:10B90B007520636F6E66696775726573204144437A
:10B91B002076616C756520666F7220746865206D8A
:10B92B0069632D636C69636B20636F6E74726F6CEC
:10B93B000D0A000D0A09536574206E657720766138
:10B94B006C7565206F72204D656173757265204152
:10B95B0044432076616C7565203F205B532F4D5D12
:10B96B0020000D0A094D6F64656D206C6F636B656C
:10B97B00642063656E746572204144432076616C6C
:06B98B007565203A20253D
:10B99100346400095265666572656E6365204144D1
:10B9A100432076616C7565202020202020202020F6
:10B9B10020203A20253464000D0A0954756E652053
:10B9C1005258206672657175656E637920746F20B7
:10B9D1006D6F64656D206C6F636B656420706F7350
:10B9E1006974696F6E205B592F4E5D20000D0A0945
:10B9F1005075736820446F776E206D69632D636C99
:10BA010069636B20627574746F6E2074776F207434
:10BA1100696D6573205B592F4E5D20000D0A094544
:10BA21006E746572205374657020667265717565F8
:10BA31006E6379205B487A5D3A00094672657175DB
:10BA4100656E6379207365742043415420636F6D83
:10BA51006D616E6420617420414F53203F205B591A
:10BA61002F4E5D20000D0A094175746F6D61746977
:10BA7100632075702070756C73652067656E6572E3
:10BA81006174696F6E20617420414F53203F205BC8
:10BA9100592F4E5D20000D0A09506F726C61726959
:10BAA1007479206F6620737465702070756C73658E
:10BAB1002C204E6F726D616C2F52657665727365C5
:10BAC100203F205B4E2F525D0009094144432076FF
:10BAD100616C7565203D2534642F3130323320206F
:10BAE100200D000D0A0D0A2020414443207370618E
:10BAF1006E2076616C7565202020415A3A202530F0
:10BB01003464202D20253034642020454C3A2025F2
:10BB1100303464202D20253034640D0A000D0A20B4
:10BB21002053657420666C6970206D6F6465206FA9
:10BB31007065726174696F6E20666F7220656C65E5
:10BB4100766174696F6E20726F746F72000D0A20D6
:10BB510020526F746174652074686520616E74652C
:10BB61006E6E6120746F2066756C6C79204343574B
:10BB710020616E6420456C65766174696F6E206D1D
:10BB8100696E696D756D20706F736974696F6E0090
:10BB91000D0A2020526F74617465207468652061FC
:10BBA1006E74656E6E6120746F2066756C6C7920A1
:10BBB100435720616E6420456C65766174696F6ED0
:10BBC100206D6178696D756D20706F736974696F2F
:10BBD1006E000D0A09414443207370616E20766145
:10BBE1006C7565202020415A3A2025303464202D7F
:10BBF100202530346420000D0A09415A206D696EF8
:10BC0100696D756D2076616C7565203F203A200065
:10BC11000D09415A206D6178696D756D2076616CF1
:10BC21007565203F203A20000D0A0953657420668E
:10BC31006C6970206D6F6465206F706572617469E5
:10BC41006F6E20666F7220656C65766174696F6EC8
:10BC510020726F746F72000D0A0D0A09414443206E
:10BC61007370616E2076616C7565202020454C3AB9
:10BC71002025303464202D202530346420000D0A25
:10BC810009454C206D696D696D756D2076616C7526
:10BC910065203F203A20000D09454C206D617869EF
:10BCA1006D756D2076616C7565203F203A20000D21
:10BCB1000A0D0A0953657420416E74656E6E612028
:10BCC1005061726B696E6720706F736974696F6E12
:10BCD100203F205B592F4E5D2020000D0A0D0A09DF
:10BCE100417A696D75746820205061726B696E6765
:10BCF100202076616C7565203A2025332E3166004F
:10BD010009456C65766174696F6E205061726B696B
:10BD11006E672076616C7565203A2025332E316679
:10BD2100000D0A0953657420545258206D6F6465E3
:10BD31002F667265712E20696E207061726B696E5B
:10BD410067203F205B592F4E5D2020000D0A0D0A10
:10BD5100095258207061726B696E67206672657155
:10BD6100203A2025362E336600095458207061721E
:06BD71006B696E6720669D
:10BD7700726571203A2025362E3366000952582005
:10BD87007061726B696E67206D6F64652028462F3E
:10BD9700552F4C29203A2000095458207061726BA6
:10BDA700696E67206D6F64652028462F552F4C29D3
:10BDB700203A20000D0A0953657420416E74656EA0
:10BDC7006E6120726F746174696F6E206C696D6942
:10BDD70074203F205B592F4E5D2020000D0A0D0A6D
:10BDE70009417A696D7574682020206D696E6D75DB
:10BDF7006D202076616C7565203A2025332E3166DB
:10BE07000009417A696D75746820206D6178696DE4
:10BE1700756D202076616C7565203A2025332E31AB
:10BE2700660009456C65766174696F6E20206D69DF
:10BE37006E6D756D2076616C7565203A2025332E01
:10BE470031660009456C65766174696F6E206D61B6
:10BE570078696D756D2076616C7565203A2025339C
:10BE67002E3166000D0A0953657420726F746F7264
:10BE770020736D6F6B652070726F74656374696F83
:10BE87006E203F205B592F4E5D2020000D0A09547C
:10BE9700696D656F75742076616C756520666F7264
:10BEA70020726F7461746F72206572726F72205B9B
:10BEB7007365635D203A20253364000D0A094175D7
:10BEC700746F207265636F766572792074696D652A
:10BED7002066726F6D206572726F72206D6F646578
:10BEE700205B312D3631206D696E5D203A20253378
:10BEF70064000D0A0D0A09417A696D75746820207E
:10BF070020446561642042616E6420203A20253216
:10BF17002E31660009456C65766174696F6E204441
:10BF27006561642042616E6420203A2025322E31FB
:10BF370066000D0A09417A696D75746820202053DF
:10BF47006B65772076616C7565203A2025322E3136
:10BF5700660009456C65766174696F6E20536B6581
:10BF6700772076616C7565203A2025322E31660080
:10BF77004B454E574F4F44005941455355202000DC
:10BF870049434F4D20006E6F6E65004C534200557C
:10BF9700534200435700464D00414F530046756CCE
:10BFA7006C000943616C6C7369676E3A20257320D6
:10BFB700204C61743A2025352E316620204C6F6E57
:10BFC700673A2025352E31662020486569676874F1
:10BFD7003A2025352E31660D0A0009414443207366
:10BFE70070616E2076616C756520202020415A3A79
:10BFF70020253564202D202535642020454C3A2006
:10C00700253564202D20253564200028466C69706D
:10C01700290009446561642062616E642020202044
:10C027002020202020415A3A2025352E3166202015
:10C037002020202020202020454C3A2025352E3155
:10C0470066200D0A0009536B6577202020202020E9
:10C057002020202020202020415A3A2025352E312B
:10C067006620202020202020202020454C3A202513
:10C07700352E3166200D0A0009416E74656E6E61BA
:10C08700207061726B696E67202020415A3A202523
:10C09700352E316620202020202020202020454CCE
:10C0A7003A2025352E3166200D0A000954525820B2
:10C0B7007061726B696E6720202052583A25362EC0
:10C0C7003366202054583A25362E336620202052D6
:10C0D70058206D6F64653A257320205458206D6F82
:10C0E70064653A25730D0A0009545258202070617F
:10C0F700726B696E672020202020204F66660D0A2C
:10C107000009416E74656E6E61207061726B696EB5
:10C11700672020204F66660D0A0009526F7461740C
:10C127006F72206C696D69742020202020415A3A73
:10C137002025352E3166202D2025352E31662020ED
:10C14700454C3A2025352E3166202D2025352E31B8
:06C1570066200D0A00093C
:10C15D00526F7461746F72206C696D697420202048
:10C16D0020204F66660D0A0009526F7461746F725C
:10C17D0020737461727420454C3A25352E3166203A
:10C18D00202050312E365F6F6E20454C3A25352ECE
:10C19D00316620202050312E365F6F666620454C6B
:10C1AD003A25352E3166200D0A0009526F746174DF
:10C1BD006F7220736D6F6B652070726F7465637431
:10C1CD00696F6E094F66660D0A000954696D656FDA
:10C1DD0075742076616C756520666F7220726F7450
:10C1ED0061746F72206572726F723A20253364200C
:10C1FD007365632E0D0A00094175746F20726563B6
:10C20D006F766572792074696D652066726F6D2029
:10C21D00726F746F72206572726F723A202533647B
:10C22D00206D696E2E0D0A00094341542052696735
:10C23D002020202020202020202020257320257341
:10C24D0000202054533731312F3831310020204612
:10C25D00542D37333600202046542D383437002FD7
:10C26D00464D4E2D46696C7465720020202825427E
:10C27D005829282542582928773D2564290020254D
:10C28D0073000D0A095374657020636F6E74726FBD
:10C29D006C204144432076616C7565202043656EAA
:10C2AD007465723A2535642020526566663A2535E7
:10C2BD0064000D0A094672657175656E63792073A8
:10C2CD0074657020202020256C64487A000D0A09C1
:10C2DD00526F746F7220737461727420202020204D
:10C2ED0020202573000D0A09434F4D20706F727485
:10C2FD002020202020202020202025732042617521
:10C30D006420382D4E2D310D0A000D0A0909507289
:10C31D0065737320616E79206B657920746F20636E
:10C32D006F6E74696E7565000D0A2534642F2530A6
:10C33D003262642F25303262642025303262643AD5
:10C34D0025303262643A25303262640D0A0053742E
:10C35D00617274696E67204461792F54696D65202F
:10C36D003F205B59592F4D4D2F44442048483A4D9D
:10C37D004D3A53535D2000446179206F66207468F7
:10C38D00652059656172205B545D203E2025352E58
:10C39D0035660D0A0054696D6520537465700D0A7C
:10C3AD0000094D696E205B315D3A200009536563CC
:10C3BD00205B305D3A200020202535732020202081
:10C3CD002535732020202020202025337320202F79
:10C3DD002533732020202020253573253130730D12
:10C3ED000A00444154450054494D4500415A004509
:10C3FD004C00506861736500446F70706C6572001D
:10C40D00253034642F25303262642F25303262643A
:10C41D002025303262643A25303262643A2530325A
:10C42D0062642020202025352E31662F25342E31B3
:10C43D006625392E3166252B392E30660D0A002AD8
:10C44D002A2A2A2A2A2A2A2A2A0A0D00092D2D2DBE
:10C45D002027512720666F722061626F727420272A
:10C46D00532720666F72207363726F6C6C202D2DB5
:10C47D002D000A0D07546F6F206F6C6420656C657D
:10C48D006D656E74732E200D0A000D0A0A09557024
:10C49D006C6F6164204B6570656C652064617461BF
:10C4AD002066696C652E2028454F463A6374726C80
:10C4BD002B5A290D0A00070D0A09525320427566A1
:10C4CD006665722046756C6C20210D0A004E415335
:10C4DD00413E232533640925730D0A000D0A0953C6
:10C4ED006174656C6C6974652028257329207365EA
:10C4FD006C656374656420617320232562640D0A85
:10C50D00002532642E2A252D313473200025326406
:10C51D002E20252D31347320000D0A0953656C65CD
:10C52D0063743A002532642E2563252D3134732032
:06C53D0000202020202058
:10C543002020000D0A0907536174656C6C697465DA
:10C55300206973206E6F7420617369676E65642E42
:10C5630020476F20746F206D656E7520332D320D5B
:10C573000A002000000D0A0A0955706C6F616420DF
:10C58300667265712F6D6F646520646174612066E6
:10C59300696C652E2028454F463A6374726C2B5A9A
:10C5A300290D0A0025732025732025732025732068
:10C5B300257320257320257320257300536174652B
:10C5C3006C6C697465202825387329207570646143
:10C5D30074656420616E642073656C65637465645F
:10C5E3002061732023253262640D0A000D0A0D0AAF
:10C5F3000955706C6F61642053746174696F6E20A8
:10C60300696E666F2E20646174612066696C652EA5
:10C613002028454F463A6374726C2B5A290D0A0041
:10C62300252A63202573202566202566202566207C
:10C63300257320256400252A632025642025642092
:10C64300256420256420257300252A632025662080
:10C65300256620256620256600252A63202573206C
:10C663002573202568782025687820256420256493
:10C6730000252A632025732025662025662025664C
:10C6830020256620256600252A632025732025663C
:10C69300202566202573202573202564202564002A
:10C6A300252A6320257320256620256620256620FC
:10C6B3002566000D0A0953746174696F6E20696EF3
:10C6C300666F726D6174696F6E20757064617465F5
:10C6D300642E0D0A00070D0A094572726F7220213C
:10C6E30020757064617465206E6F7420636F6D7064
:10C6F3006C657465642E0D0A000D0A0D0A5472618F
:10C703006B426F7820686F7374206D6F64652E00C1
:10C713000D0A436F6D6D616E643A4D557878782CD0
:10C723004D447878782C46557878782C4644787838
:10C73300782C415A7878785F454C78782C53787800
:10C74300782C5478782C512C3F412C3F0D0A0054FF
:10C7530072616B426F7820486F73746D6F6465000C
:10C7630000202020202020202020202020202020E6
:10C773002000000D0A5472616B426F783E3E200028
:10C7830025732025730046555F202020202020207C
:10C79300202020202020000046445F20202020204D
:10C7A30020202020202020200000467265712E20AA
:10C7B300666F726D6174206572726F72202120281A
:10C7C30065782E2046553134353930303030290DD7
:10C7D3000A00465F666F726D6174206572726F72D4
:10C7E3002000004D6F6465206572726F72202020F7
:10C7F300202000004D6F6465206572726F722021E6
:10C80300202865782E204D554C2F4D55552F4D55CD
:10C8130046290D0A004D6F6465206572726F7220A0
:10C823002120202000004D6F6465206572726F72B5
:10C833002021202865782E204D444C2F4D44552F20
:10C843004D4446290D0A004D6F646520666F726D75
:10C853006174206572726F722021202865782E2002
:10C863004D554C53422C4D44464D290D0A004D5F06
:10C87300666F726D6174206572726F722000004181
:10C883007A2F456C20666F726D6174206572726FCA
:10C89300722021202865782E20417A3037352045B3
:10C8A3006C3135290D0A00417A5F666F726D6174D0
:10C8B300206572726F72200000547261636B2023D3
:10C8C300204572726F7220210D0A000D0A436F6DAD
:10C8D3006D616E643A4D557878782C4D447878784C
:10C8E3002C46557878782C46447878782C415A78B9
:10C8F30078785F454C78782C537878782C5478780E
:10C903002C3F412C3F2C510D0A00436F6D6D616E1E
:10C9130064206572726F722021200D0A00436F6DCF
:06C923006D616E642065E9
:10C9290072726F722020200000FFA22DFFA25FFF0C
:10C93900A28BFFA2B7FFA2E3FFA2F5FFA307FFA8FF
:10C9490007FFA80DFFA813FFA818FFA81DFFA8221D
:10C95900FFA827FFA82CFFA832FFA844FFA856FF6D
:10C96900A868FFA87AFFA88CFFAAEEFFAAF3FFAA7E
:10C97900FEFFAB01FFAB05FFAB19FFAB2DFFAB41D1
:10C98900FFAB55FFAB69FFAB7DFFAB91FFABA5FFDC
:10C99900ABB9FFABCDFFABE1FFABF5FFAC09FFAC2A
:10C9A9001DFFAC31FFAC45FFAC59FFAC6DFFAC814D
:10C9B900FFAC95FFAC9AFFAC9FFFACA4FFACA9FFFD
:10C9C900BF77FFBF7FFFBF87FFA807FFA80DFFBF86
:10C9D9008DFFBF92FFBF96FFBF9AFFBF9DFFBFA00C
:10C9E900FFBFA4FFA813FFA818FFA81DFFA822FFD7
:05C9F900A827FFA82C97
:10C9FE004A66A7FA00FD00FE80FF40FFA0465D7B61
:10CA0E0040D0E8F4FAFD5A65AF001F1C1F1E1F1E12
:10CA1E001F1F1E1F1E1F001F1D1F1E1F1E1F1F1E3E
:10CA2E001F1E1F60784EC73E8D06BC3E8CAFD53E96
:10CA3E008DBFCF3E8D68E83E8D12023E8CBB1B3EF5
:10CA4E008DCB143E8D742E3E8D1D263E8CC63F3EE4
:10CA5E008DD6393E8D7F523E8D286B3E8CD1853ED4
:10CA6E008DE17E3E8D8A983E8D33B13E8CDCCA3E82
:10CA7E008DECA23E8D95BC3E8D3ED53E8CE7EF3EB5
:10CA8E008DF7E83E8DA1013E8D4A1B3E8CF3343E60
:0FCA9E008E032E3E8DAC263E8D553F3E8CFE58AE
:10000300E49067D8F01201F378967C4E7D017BFF74
:100013007AA3791912D6E1EF600F1202B21201F33B
:100023007BFF7AA3791F120C439065FAE030E30952
:1000330090E102E04450F0800790E102E054AFF019
:100043009065F9E054DFF07F307E7512084D90C95A
:100053003E12D43D1208C17FC012050190C944125B
:10006300D43D1208C11208667F007E007DC67C4322
:1000730090655512D38812CDC3600B40097BFF7A7C
:10008300A379311208A312087C9067D9EFF060605E
:100093009054E7E04401F0A3E0F07BFF7AA37948B2
:1000A3001208A390E102E054F0F012087C9067D9A3
:1000B300EFF014FF90665BF03395E0FE74682FF564
:1000C30082EE3466F583E0C36480948040069067D3
:1000D300D9E0700A12087C9067D9EFF080C590547C
:1000E300E7E0A330E10512261880B8122B3280B363
:1000F3009054E7E054FEF012086690E102E054F0F9
:10010300F09054E7E054FDF09065F9E04404F0A367
:10011300E0F09054E7E0A330E4089067D87407F068
:100123008008120CC19067D8EFF09067D8E012D422
:1001330049015601018B0201BE0301C40401CA0532
:1001430001D00601D60701DC0801E26D01567300F8
:100153000000FA7BFF7AA3794C1208A3128A23903A
:1001630067DAEFF0F46090906770E0FF9067DAE091
:10017300FD3395E0FCC3ED9F7480F86C9840030257
:1001830000FA122B320200FA7BFF7AA37975120868
:10019300A3128A239067DAEFF0F470030200FAE007
:1001A300FF3395E0FE74682FF582EE3466F583E045
:1001B300FF3395E0FE1278FC0200FA120E020200F1
:1001C300FA120FF20200FA1213370200FA12214553
:1001D3000200FA129C360200FA1260C70200FA907B
:1001E30054E7E04402F0A3E0F01226180200FA22DA
:1001F30090E2017403F090E1037482F090E100E473
:10020300F0759852758922758850C2CAC28EA3E0D0
:1002130020E705758DD080289056E5E0FFC3940054
:100223004006EFD39405400B9056E57404F0758DAA
:10023300FA800D747B2FF582E4345DF583E0F58D50
:1002430075C8049065FCE025E024A7F582E43466D4
:10025300F583E0FCA3E0FDECF5CBF5CDEDF5CAF5B8
:10026300CCD2CAD28E90E00FE054046404601F7BAA
:10027300FF7AA3799E1208A390E00F7407F0740429
:10028300F090E00DE054FEF090E00F7404F07F383E
:100293001205017F381205017F0C1205017F06123A
:0F02A30005017F0112050190E00DE054FBF022F0
:1002B2007BFF7AA379A01208A3E49065FBF0906516
:1002C200F9F0A3F09054E7F0A3F01205C8125DC74D
:1002D200787D7C4E7D017BFF7AA379D77E007F07F4
:1002E20012D55878967C4E7D017BFF7AA379DF7E0A
:1002F200007F0612D55890E101E020E705758DE8F0
:1003020080069056E57404F09065FC7402F090E06B
:100312000F7407F07404F090E00DE054FEF090E0EA
:100322000F7404F0E490676AF0A3F09055DD12D3E5
:10033200B041DB20C59055E112D3B04300A8317F14
:10034200007E007D007C009055E112D38812CDC35F
:10035200600250197F007E007D807CBF9055E112C3
:10036200D38812CC219055E512D3A480179055E181
:1003720012D3887F007E007DB47C4312CB2C905533
:10038200E512D3A49055E912D3B04248000090661A
:100392000F12D3B00000000090660B12D3B0000021
:1003A200000090661312D3B040400000906617120E
:1003B200D3B03F8000009066B1E4F0A3740BF090DC
:1003C20000157403F0A3746AF0906601E4F0A3745C
:1003D20002F090676804F0A374ACF0904F3F12D320
:1003E200B0000000009055F112D3B0000000009060
:1003F20065D112D3B0000000009065CD12D3B000D9
:100402000000009066637404F0906662F09066618A
:10041200F0906660F09065D912D3B00000000090B1
:1004220065DD12D3B043B400009065E112D3B00091
:100432000000009065E512D3B042B40000904EBEB9
:1004420012D3B0C0000000905F8712D3B0C0A000EA
:1004520000904F4312D3B0C0C00000E490665BF03E
:10046200904EC27403F090655D12D3B0000000009C
:1004720090674B12D3B00000000AE4905D7AF090CE
:100482000005742EF090677DF090000CF090000053
:10049200F0904E95F0904E78741EF090000AE4F0C1
:1004A200A37432F09000177401F090674F04F0903B
:1004B20065ED12D3B00000006490659D7402F0A354
:1004C2007426F09060837402F0A37430F09066A5F5
:1004D200E4F0A3743DF0905D81E4F0A37478F090B1
:1004E20054E77468F0A37440F09065F9740DF0A3BA
:0F04F2007483F0A3E04401F054FDF012052B22B7
:10050100C292C29190E100EFF07F0A7E0012084D85
:05051100D290C290220F
:10051600D292C29190E100EFF07F0A7E0012084D60
:05052600D290C29022FA
:10052B009066B1E0FEA3E0FFC3900016E09FFF9042
:10053B000015E09EFE12E751AC06AD07EC12CE465D
:10054B007B007A0079B4784312CD2A9066B312D32C
:10055B00A49065F9E0A330E632906601E0FEA3E0DB
:10056B00FFC3906769E09FFF906768E09EFE12E70C
:10057B0051AC06AD07EC12CE467B007A007934788D
:10058B004312CD2A90660712D3A422906601E0FE97
:10059B00A3E0FFC3906769E09FFF906768E09EFE52
:1005AB0012E751AC06AD07EC12CE467B007A007910
:0D05BB00B4784212CD2A90660712D3A42214
:1005C800E4F50874612508F582E43465F583E4F000
:1005D800741F2508F582E43466F583E4F0E5082500
:1005E800E025E02496F582E4345BF58312D3B0006D
:1005F800000000E50825E025E02483F582E4345D69
:10060800F58312D3B000000000E50825E025E024BA
:1006180037F582E43450F58312D3B000000000E5CA
:100628000825E025E024EDF582E43454F58312D35F
:10063800B000000000E50825E025E024B6F582E4D6
:100648003459F58312D3B00000000074F32508F57F
:1006580082E4345EF583E4F0E50825E025E024A68D
:10066800F582E4345AF58312D3B000000000E5089F
:1006780025E025E024C6F582E43458F58312D3B08A
:1006880000000000E50825E02473F582E4345EF5F7
:1006980083E4F0A3F0E50825E025E0248AF582E468
:1006A800345CF58312D3B03F800000E50825E025CF
:1006B800E024F5F582E43455F58312D3B000000048
:1006C8000175F010E50890513312D3E112D3B00050
:1006D80000000075F010E50890512F12D3E112D3F5
:1006E800B00000000075F010E50890512B12D3E11E
:1006F80012D3B00000000075F010E50890512712E1
:10070800D3E112D3B000000000E50825E025E0247D
:1007180047F582E4344FF58312D3B000000000E5BA
:100728000825E025E02493F582E4345FF58312D3AD
:10073800B000000000E50825E025E024D6F582E4B5
:100748003457F58312D3B000000000E50825E025F2
:10075800E024E6F582E43456F58312D3B0000000B5
:1007680000E50825E024BCF582E43466F583E0540E
:10077800FBF0E50825E024BCF582E43466F583E067
:1007880054FEF0E50825E024BCF582E43466F583E0
:10079800E054FDF0E50825E024BCF582E43466F574
:1007A80083E054EFF07E007F14C006C0077D00E5AB
:1007B8000875F014A424A1F9746035F0FA7B01D00F
:1007C80007D00612D46F0508E508643C60030205EB
:1007D800CBE4F50874682508F582E43466F583747B
:1007E800FFF00508E508B43CEBE4F508E50825E06A
:1007F80025E02473F582E4345FF58312D3B000005A
:100808000000E50825E025E0248DF582E43460F554
:100818008312D3B0000000000508E508B405CD2216
:1008280090676AE0FEA3E0FFC3EF9420EE944E5079
:1008380013741E2FF582EE3400F583E4F00FBF0029
:05084800010E80E42216
:10084D00E4FDFCEF2401FBE43EFAC3ED9BEC9A5072
:09085D00070DBD00010C80EB2227
:10086600124538904EC312D36C90673312D3A490BE
:06087600676C12D3A422FE
:10087C009065F9E0A320E40990E101E0F4540FFF46
:10088C00227F02120C7BE52DAE2C7806CEC313CE44
:07089C0013D8F9540FFF22ED
:1008A3008B088A09890A7808E475F00112D3ED12DE
:0E08B300D0F8F50B6007AF0B12E6F980E922D2
:1008C1008B088A09890A7808E475F00112D3ED12C0
:0E08D100D0F8F50B6007AF0B12051680E92278
:1008DF008B088A09890A7808E475F00112D3ED12A2
:1008EF00D0F8F50B6009E4FFAD0B12CAAE80E7221A
:1008FF008B088A09890A7808E475F00112D3ED1282
:0E090F00D0F8F50B6007AF0B12CAD280E922B8
:10091D0090690E12D434E4906911F0A3F012E7201F
:10092D008F22E522640D6050E522640A604AE522BB
:10093D006408600FE522B47F24906911E07002A372
:10094D00E0601A90690E74FFF5F012D406E412D12E
:10095D003E90691174FFF5F012D19A80C090690E26
:10096D00E475F00112D406E52212D13E906911E42E
:10097D0075F00112D19A80A590690EE475F00112FF
:0F098D00D406E412D13E906911E0FEA3E0FF22F0
:10099C001208A37B017A68794D12091D90684A12DE
:1009AC00D3FDE4F5F012D1C67B017A68794D12E8DB
:1009BC000E90684A12D3FDEE8FF012D1C67B017AED
:0709CC0068794D12E94D228C
:1009D3001208A37B017A6879BE12091D9068BB12C5
:1009E300D3FDE4F5F012D1C67B017A6879BE12E833
:1009F3000E9068BB12D3FDEE8FF012D1C67B017A45
:070A03006879BE12DFD92261
:100A0A0090693C12D3A47F007EFE7DFF7C469069EC
:100A1A004012D38812CDC3600250517F007E007D00
:100A2A00007CC790694012D38812CDC3403E9069BA
:100A3A004012D36C12CE7FAC06AD07EC12CE4690B4
:100A4A00694012D38812CDC3702290694012D36CC8
:100A5A0012CE7F906950EEF0A3EFF090693C12D36A
:100A6A006C120AC590694812D3A480487F007E00A0
:100A7A007D007C0090693C12D38812CDC3602B4064
:100A8A002990693C12D36C12E0F090694412D3A405
:100A9A0090694012D36C90694412D38812CC211207
:100AAA00E05A90694812D3A4800A90694812D3B0D8
:0B0ABA000000000090694812D36C227D
:100AC50090694C12D3A4906950E0FEA3E0FF12E7B1
:100AD50051906952EEF0A3EFF0A312D3B03F80001E
:100AE50000906952E0FEA3E0FF4E603BEF30E0135B
:100AF500A312D36C90694C12D38812CC21906954FF
:100B050012D3A490694C12D36CA804A905AA06AB0C
:100B15000712CC2190694C12D3A4906952E0C313FB
:100B2500F0A3E013F080BAC3906950E0648094802C
:100B3500400E90695412D36C90695812D3A4801753
:100B450090695412D3887F007E007D807C3F12CD52
:0E0B55002A90695812D3A490695812D36C22CA
:080B630012CE7FEC12CE4122FC
:100B6B0090693C12D3A490693C12D36C12CE7FAC2B
:100B7B0006AD07EC12CE4690694012D3A4906940A3
:100B8B0012D38890693C12D36C12CB2C12DFCC7B26
:100B9B00BD7A377986783512CDC350197F007E0028
:100BAB007D807C3F90694012D38812CB3090694492
:100BBB0012D3A4800C90694012D36C90694412D369
:080BCB00A490694412D36C22CE
:100BD3001208A37BFF7AA379E61208A312E720AEDB
:100BE30007EE4420FDBD79037F0122BD6E037F0024
:040BF300227FFF223C
:100BF70090E00DE04401F0E030E11090E00DE054AA
:0C0C0700FEF07F0A7E0012084D80E522FE
:100C1300120BF7E4FFEFFDC3740B9DFD74E094002A
:100C2300FC8D82F583E0540F4430FE74302FF8A618
:100C3300060FBF0CE0E4F53C90E00DE054FEF0221B
:100C43009067FA12D4347F10E4FEFD9067FA12D352
:100C5300FD8F8275830012D11124D0FCE42DF5821F
:100C6300E434E0F583ECF01F0EEEC394024003E49A
:080C7300FE1F0DEDB40CD422AC
:100C7B00EF540790E200F07F1E7E0012084DA3E0B8
:100C8B00FF90E200E0FDEF7F00FEEDFFE4EF780662
:100C9B00CEC313CE13D8F9FFEE5403F52C8F2D22B0
:100CAB007BFF7AA379F01208A330980412E7202275
:060CBB0012648080F422A7
:100CC10090C93212D43D1208A390C93512D43D12F5
:100CD10008A390C93812D43D1208A390C93B12D47D
:100CE1003D1208A37F8012050190C93E12D43D1226
:100CF10008C17FC012050190C94112D43D1208C13B
:100D01007BFF7AA479221208A37BFF7AA47942128D
:100D110008A37BFF7AA4795B1208A37BFF7AA479ED
:100D2100731208A37BFF7AA479941208A37BFF7A3C
:100D3100A479B31208A37BFF7AA479D01208A37B0C
:100D4100FF7AA479E51208A37BFF7AA479F6120849
:100D5100A37BFF7AA579161208A330982F12E720FA
:100D6100AE07EEC39430400BEED394385005EE2419
:100D7100D0FF22EE4420FDBD73037F7322BD6D03BE
:100D81007F6D227BFF7AA579161208A39054E7E0C4
:100D9100FEA3E0FF30E4C330E2C07F011236588089
:020DA100B92275
:100DA3007BFF7AA5792C1208A37BFF7AA5795512CC
:100DB30008A37BFF7AA579891208A37BFF7AA5791B
:100DC300BC1208A37BFF7AA579F11208A37BFF7AF3
:100DD300A679141208A37BFF7AA6794F1208A312EF
:100DE300E720AE07EEC39431400BEED394355005A4
:0F0DF300EE24D0FF22EE4420FFBF71DA7F712281
:100E0200120DA39067DEEFF024FE604C1470030213
:100E12000F23147003020F23147003020FA62494ED
:100E22007003020FF1247070D77BFF7AA6795B12F0
:100E320008A3128A239067DBEFF0F460C3E0FF336C
:100E420095E0FE74682FF582EE3466F583E0FF3399
:100E520095E0FE12146380A87BFF7AA67982120BBA
:100E6200D39067DCEFF0D3648094804093E4906782
:100E7200DDF09067DDE0FFC3943C5018EF25E024DD
:100E8200BCF582E43466F583E054EFF09067DDE070
:100E920004F080DE7BFF7AA679B11208A37BFF7A89
:100EA200A679DD1208A37BFF7AA779111208A37B2A
:100EB200FF7AA6794F1208A312E720EF24CE601022
:100EC20014605824026003020E02128813020E02FA
:100ED200E49067DDF09067DDE0FF904EA4E0FCA3B4
:100EE200E0FDC3EF9DE49C502C9067DDE02468F5A3
:100EF20082E43466F583EFF0EF25E024BCF582E46A
:100F02003466F583E04410F09067DDE004F0E09091
:100F12006770F080C0128B9F020E02128C2E020E9E
:100F2200029067DEE0B403217BFF7AA77941120BBE
:100F3200D39067DCEFF0D3648094805003020E02FA
:100F4200E490676AF0A3F080229067DEE0B4041BAD
:100F5200C3904EA5E0943C904EA4E09400400C7BDC
:100F6200FF7AA779781208A3020E027BFF7AA7798B
:100F7200931208A312E720E49067DDF09067DDE0AA
:100F8200FFC3943C5018EF25E024BCF582E434669C
:100F9200F583E054EFF09067DDE004F080DE12802C
:100FA200E0020E027B017A6779DF90684A12D4343C
:100FB2007BFF7AA779AF12099C9067DEEFF0C394AA
:100FC200024016E0FFD39405500F904EA4E0FCA31C
:100FD200E0FDD3EF9DE49C400B7BFF7AA779F412EE
:100FE20008A380C09067DEE0904EC2F0020E02229B
:100FF20078EB7C677D017BFF7AC979477E007F06AB
:1010020012D55878F17C677D017BFF7AC9794D7ED4
:10101200007F1212D55878037C687D017BFF7AC964
:10102200795F7E007F1212D5589054E7E0FFA3E06B
:10103200906815CFF0A3EFF07BFF7AA8799E120893
:10104200A37BFF7AA879C81208A37BFF7AA879FA52
:101052001208A37BFF7AA6794F1208A312E7209009
:101062006817EFF06431600EE0FF64326008EF440D
:1010720020FFBF71DE22906817E0B4320412939A07
:1010820022906817E0643160030213367BFF7AA96D
:10109200792D1208A390680312D3FD90679512D49C
:1010A200347B017A4E797D90679812D4347BFF7A33
:1010B200A9795A12D8AB7B017A6779DD12091DEF43
:1010C2004E600F787D7C4E7D017B017A6779DD125F
:1010D200D7B690680612D3FD90679512D434905516
:1010E200DD12D36C90679812D3A47BFF7AA979653D
:1010F20012D8AB7B017A6779DB9068BB12D4347B60
:10110200FF7AA979731209D39067E712D3A4906783
:10111200DBE07002A3E0600C9067E712D36C90559D
:10112200DD12D3A490680912D3FD90679512D434CE
:101132009055E112D36C90679812D3A47BFF7AA9E1
:10114200796512D8AB7B017A6779DB9068BB12D4E0
:10115200347BFF7AA979731209D39067E712D3A47B
:101162009067DBE07002A3E0600C9067E712D36C3B
:101172009055E112D3A47F007E007D007C00905543
:10118200E112D38812CDC350197F007E007D807C8E
:10119200BF9055E112D38812CC219055E512D3A409
:1011A200802A7F007E007D007C009055E112D3886A
:1011B20012CDC340179055E112D3887F007E007D87
:1011C200B47C4312CB2C9055E512D3A490680C1238
:1011D200D3FD90679512D4349055E912D36C906781
:1011E2009812D3A47BFF7AA9797512D8AB7B017AC6
:1011F2006779DB9068BB12D4347BFF7AA9797312CA
:0812020009D39067E712D3A4A1
:10120A009067DBE07002A3E0600C9067E712D36C92
:10121A009055E912D3A490680F12D3FD90679512E6
:10122A00D434E4FE906816E054087803CEC313CE93
:10123A0013D8F99067EB75F00312D3E1EE75F0035A
:10124A00A42583F58312D3FD90679812D4347BFFCB
:10125A007AA9798212D8AB7B017A6779DD12091DE6
:10126A009067DDE04420FFBF6E099054E8E044082F
:10127A00F0800ABF73079054E8E054F7F09067DEF5
:10128A00E04420FFBF610C9065F9E04410F0A3E050
:10129A00F080079065F9E054EFF090681212D3FDE0
:1012AA0090679512D4349056E5E075F003A424F1C2
:1012BA00F582E43467F58312D3FD90679812D4342B
:1012CA007BFF7AA9798E12D8AB7B017A6779DB909A
:1012DA00684A12D4347BFF7AA9797312099CBE0139
:1012EA0009BF2C06E49056E5F022BE040ABFB007F7
:1012FA009056E57401F022BE090ABF60079056E5D0
:10130A007402F022BE120ABFC0079056E57403F0B9
:10131A0022BE250ABF80079056E57404F022E4B580
:0D132A00070AEEB44B069056E57405F0225C
:101337007BFF7AA979981208A37BFF7AA979BE1255
:1013470008A37BFF7AA979D41208A31245387BFF3B
:101357007AAA79001208A37BFF7AAA791390679576
:10136700E53FF0A3E540F0A3E52BF0A3E528F0A3C4
:10137700E529F0A3E52AF0A3E527F012D8AB3098CA
:10138700CA12E7209067F9EFF04420FFBF79089071
:10139700E00DE04408F022EF64717003021462125A
:1013A70045387BFF7AAA79361208A37BFF7AAA7998
:1013B70063906795E53FF0A3E540F0A3E52BF0A325
:1013C700E528F0A3E529F0A3E52AF0A3E527F01225
:1013D700D8AB7BFF7AAA79871208A3E49067E0F07D
:1013E7009067DDF07B017A6779DB12091D9067E072
:1013F700E0FF9067DDE04F642F70549067E9E0FFEE
:101407009067E6E04F643A704690E00F7407F07417
:1014170004F090E00DE054FEF090E00F7404F07BD0
:10142700017A6779DB90679512D4347BFF7AAA79C2
:10143700AF12D8AB7BFF7AAA79C11208A312E720B3
:101447009067F9EFF07B017A6779DB120C43227B17
:0C145700FF7AAA79D91208A312133722D9
:101463009067E1EEF0A3EFF078617C687D017BFF8C
:101473007AC979717E007F0612D55878677C687DBA
:10148300017BFF7AC979777E007F0612D558786D84
:101493007C687D017BFF7AC9797D7E007F3C12D514
:1014A3005878A97C687D017BFF7AC979B97E007F72
:1014B3000F12D5587BFF7AAC79AE1208A390686DF2
:1014C30012D3FD90679512D4349067E1E0FEA3E058
:1014D300FF7C007D1412D15074A12FF974603EFA81
:1014E3007B0190679812D4347BFF7AAC79D312D8FE
:1014F300AB7B017A68794912091DEF4E602490672E
:10150300E1E0FEA3E0FF7C007D1412D15074A12F13
:10151300F974603EA801FC7D017B017A6879491268
:10152300D7B690689712D3FD90679512D43490671D
:10153300E2E025E0FF9067E1E033FE74732FF5826C
:10154300EE345EF583E0FFA3E0906798CFF0A3EF5E
:10155300F07BFF7AAC79DD12D8AB7B017A6779E354
:101563009068BB12D4347BFF7AAC79E41209D312AE
:10157300CE7F9067E3E07002A3E06020AC06AD0786
:101583009067E2E025E0FF9067E1E033FE74732F9C
:10159300F582EE345EF583ECF0A3EDF09068701203
:1015A300D3FD90679512D4349067E1E0FEA3E07811
:1015B30002C333CE33CED8F9248AF582EE345CF5F8
:1015C3008312D36C90679812D3A47BFF7AAC79EB28
:1015D30012D8AB7B017A6779E39068BB12D4347B72
:1015E300FF7AAC79F51209D390685D12D3A49067A2
:1015F300E3E07002A3E0603290685D12D36CC00434
:10160300C005C006C0079067E1E0FEA3E07802C30F
:1016130033CE33CED8F9248AF582EE345CF583D009
:1016230007D006D005D00412D3A490687312D3FD5B
:1016330090679512D4349067E1E0FEA3E07802C38B
:1016430033CE33CED8F924F5F582EE3455F5831233
:10165300D36C90679812D3A47BFF7AAC79FB12D832
:10166300AB7B017A6779E39068BB12D4347BFF7A52
:10167300AD79041209D390685D12D3A49067E3E0B7
:101683007002A3E0603590685D12D36C12CE7FC008
:1016930004C005C006C0079067E1E0FEA3E078023E
:1016A300C333CE33CED8F924F5F582EE3455F58322
:1016B300D007D006D005D00412D3A490687612D3F5
:1016C300FD90679512D4349067E1E0FEA3E07802C1
:1016D300C333CE33CED8F924C6F582EE3458F5831E
:0F16E30012D36C90679812D3A47BFF7AAC79EB8B
:1016F20012D8AB7B017A6779E39068BB12D4347B52
:10170200FF7AAD790A1209D390685D12D3A490676B
:10171200E3E07002A3E0603290685D12D36CC00413
:10172200C005C006C0079067E1E0FEA3E07802C3EF
:1017320033CE33CED8F924C6F582EE3458F583D0B1
:1017420007D006D005D00412D3A490687912D3FD35
:1017520090679512D4349067E1E0FEA3E07802C36B
:1017620033CE33CED8F924B6F582EE3459F583124E
:10177200D36C90679812D3A47BFF7AAC79EB12D822
:10178200AB7B017A6779E39068BB12D4347BFF7A32
:10179200AD79101209D390685D12D3A49067E3E08B
:1017A2007002A3E0603290685D12D36CC004C00581
:1017B200C006C0079067E1E0FEA3E07802C333CE23
:1017C20033CED8F924B6F582EE3459F583D007D05A
:1017D20006D005D00412D3A490687C12D3FD906782
:1017E2009512D4349067E1E0FEA3E07802C333CED1
:1017F20033CED8F924EDF582EE3454F58312D36C4E
:1018020090679812D3A47BFF7AAC79EB12D8AB7BAA
:10181200017A6779E39068BB12D4347BFF7AAD79A1
:10182200161209D390685D12D3A49067E3E07002A8
:10183200A3E0603290685D12D36CC004C005C0069C
:10184200C0079067E1E0FEA3E07802C333CE33CE57
:10185200D8F924EDF582EE3454F583D007D006D0C2
:1018620005D00412D3A490687F12D3FD906795121D
:10187200D4349067E1E0FEA3E07802C333CE33CEE6
:10188200D8F92437F582EE3450F58312D36C906781
:101892009812D3A47BFF7AAC79EB12D8AB7B017A96
:1018A2006779E39068BB12D4347BFF7AAD791C125E
:1018B20009D390685D12D3A49067E3E07002A3E0BD
:1018C200603290685D12D36CC004C005C006C007C8
:1018D2009067E1E0FEA3E07802C333CE33CED8F9BD
:1018E2002437F582EE3450F583D007D006D005D0E8
:1018F2000412D3A490688212D3FD90679512D43457
:101902009067E1E0FEA3E07802C333CE33CED8F98C
:101912002483F582EE345DF58312D36C90679812BE
:10192200D3A47BFF7AAC79EB12D8AB7B017A6779CF
:10193200E39068BB12D4347BFF7AAD79221209D3CB
:1019420090685D12D3A49067E3E07002A3E0603276
:1019520090685D12D36CC004C005C006C0079067D2
:10196200E1E0FEA3E07802C333CE33CED8F924837C
:10197200F582EE345DF583D007D006D005D004128F
:10198200D3A490688512D3FD90679512D4349067E2
:10199200E1E0FEA3E07802C333CE33CED8F9249639
:1019A200F582EE345BF58312D36C90679812D3A460
:1019B2007BFF7AAC79EB12D8AB7B017A6779E39043
:1019C20068BB12D4347BFF7AAD79281209D39068B0
:1019D2005D12D3A49067E3E07002A3E060329068E6
:1019E2005D12D36CC004C005C006C0079067E1E079
:1019F200FEA3E07802C333CE33CED8F92496F58223
:101A0200EE345BF583D007D006D005D00412D3A400
:101A120090688812D3FD90679512D4349067E1E004
:101A2200FEA3E07802C333CE33CED8F924A6F582E2
:101A3200EE345AF58312D36C90679812D3A47BFFCD
:101A42007AAD792E12D8AB7B017A6779E39068BBC5
:101A520012D4347BFF7AAD79351209D390685D12C6
:101A6200D3A49067E3E07002A3E0603290685D1255
:101A7200D36CC004C005C006C0079067E1E0FEA3B6
:101A8200E07802C333CE33CED8F924A6F582EE3401
:101A92005AF583D007D006D005D00412D3A490689B
:101AA2008B12D3FD90679512D4349067E1E0FEA3C8
:101AB200E07802C333CE33CED8F92447F582EE3430
:101AC2004FF58312D36C90679812D3A47BFF7AAD43
:101AD200793A12D8AB7B017A6779E39068BB12D46A
:101AE200347BFF7AAD79441209D390685D12D3A496
:101AF2009067E3E07002A3E0603290685D12D36CFD
:101B0200C004C005C006C0079067E1E0FEA3E0780C
:101B120002C333CE33CED8F92447F582EE344FF5E3
:101B220083D007D006D005D00412D3A49068A612A1
:101B3200D3FD90679512D4349067E1E0FEA3E0787C
:101B420002C333CE33CED8F92493F582EE345FF557
:101B52008312D36C90679812D3A47BFF7AAD794A33
:101B620012D8AB7B017A6779E39068BB12D4347BDD
:101B7200FF7AAD79541209D390685D12D3A49067AD
:101B8200E3E07002A3E0603290685D12D36CC0049F
:101B9200C005C006C0079067E1E0FEA3E07802C37B
:101BA20033CE33CED8F92493F582EE345FF583D069
:101BB20007D006D005D00412D3A49068A012D3FD9A
:101BC20090679512D4349067E1E0FEA3E07802C3F7
:101BD20033CE33CED8F924E6F582EE3456F58312AD
:101BE200D36C90679812D3A47BFF7AAD793A12D85E
:101BF200AB7B017A6779E39068BB12D4347BFF7ABE
:101C0200AD795A1209D390685D12D3A49067E3E0CC
:101C12007002A3E0603290685D12D36CC004C0050C
:101C2200C006C0079067E1E0FEA3E07802C333CEAE
:101C320033CED8F924E6F582EE3456F583D007D0B8
:101C420006D005D00412D3A490688E12D3FD9067FB
:101C52009512D4349067E2E0C4F8540FC868FB9040
:101C620067E1E0C454F048FA74272BF582EA345154
:101C7200F58312D36C90679812D3A4742B2BF58240
:101C8200EA3451F58312D36C90679C12D3A4906707
:101C9200E2E0C4F8540FC868FB9067E1E0C454F076
:101CA20048FA742F2BF582EA3451F58312D36C90E3
:101CB20067A012D3A474332BF582EA3451F5831250
:101CC200D36C9067A412D3A47BFF7AAD796712D844
:101CD200AB7B017A6779E512091DEF4E7003021D95
:101CE200807BFF7AAD798C9067C512D4349067E21D
:101CF200E0C4F8540FC868FF9067E1E0C454F048AC
:101D0200FE74272FF974513EFA7B019067C812D4F2
:101D1200349067E2E0C4F8540FC868FF9067E1E0CE
:101D2200C454F048FE742B2FF974513EFA9067CBDD
:101D320012D4349067E2E0C4F8540FC868FF906789
:101D4200E1E0C454F048FE742F2FF974513EFA902A
:101D520067CE12D4349067E2E0C4F8540FC868FF2B
:101D62009067E1E0C454F048FE74332FF974513E99
:101D7200FA9067D112D4347A6779E512DD39906826
:101D8200A312D3FD90679512D4349067E1E0FEA3CD
:101D9200E07802C333CE33CED8F924D6F582EE34BE
:101DA20057F58312D36C90679812D3A47BFF7AAD58
:101DB200793A12D8AB7B017A6779E39068BB12D487
:101DC200347BFF7AAD79981209D390685D12D3A45F
:101DD2009067E3E07002A3E0603290685D12D36C1A
:101DE200C004C005C006C0079067E1E0FEA3E0782A
:101DF20002C333CE33CED8F924D6F582EE3457F56A
:101E020083D007D006D005D00412D3A490689112D3
:101E1200D3FD90679512D4349067E2E02461F58295
:101E2200E43465F583E075F003A424A9F582E43473
:101E320068F58312D3FD90679812D4347BFF7AAD94
:101E420079A512D8AB7B017A68794912091DEF4E48
:101E52006071906849E04420249D603424FD604212
:101E620024F8605024F96016240970579067E2E064
:101E72002461F582E43465F5837401F0804590674E
:101E8200E2E02461F582E43465F5837402F0803384
:101E92009067E2E02461F582E43465F5837403F02F
:101EA20080219067E2E02461F582E43465F5837471
:101EB20004F0800F9067E2E02461F582E43465F576
:101EC20083E4F090689412D3FD90679512D4349015
:101ED20067E2E0241FF582E43466F583E075F003DF
:101EE200A424A9F582E43468F58312D3FD9067989F
:101EF20012D4347BFF7AAD79A512D8AB7B017A6814
:101F0200794912091DEF4E6071906849E04420241E
:101F12009D603424FD604224F8605024F960162448
:0E1F22000970579067E2E0241FF582E43466F0
:101F3000F5837401F080459067E2E0241FF582E4A8
:101F40003466F5837402F080339067E2E0241FF575
:101F500082E43466F5837403F080219067E2E02424
:101F60001FF582E43466F5837404F0800F9067E215
:101F7000E0241FF582E43466F583E4F090689A1259
:101F8000D3FD90679512D4349067E2E025E0FF908E
:101F900067E1E033FE74BB2FF582EE3466F583E42F
:101FA000A3E0540190686175F00312D3E1E475F089
:101FB00003A42583F58312D3FD90679812D4347B54
:101FC000FF7AAD79A512D8AB7B017A6879491209FD
:101FD0001DEF4E6045906849E04420FDBD631D90B3
:101FE00067E2E025E0FF9067E1E033FE74BC2FF587
:101FF00082EE3466F583E054FEF0801EBD6D1B90CA
:1020000067E2E025E0FF9067E1E033FE74BC2FF566
:1020100082EE3466F583E04401F090689D12D3FDB2
:1020200090679512D4349067E2E025E0FF9067E175
:10203000E033FE74BB2FF582EE3466F583E4A3E053
:102040005402FFE4C313FEEF1390686775F00312A8
:10205000D3E1EE75F003A42583F58312D3FD9067D9
:102060009812D4347BFF7AAD79B112D8AB7B017A68
:1020700068794912091DEF4E6044906849E0442098
:10208000FDBD791C9067E2E025E0FF9067E1E03359
:10209000FE74BC2FF582EE3466F583E04402F02234
:1020A000BD6E1B9067E2E025E0FF9067E1E033FE44
:0F20B00074BC2FF582EE3466F583E054FDF02208
:1020BF007BFF7AAD79BE1208A37BFF7AAD79E81268
:1020CF0008A37BFF7AAE790C1208A37BFF7AAE7957
:1020DF00341208A37BFF7AAE794D1208A37BFF7AE7
:1020EF00AE79701208A37BFF7AAE799D1208A37B9D
:1020FF00FF7AAE79C81208A37BFF7AAE79E5120892
:10210F00A37BFF7AAF79081208A37BFF7AAF7926FA
:10211F001208A37BFF7AA6794F1208A312E720AE0D
:10212F0007EED394395005EE24D0FF22EE4420FF62
:06213F00BF71E07F712278
:102145001220BFEF12D449217100217601217B02B3
:10215500218003218504218A05218F0621940721E9
:102165009908219E0921D071000021451274BA8079
:10217500CF126D5180CA126E3280C51273A180C014
:10218500126F7F80BB120CAB80B61260C780B11294
:1021950021D180AC1265DD80A77BFF7AA77941123A
:1021A50008A312E720EF4420FFBF79941202B27B07
:1021B500FF7AAF79441208A312E720EF442064792F
:0C21C500600302214512939A022145227A
:1021D100E49067F0F0A3F07BFF7AAF79711208A366
:1021E10012E7209067EFEFF04420646B7041905D3F
:1021F1007AF07BFF7AAF799C1208A312E7209067EF
:10220100EFEFF04420FFBF791C7BFF7AAF79D31247
:1022110008A37BFF7AB079071208A39065FAE0441E
:1022210020F00223BA9065FAE054DFF00223BA905D
:1022310067EFE04420647960030222D1905D7A0463
:10224100F07BFF7AB079331208A312E720EF24CF95
:10225100603524FE601B047044904E957421F0900B
:102261004E787411F09065FBE04402F054FEF0806A
:102271002C904E787401F0904E95F09065FBE054EF
:10228100FDF054FEF08016904E95742EF0904E782D
:10229100741EF09065FBE054FDF04401F07BFF7A81
:1022A100B079601208A312E7209067EFEFF04420A5
:1022B100FFBF790A9054E8E04440F00223BAEF648A
:1022C1006E60030223BA9054E8E054BFF00223BACF
:1022D1009067EFE04420646960030223BA905D7A5D
:1022E1007402F07BFF7AB0797C900005E0906795ED
:1022F100F012D8AB7B017A6779DB12091DEF4E60D2
:102301001F7BFF7AB079A79067C512D4347B017A1D
:102311000079059067C812D4347A6779DB12DD3908
:102321007BFF7AB079AB90000CE0906795F012D802
:10233100AB7B017A6779DB12091DEF4E601F7BFFD2
:102341007AB079A79067C512D4347B017A00790CF1
:102351009067C812D4347A6779DB12DD397BFF7A52
:10236100B079D412D8AB12E720EF4420FFBF79092E
:102371009065FBE04410F080079065FBE054EFF0BE
:102381007BFF7AB079ED90000AE0FFA3E0906795BA
:10239100CFF0A3EFF012D8AB7B017A6779F29068A6
:1023A1004A12D4347BFF7AB1790C12099CEF4E604A
:1023B1000890000AEEF0A3EFF07B017A6779F290C2
:1023C100684A12D4347BFF7AB1791612099C90675E
:1023D100F0EEF0A3EFF0BE040ABFB007E49065FC95
:1023E100F080409067F0E0FEA3E0FFBE090BBF6004
:1023F100089065FC7401F0802ABE120BBFC00890E2
:1024010065FC7402F0801CBE250BBF80089065FC42
:102411007403F0800EE4B5070AEEB44B069065FC38
:102421007404F0C2CA9065FCE025E024A7F582E4BB
:102431003466F583E0FCA3E0FDECF5CBF5CDEDF5DD
:10244100CAF5CCD2CA7BFF7AB179471208A312E749
:1024510020EF44202492601024F570139054E7E09B
:102461004420F0A3E0F080079054E7E054DFF07BD4
:10247100FF7AB1796E1208A312E720EF442024926B
:10248100602E24F56017240770349054E7E044402F
:10249100F0A3E0F09065FAE04410F080219054E759
:1024A100E04440F0A3E0F09065FAE054EFF0800ED4
:1024B1009054E7E054BFF09065FAE054EFF07BFFF1
:0424C1007AB17999DA
:1024C5001208A312E720EF4420249F600C24FB7020
:1024D5000F9054E8E04480F0229054E8E0547FF0F7
:0124E50022D4
:1024E6007BFF7AB179CB906795E53FF0A3E540F0A5
:1024F600A3E52BF0A3E528F012D8AB7BFF7AB279DF
:102506000C1208A37BFF7AB2795D1208A3E4F523C7
:10251600904EC2E0FFE523C39F503574682523F52E
:1025260082E43466F583E0FF3395E0FE7C007D149B
:1025360012D15074A12FF974603EFA7B0190679511
:1025460012D4347BFF7AB2796C12D8AB052380C0E3
:10255600904EC2E0F523E523C39405500D7BFF7A28
:10256600B279721208A3052380EC7BFF7AB27980D8
:042576001208A32282
:10257A007BFF7AB179CB906795E53FF0A3E540F010
:10258A00A3E52BF0A3E528F012D8AB7BFF7AB2794A
:10259A00831208A37BFF7AB279CE1208A37BFF7A53
:1025AA00B379191208A39054E7E0A330E10B7BFF3B
:1025BA007AB379631208A380097BFF7AB279801211
:1025CA0008A390665BE0FF3395E0FE74682FF582FE
:1025DA00EE3466F583E0FF3395E0FE7C007D14124D
:1025EA00D15074A12FF974603EFA7B01906795125D
:1025FA00D4347BFF7AB379A012D8AB7BFF7AB37954
:0E260A00B712D8AB7BFF7AB4790612D8AB2298
:102618009068117420F0E4F524F525E525AE2478BA
:1026280002C333CE33CED8F9FBAA06242EF582EAAC
:102638003468F58312D3B000000000741A2BF582B9
:10264800EA3468F58312D3B0000000000525E525BB
:1026580070020524E5256405452470BFE49067DC15
:10266800F09067DBF09065F9E04404F0A3E0F090A7
:1026780054E7E0A330E02F12087CEF149067DCF0F9
:10268800C3648094804018904EC2E0FF9067DCE0FD
:10269800FD3395E0FCC3ED9F7480F86C984070E4BE
:1026A8009067DCF080697BFF7AB47953904EC2E082
:1026B800906795F012D8AB128A2390665BE0FFF41E
:1026C8007003022B31EFFD3395E0FC74682DF58221
:1026D800EC3466F583E0C3648094804014904EC265
:1026E800E0FDEF3395E0FEC3EF9D7480F86E9840EF
:1026F800167BFF7AB47995904EC2E0906795F012F8
:10270800D8ABE490665BF090665BE09067DCF09095
:102718004EC2E0FF904EA4E0FCA3E0FDD3EF9DE4A1
:102728009C4005E0904EC2F09067DCE0FF3395E0F6
:10273800FE74682FF582EE3466F583E09067DDF06D
:102748001208661224E690E102E054F0F09054E793
:10275800E0FEA3E0FF30E214EE30E3089068117465
:1027680026F0800E9068117421F08006906811742C
:1027780020F0E4F524F525904EC2E0FFC3E5259F3F
:10278800E524940050C774682525F582E43466F57D
:1027980083E09067DBF0C36480948040DAE0FFD385
:1027A800648094BC50D11247231245389067DBE00F
:1027B800FF124C6790676012D36CC004C005C00656
:1027C800C007E525AE247802C333CE33CED8F9242A
:1027D8001AF582EE3468F583D007D006D005D00408
:1027E80012D3A490678212D36CC004C005C006C07F
:1027F80007E525AE247802C333CE33CED8F9242E8C
:10280800F582EE3468F583D007D006D005D00412DF
:10281800D3A49067DDE0FF9067DBE0B50718906709
:102828006012D36C90681212D3A490678212D36C92
:1028380090681612D3A4E59020E406126480022959
:10284800827BFF7AB479D6906811E0906795F0A3FF
:10285800E529F0A3E52AF0A3E527F012D8AB7BFF22
:102868007AB479EC90681A12D36C90679512D3A455
:1028780090682E12D36C90679912D3A490681E1298
:10288800D36C90679D12D3A490683212D36C906772
:10289800A112D3A490682212D36C9067A512D3A476
:1028A80090683612D36C9067A912D3A49068261248
:1028B800D36C9067AD12D3A490683A12D36C90672A
:1028C800B112D3A412D8AB7BFF7AB5791D90682AD0
:0328D80012D36CAC
:1028DB0090679512D3A490683E12D36C90679912AF
:1028EB00D3A412D8AB7F801205017BFF7AB5792B6D
:1028FB0090679512D434906798E529F0A3E52AF0F8
:10290B00A3E527F0906811E090679BF09067DDE0FE
:10291B00FF3395E0FE7C007D1412D15074A12FF98A
:10292B0074603EFA7B0190679C12D4347A6779DF2E
:10293B0012D8A57B017A6779DF1208C17FC0120517
:10294B00017BFF7AB5794390679512D43490681266
:10295B0012D36C90679812D3A490681612D36C9014
:10296B00679C12D3A47B017A6779DF12D8A57B0110
:10297B007A6779DF1208C19054E7E0A330E0751253
:10298B00087C9067DEEFF070089054E7E054FDF0A0
:10299B00229067DEE014F0904EC2E0FF9067DEE01D
:1029AB00FDFB3395E0FAC3EB9F7480F86A98400AFD
:1029BB00906668E09067DDF08020EDFF3395E0FED8
:1029CB0074682FF582EE3466F583E0FF9067DDE0E7
:1029DB00FEEF6E6005EFF002275590E101E0F43059
:1029EB00E4099054E8E04404F080649054E8E05427
:1029FB00FBF0805B30985812E720EF4420249B605B
:102A0B000F24F5602014704790E102E054DFF022B0
:102A1B009054E8E030E20554FBF080339054E8E04A
:102A2B004404F0802A9054E7E0FEA3E0FFEE30E38D
:102A3B000E9054E754F7F09068117421F08010EE6B
:102A4B0044089054E7F0EFA3F09068117426F090CF
:102A5B005F8712D36C90678212D38812CDC3402943
:102A6B009054E8E030E22290665BE525F07BFF7A3C
:102A7B00A3799E1208A39054E7E054FBF0122B327B
:102A8B009054E7E0A330E256227F007E007D407C2D
:102A9B00C090678212D38812CDC3401990E000E03A
:102AAB0030E00990E102E04420F0803290E102E056
:102ABB0054DFF0802990E102E054DFF09054E7E01E
:102ACB00FEA3E0FF30E40D30E20A9067DBE0FF127B
:102ADB003658800A90E102E054F0F01208669065D7
:102AEB00FAE030E63690665BE0FF3395E0FEEF7878
:102AFB0002C333CE33CED8F9242EF582EE3468F5EB
:102B0B008312D36C904F4312D38812CDC3600C4009
:102B1B000A4390409065FAE054BFF00525E5257017
:072B2B0002052402277F22AE
:102B32009068C87420F0A3742AF09054E7E0FEA3D2
:102B4200E0FFEE30E11A90E00E740AF0EE30E30896
:102B52009068C97426F080159068C97421F0800DC0
:102B62009068C9742AF090E00EE04401F090E1020E
:102B7200E054DFF09054E7E0FEA3E0FFEE30E01B0C
:102B820020E11812087CEF1490665BF0C364809415
:102B92008040E1E0D3648094BC50D99065F9E04470
:102BA20005F0A3E04481F09065F9E0545FF090E015
:102BB2000DE054FBF090665BE0FF906894F0339573
:102BC200E0FE74682FF582EE3466F583E0FFC3649D
:102BD200809480409F906892EFF01247239054E9CE
:102BE20012D3B00000000090655D12D3B000000067
:102BF20000905D7AE06401706FFFFD123D459065C3
:102C0200FBE030E04E7F047DC912CAAE7F047D60D6
:102C120012CAAE7F04E4FD12CAAE7F04E4FD12CAFA
:102C2200AE7F04904E78E0FD12CAAE7F047D05129D
:102C3200CAAE7F047D1012CAAE7F04E4FD12CAAE92
:102C42007F04E4FD12CAAE7F04904E78E0FD12CA02
:102C5200AE800E9065FBE030E107E4FF7D4E123D51
:102C620045E4FF7D80123D459065F112D36C905F83
:102C72006312D3A49066B712D36C90655112D3A499
:102C8200906892E0FF1242A17FCD7ECC7DCC7C3D4C
:102C920090660312D38812CDC3600A4008906892EE
:102CA200E0FF1240017FCD7ECC7DCC7C3D9065FD66
:102CB20012D38812CDC3600A4008906892E0FF12D6
:102CC2003D92906661E0B4040C90674B12D3B00061
:102CD2000000C8800A90674B12D3B00000000A12AD
:102CE200086612257A90E102E054F0F09054E7E091
:102CF200FEA3E0FF30E20A9068C9E09068C7F08066
:102D0200069068C77420F0EE30E07A12087C906872
:102D120093EFF09054E7E0FEA3E0FFEE20E12C9069
:102D22006893E0700BEE44029054E7F0EFA3F022B8
:102D3200906893E014F090665BE0FF906893E0FE89
:102D42006F601690665BEEF0022B76906893E070EF
:102D5200089054E7E054FDF02290E101E0F430E401
:102D6200129054E8E04404F09068C9E09068C7F01B
:102D72000230519054E8E054FBF09068C8E090684B
:102D8200C7F002305120980302305112E720EF447D
:102D92002012D4492ECC202EF3282FA52B2FC12D63
:102DA2002FE0302DCD312E0C322E4C332E8C342F81
:102DB200EC3F2F71653039692F276E2F3D702F0A36
:102DC200713027742F987900003051906892E0FF9B
:102DD200FD3395E0FC74F32DF582EC345EF583E46B
:102DE200F0EF3395E0FEEFC4F8540FC868FFEEC46D
:102DF20054F048FE74272FF582EE3451F58312D336
:102E02006C90660312D3A4023051906892E0FFFDE9
:102E12003395E0FC74F32DF582EC345EF583740196
:102E2200F0EF3395E0FEEFC4F8540FC868FFEEC42C
:102E320054F048FE742B2FF582EE3451F58312D3F1
:102E42006C90660312D3A4023051906892E0FFFDA9
:102E52003395E0FC74F32DF582EC345EF583740255
:102E6200F0EF3395E0FEEFC4F8540FC868FFEEC4EC
:102E720054F048FE742F2FF582EE3451F58312D3AD
:102E82006C90660312D3A4023051906892E0FFFD69
:102E92003395E0FC74F32DF582EC345EF583740314
:102EA200F0EF3395E0FEEFC4F8540FC868FFEEC4AC
:102EB20054F048FE74332FF582EE3451F58312D369
:012EC2006CA3
:102EC30090660312D3A402305190665BE004F09045
:102ED3006770E0FF90665BE0FD3395E0FCC3ED9F18
:102EE3007480F86C985003023051E014F0023051B2
:102EF30090665BE014F0E0C364809480400302308A
:102F030051E004F002305190E102E054F0F0E0545B
:102F1300DFF09054E7E04404F0A3E0F09065F9E0BB
:102F230054DFF0229054E7E0A320E10302305190F4
:102F3300E102E054DFF01224E6229054E7E0FEA31E
:102F4300E0FFEE20E10302305130E30F9054E754E9
:102F5300F7F09068C97421F0023051EE44089054A0
:102F6300E7F0EFA3F09068C97426F0023051905453
:102F7300E8E020E20E4404F09068C9E09068C7F0EE
:102F83000230519054E8E054FBF09068C8E0906838
:102F9300C7F002305190E00DE04408F012086602D9
:102FA300305190655D12D36CEF2464FFE43EFEE480
:102FB3003DFDE43CFC90655D12D3A4023051906565
:102FC3005D12D36CC3EF9464FFEE9400FEED9400A6
:102FD300FDEC9400FC90655D12D3A4807190655D57
:102FE30012D3B000000000806590665BE0FF33956C
:102FF300E0FE74682FF582EE3466F583E0FF3395C7
:10300300E0FE7C007D1412D15074A12FF974603E50
:10301300FA7B0190679512D4347BFF7AB579581205
:10302300D8AB802A906892E0FF124001906892E04A
:10303300FF123D928018906892E0FF1242A19068BF
:1030430092E0FF124001906892E0FF123D92906679
:103053005BE0FF906894E06F6003022B9D1245389C
:10306300906892E0FF124C6790676012D36C905E99
:10307300EF12D3A490678212D36C905C8612D3A410
:10308300906892E0FF1267AEE59020E40612648038
:1030930002324C7BFF7AB5795F9068C7E090679501
:1030A300F0A3E529F0A3E52AF0A3E527F012D8ABB6
:1030B30090676012D36C90679512D3A490678212C5
:1030C300D36C90679912D3A4904E4612D36C906739
:1030D3009D12D3A47F487E517DC77CC59060891221
:1030E300D38812CB309067A112D3A490000612D3D9
:1030F3006C9067A512D3A4904E7012D36C9067A9FD
:1031030012D3A4904E4212D36C9067AD12D3A49005
:103113005F6712D36C9067B112D3A47BFF7AB57942
:103123007412D8AB90655D12D36CEC12CE419067EC
:103133009512D3A47BFF7AB5799E12D8AB7F801208
:1031430005017BFF7AB5792B90679512D43490678C
:0331530098E529D3
:10315600F0A3E52AF0A3E527F09068C7E090679B07
:10316600F090665BE0FF3395E0FE74682FF582EE23
:103176003466F583E0FF3395E0FE7C007D1412D1C2
:103186005074A12FF974603EFA7B0190679C12D4AB
:10319600347A68799512D8A57B017A6879951208F0
:1031A600C17FC012050190665BE0FF3395E0FE74B7
:1031B600682FF582EE3466F583E0FF3395E0FEEF87
:1031C60025E0FFEE33FE74BB2FF582EE3466F58301
:1031D600A3E030E13B7BFF7AB579A890679512D4DE
:1031E6003490676012D36C90679812D3A49067826C
:1031F60012D36C90679C12D3A4904E4212D36C905B
:1032060067A012D3A47B017A68799512D8A5802D80
:103216007BFF7AB579C190679512D43490676012B6
:10322600D36C90679812D3A490678212D36C906780
:103236009C12D3A47B017A68799512D8A57B017A72
:103246006879951208C1905F8712D36C90678212D5
:10325600D38812CDC3402B5390BF9065FAE044400B
:10326600F09065F9E0FEA3E0FFEE30E6759054E8D5
:10327600E030E26EEE20E76A906892E0FF12377067
:1032860080609054E7E0A330E12590E102E054F03D
:10329600F01224E67BFF7AA3799E1208A39065F9C3
:1032A600E04404F0A3E0F09065F9E054DFF02290EA
:1032B60065FAE030E62C904F4312D36C9067821289
:1032C600D38812CDC36002501943904090655D12B9
:1032D600D3B0000000009065F9E0545FF0A3E0541D
:1032E600BFF09065FAE030E72C7F007E007D007C21
:1032F60000905C8612D38812CDC36019401790687F
:1033060092E0FF1242A1906892E0FF1240019065A0
:10331600FAE0547FF09054E8E030E00B906892E0D9
:10332600FF123A100233BF9054E8E020E7157F0001
:103336007E007D407CC0905C8612D38812CDC3602F
:103346007840769066B712D38890655112D36C1286
:10335600D1F212E7637B2C7A0179007800C312D38D
:103366002B501C9054E7E0A330E5149066B712D3B7
:103376006C90655112D3A4906892E0FF12400190C0
:1033860065F112D388905F6312D36C12D1F212E703
:103396006390674B12D388C312D341501C9054E7F5
:1033A600E0A330E6149065F112D36C905F6312D3FC
:1033B600A4906892E0FF123D9290E101E020E56A58
:1033C600E020E638906892E0FF3395E0FEEF780261
:1033D600C333CE33CED8F92493F582EE345FF5832A
:1033E600C083C08212D36C7B007A0079487842127F
:1033F600CB30D082D08312D3A402348F90E101E087
:0934060020E70C90655D12D3B0C3
:10340F0000000000807A90655D12D36CEF2432FFCC
:10341F00E43EFEE43DFDE43CFC90655D12D3A480E8
:10342F005F90E101E020E758E020E637906892E0F6
:10343F00FF3395E0FEEF7802C333CE33CED8F924B5
:10344F0093F582EE345FF583C083C08212D36C7B19
:10345F00007A007948784212CB2CD082D08312D3D5
:10346F00A4801D90655D12D36CC3EF9432FFEE9470
:10347F0000FEED9400FDEC9400FC90655D12D3A46A
:10348F00905D81E0FEA3E0FFE4FCFDC004C005C039
:10349F0006C00790676C12D388904EC312D36C127C
:1034AF00D1F2A804A905AA06AB07D007D006D0050C
:1034BF00D004D312D3415038905D81E0FEA3E0FFDA
:1034CF00E4FCFDC004C005C006C00790673312D3EB
:1034DF0088904EC312D36C12D1F2A804A905AA0684
:1034EF00AB07D007D006D005D004D312D341400389
:1034FF001239389065FAE030E30990E102E0445068
:10350F00F0800790E102E054AFF090E00DE020E290
:10351F000302364C9054E7E0FEA3E0FFEE20E303F6
:10352F0002364C20E10302364C90E00DE054FBF0E4
:10353F00E490688FF0A3F0904EC2E0FFC3906890C4
:10354F00E09F90688FE094004003023644A3E0248C
:10355F0068F582E43466F583E0906891F0C3648087
:10356F0094805003023637E0FFD3648094BC40034D
:10357F00023637124723124538906891E0FF124CFC
:10358F00677F007E007D007C0090678212D38812D7
:10359F00CDC36002500302363790665BE0FF339570
:1035AF00E0FEC3906890E09F90688FE09E503EA32E
:1035BF00E0FF90665BF03395E0FE74682FF582EEC6
:1035CF003466F583E0FF3395E0FE7C007D1412D165
:1035DF005074A12FF974603EFA7B0190679512D455
:1035EF00347BFF7AB579D712D8AB022B9D90665BEF
:1035FF00E0FF3395E0FED3906890E09F90688FE0F6
:10360F009E40327F007E007D007C00905C8612D34E
:10361F008812CDC3501F9065FAE020E7189068908C
:10362F00E090665BF0022B9D90688FE475F00112BD
:10363F00D19A023546906892E0FF12472390689224
:09364F00E0FF1267AE022CEE222E
:103658009068CBEFF01245389065F9E0FEA3E0FFE3
:10366800EE30E16E30E26B7F007E247D747C499001
:1036780065CD12D38812CC2112CE7F9065F112D37A
:10368800A47F007E247D747C499065D112D3881272
:10369800CC2112CE7F9066B712D3A4906662E090D8
:1036A8006660F0906663E0906661F09068CBE0FF3A
:1036B8001242A19068CBE0FF1240019068CBE0FF76
:1036C800123D929065F9E054FBF09068CBE0FF1250
:1036D80047239065F9E054DFF0904F3F12D36C9088
:1036E8005C8612D3A49055F112D36C905EEF12D37E
:1036F800A4126A49905D81E0FEA3E0FFE4FCFDC0EE
:1037080004C005C006C00790676C12D388904EC3EA
:1037180012D36C12D1F2A804A905AA06AB07D007E8
:10372800D006D005D004D312D3415038905D81E043
:10373800FEA3E0FFE4FCFDC004C005C006C007907E
:10374800673312D388904EC312D36C12D1F2A804F7
:10375800A905AA06AB07D007D006D005D004D31216
:08376800D3414003123938225D
:103770009068CAEFF090676012D36C9068CB12D358
:10378000A490E102E054F0F07F007E007D207C41B7
:1037900090678E12D38812CDC3401990655512D30D
:1037A0006C7B607A0B7936783A12CB309065551283
:1037B000D3A4801790655512D36C7B2F7A8E79E352
:1037C000783B12CB3090655512D3A49068CAE0FFC5
:1037D000124C677FC01205017BFF7AB579FE120893
:1037E000C19054E8E030E3030238757F007E007D2D
:1037F000B47C429068CB12D38812CDC36028402697
:103800007F007E007D347C439068CB12D38812CD3C
:10381000C350137F007E007D347C4390676012D3D9
:103820008812CDC350427F007E007D877C43906824
:10383000CB12D38812CDC340030238F97F007E003B
:103840007D347C439068CB12D38812CDC3500302E1
:1038500038F97F007E007D347C4390676012D38806
:1038600012CDC340030238F99065F9E04420F0A37B
:10387000E0F00239227F007E007D877C439068CB98
:1038800012D38812CDC3602840267F007E007DB40D
:103890007C439068CB12D38812CDC350137F007E37
:1038A000007DB47C4290676012D38812CDC3403D46
:1038B0007F007E007DB47C429068CB12D38812CD0D
:1038C000C350367F007E007D007C009068CB12D311
:1038D0008812CDC3602340217F007E007D877C431A
:1038E00090676012D38812CDC3600E400C9065F9CA
:1038F000E04420F0A3E0F08029905F8712D36C9021
:10390000678212D38812CDC350099065F9E054DF65
:10391000F0800F90676012D36C9068CB12D3A40232
:1039200037889065F9E04480F0A3E0F012453890C4
:0839300068CAE0FF124C672297
:103938009065F9E0A330E303023A0F90E102E05406
:10394800F0F07BFF7AB6790F906795E529F0A3E54B
:103958002AF0A3E527F012D8AB7F801205017BFF80
:103968007AB6796A1208C17FC01205017BFF7AB660
:10397800797B1208C19068CCE4F0A3E52AF0A3E4AF
:10398800F0A3E527F090E000E030E00990E102E0E4
:103998004420F0800790E102E054DFF012453890AF
:1039A80068CCE0FCA3E0FDC3E52A9DE49CC36480E9
:1039B80094805006743C252AF52A9068CEE0FAA334
:1039C800E0B527C1E4B502BDC3E52A9DFFE49CFE2E
:1039D8009066A5E0FCA3E0B507ABEEB504A77BFFB6
:1039E8007AB6798C906795E529F0A3E52AF0A3E5E6
:1039F80027F012D8AB904EC312D36C90673312D312
:083A0800A490676C12D3A42204
:103A10009068CAEFF090659DE0FEA3E0FFC3906060
:103A200084E09F9068CEF0906083E09E9068CDF037
:103A3000900017E0FF7E007C017DF412D150906869
:103A4000CFEEF0A3EFF07F007E007D001C905C863F
:103A500012D38812CDC35003023B517F03120C7B5B
:103A600090659DE0FEA3E0FFC3E52D9F9068CCF03C
:103A7000E52C9E9068CBF09068CDE0FEA3E0FF12AD
:103A8000E751C006C0079068CBE0FEA3E0FF12E755
:103A900051AC06AD07D007D006C3ED9FEE6480F8A9
:103AA000EC6480985003023B51C39068CDE0648081
:103AB00094805043D39068CCE094009068CBE0644D
:103AC00080948040199065FAE030E30990E102E0CB
:103AD00054BFF0806390E102E04440F0805A90656A
:103AE000FAE030E30990E102E054EFF0804A90E11F
:103AF00002E04410F08041D39068CCE094009068DC
:103B0000CBE06480948040199065FAE030E309903E
:103B1000E102E054EFF0802090E102E04410F080F8
:103B2000179065FAE030E30990E102E054BFF080BD
:103B30000790E102E04440F0E4FFFE9068CFE0FC33
:103B4000A3E0FDC3EF9DEE9C50070FBF00010E8068
:023B5000EA2267
:103B5200900017E0FF7E007C037DE812D150906850
:103B6200CFEEF0A3EFF090674FE0FF7E0012D1504E
:103B72009068D1EEF0A3EFF090673712D38890658A
:103B8200F112D36C12D1F29068D312D3A49065EDE6
:103B920012D3889068D312D36C12E6B512E7639001
:103BA20068D712D3A47BFF7AB679BB90673712D35A
:103BB2006C90679512D3A49065F112D36C906799BB
:103BC20012D3A49068D312D36C90679D12D3A490A1
:103BD20068D712D36C9067A112D3A412D8AB7F001E
:103BE2007E007D007C009068D312D388D312D32B41
:103BF200400B7BFF7AB679E81208A3801D7F007E16
:103C0200007D007C009068D312D388C312D32B505E
:103C1200097BFF7AB679F21208A3E49068CBF0A38D
:103C2200F09068CBE0FEA3E0FFE4FCFD9068D712C1
:103C3200D388D312D3415003023D347F007E007DEE
:103C4200007C009068D312D388D312D32B401990F2
:103C520065FAE030E30990E102E054EFF080209051
:103C6200E102E04410F080179065FAE030E3099039
:103C7200E102E054BFF0800790E102E04440F07BB3
:103C8200FF7AB679FD1208A3E49068CDF0A3F09014
:103C920068CFE0FEA3E0FFC39068CEE09F9068CDBE
:103CA200E09E500C9068CDE475F00112D19A80DF4D
:103CB2007F007E007D007C009068D312D388D312EF
:103CC200D32B40199065FAE030E30990E102E04419
:103CD20010F0802090E102E054EFF080179065FA36
:103CE200E030E30990E102E04440F0800790E10215
:103CF200E054BFF07BFF7AB679FF1208A3E4906824
:103D0200CDF0A3F09068D1E0FEA3E0FFC39068CEAF
:103D1200E09F9068CDE09E500C9068CDE475F00174
:103D220012D19A80DF9068CBE475F00112D19A0229
:103D32003C237BFF7AB279801208A39065FAE054A3
:033D4200FEF0226E
:103D45008D08AE077F04AD0612CAAE7F04E4FD12EE
:103D5500CAAE7F04E4FD12CAAE7F04E4FD12CAAE0A
:083D65007F04AD0812CAAE2272
:103D6D009068FEEFF0E4FF7DFE12CAAEE4FF7DFE2B
:103D7D0012CAAEE4FF9068FEE0FD12CAAEE4FF7D0C
:053D8D000212CAAE2283
:103D92009068CCEFF0905D7AE0705B7BFF7AB77948
:103DA2000190679512D4349065F112D36C906798A4
:103DB20012D3A47B017A6879D212D8A59065FAE071
:103DC20030E5299068CCE0FF3395E0FEEF25E0FF77
:103DD200EE33FE74BB2FF582EE3466F583A3E0303A
:103DE200E30A7B017A6879D21208FF227B017A68A2
:103DF20079D21208DF22905D7AE064016003023F0B
:103E020014FFFD123D457B0A7A0079007800906527
:103E1200F112D36C12D28B9068FA12D3A47BFF7A80
:103E2200B7790C90679512D4349068FA12D36C90DB
:103E3200679812D3A47B017A6879D212D8A59068C8
:103E4200D2E0B4311EA3E0B43219A3E024D0540F5F
:103E52009068D0F044C0FF9068CFF0FD7F0412CA92
:103E6200AE80329068D2E06430702AA3E024D0544D
:103E72000FFF9068D1F09068D4E024D0540FFE90E8
:103E820068D0F0EFC454F054F04EFF9068CFF0FDCC
:103E92007F0412CAAE9068CDE4F0A37403F0E490FC
:103EA20068D1F09068D0F09068CEE0FF24D2F5821D
:103EB200E43468F583E024D0540FFE9068D1F074A6
:103EC200D32FF582E43468F583E024D0540FFF90B9
:103ED20068D0F0EEC454F054F04FFF9068CFF0FD7C
:103EE2007F0412CAAE9068CDE475F00212D19AC373
:103EF2009068CEE094089068CDE064809480409E03
:103F02007F04904E78E0FD12CAAEE4FF7D80123D40
:103F12004522905D7AE0640260030240009065F100
:103F220012D36C9068FA12D3A47BFF7AB7791390FC
:103F3200679512D4349068FA12D36C90679812D3B2
:103F4200A47B017A6879D212D8A59065FBE020E4BF
:103F52002590677DE0FF123D6DE4FF7D0712CAAE3A
:103F6200E4FF7DD112CAAEE4FF7DFD12CAAE90001D
:103F72000BE0FF12CB0E90677DE0FF123D6DE4FF78
:103F8200FD12CAAE9068CDE4F0A37409F0E4906823
:103F9200D1F09068D0F09068CEE0FF24D2F582E4B0
:103FA2003468F583E024D0540FFE9068D0F074D1C9
:103FB2002FF582E43468F583E024D0540FFF906833
:103FC200D1F0C454F054F04EFF9068CFF0FDE4FFFE
:103FD20012CAAE9068CD74FF75F0FE12D19AD390DA
:103FE20068CEE094009068CDE064809480509EE4B6
:0F3FF200FF7DFD12CAAE90000BE0FF12CB0E2236
:104001009068CCEFF0905D7AE060030240987BFF0E
:104011007AB7791B90679512D4349066B712D36C36
:1040210090679812D3A47B017A6879D612D8A590AB
:1040310065FAE030E5459068CCE0FF3395E0FEEFAE
:1040410025E0FFEE33FE74BB2FF582EE3466F58377
:10405100A3E030E3137BFF7AB779261208DF7B01F7
:104061007A6879D61208DF227BFF7AB7792612089F
:10407100FF7B017A6879D61208FF227BFF7AB77934
:10408100261208DF7B017A6879D61208DF7BFF7A76
:10409100B7792B1208DF22905D7AE0640160030298
:1040A10041B4FFFD123D457B0A7A0079007800900A
:1040B10066B712D36C12D28B9068D212D3A47BFF55
:1040C1007AB7790C90679512D4349068D212D36C78
:1040D10090679812D3A47B017A6879D612D8A590FB
:1040E10068D6E0B4311EA3E0B43219A3E024D05461
:1040F1000F9068D0F044C0FF9068CFF0FD7F0412AC
:10410100CAAE80329068D6E06430702AA3E024D031
:10411100540FFF9068D1F09068D8E024D0540FFE7E
:104121009068D0F0EFC454F054F04EFF9068CFF097
:10413100FD7F0412CAAE9068CDE4F0A37403F0E4ED
:104141009068D1F09068D0F09068CEE0FF24D6F569
:1041510082E43468F583E024D0540FFE9068D1F0F6
:1041610074D72FF582E43468F583E024D0540FFF2F
:104171009068D0F0EEC454F054F04FFF9068CFF047
:10418100FD7F0412CAAE9068CDE475F00212D19A97
:10419100C39068CEE094089068CDE064809480403C
:1041A1009E7F04904E95E0FD12CAAEE4FF7D801221
:1041B1003D4522905D7AE0640260030242A0906670
:1041C100B712D36C9068D212D3A47BFF7AB779135C
:1041D10090679512D4349068D212D36C906798127C
:1041E100D3A47B017A6879D612D8A59065FBE0202B
:1041F100E425900000E0FF123D6DE4FF7D0712CA47
:10420100AEE4FF7DD012CAAEE4FF7DFD12CAAE90CE
:10421100000BE0FF12CB0E900000E0FF123D6DE4B9
:10422100FFFD12CAAE9068CDE4F0A37409F0E490EA
:1042310068D1F09068D0F09068CEE0FF24D6F58286
:10424100E43468F583E024D0540FFE9068D0F07414
:10425100D52FF582E43468F583E024D0540FFF9024
:1042610068D1F0C454F054F04EFF9068CFF0FDE4F3
:10427100FF12CAAE9068CD74FF75F0FE12D19AD3C9
:104281009068CEE094009068CDE064809480509E68
:10429100E4FF7DFD12CAAE90000BE0FF12CB0E22AF
:1042A1009068CCEFF0905D7AE060030243B77BFF4A
:1042B1007AB7793090679512D434906660E0906750
:1042C10098F07B017A6879CE12D8A57BFF7AB7790D
:1042D1003090679512D434906661E0906798F07BD6
:1042E100017A6879F612D8A59065FAE020E5030213
:1042F10043809068CCE0FF3395E0FEEF25E0FFEED0
:1043010033FE74BB2FF582EE3466F583A3E030E310
:10431100377BFF7AB779261208DF7BFF7AB77938C6
:104321001208DF7B017A6879CE1208DF7BFF7AB74A
:10433100792B1208FF7BFF7AB7793D1208FF7B01C9
:104341007A6879F61208FF227BFF7AB7792612087C
:10435100FF7BFF7AB779381208FF7B017A6879CE43
:104361001208FF7BFF7AB7792B1208DF7BFF7AB740
:10437100793D1208DF7B017A6879F61208DF227B2A
:10438100FF7AB779261208DF7BFF7AB779381208EE
:10439100DF7B017A6879CE1208DF7BFF7AB7792B50
:1043A1001208DF7BFF7AB7793D1208DF7B017A685B
:1043B10079F61208DF22905D7AE064017073FFFDE7
:1043C100123D45906660E0FF602624FE600A04709D
:1043D1000FE49068CDF0800E9068CD7401F08006F6
:1043E1009068CD7408F09068CDE0FF7D27123D45BF
:1043F100906661E024FE600A04700FE49068CDF0DD
:10440100801D9068CD7401F080159054E8E030E68D
:10441100089068CD7488F080069068CD7408F0909B
:1044210068CDE0FF7D17123D45E4FF7D80123D45DB
:1044310022905D7AE0640260030245379065FBE0FB
:1044410020E425900000E0FF123D6DE4FF7D07129E
:10445100CAAEE4FF7DD012CAAEE4FF7DFD12CAAE42
:1044610090000BE0FF12CB0E900000E0FF123D6DBB
:10447100E4FF7D0112CAAE906660E024FE60121472
:10448100601814601E24037021E4FFFD12CAAE807F
:1044910019E4FF7D0112CAAE8010E4FF7D0312CA48
:1044A100AE8007E4FF7D0512CAAEE4FF7DFD12CAAE
:1044B100AE90000BE0FF12CB0E9065FBE020E425EF
:1044C10090677DE0FF123D6DE4FF7D0712CAAEE407
:1044D100FF7DD112CAAEE4FF7DFD12CAAE90000B82
:1044E100E0FF12CB0E90677DE0FF123D6DE4FF7D92
:1044F1000112CAAE906661E024FE601214601814C5
:10450100601E24037021E4FFFD12CAAE8019E4FF8E
:104511007D0112CAAE8010E4FF7D0312CAAE80078E
:10452100E4FF7D0512CAAEE4FF7DFD12CAAE900024
:074531000BE0FF12CB0E228C
:10453800120C13E53075F00AA4FF7C002531FFEC5E
:1045480035F0CF245CF540EF3405F53FE5306439AC
:10455800600B74642540F540E4353FF53FE53224AF
:10456800D075F00AA4FFE53324D02FF52BE53424C9
:10457800D075F00AA4FFE53524D02FF528E53624B8
:10458800D075F00AA4FFE53724D02FF529E53824A3
:10459800D075F00AA4FFE53924D02FF52AE53A248E
:1045A800D075F00AA4FFE53B24D02FF527AF40AE25
:1045B8003FAD2BAB281246C790001CEEF0A3EFF0DE
:1045C800E4FCFD7B807A517901F812D200C004C066
:1045D80005C006C007AF29E4FCFDFE7B107A0EF982
:1045E800F812D200D003D002D001D00012D1E5C019
:1045F80004C005C006C007AF2AE4FCFDFE7B3CFAF8
:10460800F9F812D200D003D002D001D00012D1E5BF
:10461800A804A905AA06AB07AF27E4FCFDFE12D142
:10462800E5904EC312D3A4904EC312D36CE412CEBD
:10463800417B007AC079A8784712CD2A9065551237
:10464800D3A4904E6EE0FEA3E0FFC3E5409FFFE5D4
:104658003F9EF5088F094F6065750A00750B01D3F9
:10466800E50B9509E50A95085054C3E540950BFFFD
:10467800E53F950AEF5403701990655512D36C7B8A
:10468800007A0079B7784312CB3090655512D3A4DD
:10469800801790655512D36C7B007A8079B6784381
:1046A80012CB3090655512D3A4D3E50B9405E50AD7
:0F46B8009400500A050BE50B7002050A80A12241
:1046C7009068D0EEF0A3EFF0A905AF037E00E4E019
:1046D70054037005FC7D0180047C007D009068D246
:1046E700ECF0A3EDF07D017C00E9FBC3ED9BEC94BE
:1046F7000050289068D3E075F00DA424AFF582E44C
:104707003465F583E5822DF582E43583F583E02F63
:0C471700FFE43EFE0DBD00010C80CE2230
:104723009068CCEFF0E0F9C3648094805003024CAE
:1047330066E9FD3395E0FCED25E0FFEC33FE747391
:104743002FF582EE345EF583E0FEA3E0FF246C9048
:104753004E6FF0EE3407904E6EF0C3EF945AEE9422
:10476300005007E475F06412D19A904E6FE024393B
:10477300FF904E6EE034F8FE9068CDF0A3EFF0C3E7
:10478300EE64809480400ED3E0941D9068CDE06485
:1047930080948040099068CDE4F0A3741DF0EDAEE1
:1047A300047802C333CE33CED8F9FBAA06248AF5A4
:1047B30082EA345CF58312D36C9065F512D3A4744A
:1047C300F52BF582EA3455F58312D36CEC12CE4106
:1047D30090677512D3A49068CCE0F9FF3395E0FE9F
:1047E300EF7802C333CE33CED8F9FBAA0624C6F53D
:1047F30082EA3458F58312D36C90677E12D3A47483
:10480300B62BF582EA3459F58312D36C90678E1276
:10481300D3A4E9FF3395E0FEEF7802C333CE33CE62
:10482300D8F9FBAA0624EDF582EA3454F58312D3B2
:104833006C90675812D3A474372BF582EA3450F581
:104843008312D36C90673F12D3A4E9FF3395E0FE44
:10485300EF7802C333CE33CED8F9FBAA062483F50F
:1048630082EA345DF58312D36C904E4A12D3A4745A
:10487300962BF582EA345BF58312D36C9000011218
:10488300D3A4E9FF3395E0FEEF7802C333CE33CEF2
:10489300D8F9FBAA0624A6F582EA345AF58312D383
:1048A3006C9065A312D3A474472BF582EA344FF5B9
:1048B3008312D36C9065FD12D3A47F007E247D7494
:1048C3007C499065FD12D38812CC2112CE7F90676C
:1048D3003712D3A49068CCE0FDFF3395E0FEEFC41C
:1048E300F8540FC868FFEEC454F048FE74272FF540
:1048F30082EE3451F583C083C082EDFB3395E0FA39
:1049030074F32BF582EA345EF583E0D082D08375AD
:10491300F00412D3E112D36C90660312D3A4741F74
:104923002BF582EA3466F583E0906660F09068CCFC
:10493300E0F9FF3395E0FE74612FF582EE3465F5FF
:1049430083E0906661F0E93395E0FEEF25E0FFEE4A
:1049530033FE74BB2FF582EE3466F583E0FEA3E0ED
:10496300FF30E0099054E8E04401F080079054E8F8
:10497300E054FEF0EF30E21290000CE090677DF01F
:10498300900005E0900000F08010900005E0906733
:104993007DF090000CE0900000F07F007E247D7499
:1049A3007C499065FD12D38812CC2112CE7F90658D
:1049B300F112D3A49065F112D388C000C001C002E4
:1049C300C0039068CCE0FF3395E0FEEF7802C33379
:1049D300CE33CED8F924E6F582EE3456F58312D3DE
:1049E3006C7B007A247974784912CC2112CE7FD063
:1049F30003D002D001D00012D1E59065F112D3A407
:104A03007F007E247D747C4990660312D38812CC88
:104A13002112CE7F9066B712D3A49066B712D388C3
:104A2300C000C001C002C0039068CCE0FF3395E032
:104A3300FEEF7802C333CE33CED8F924D6F582EE17
:104A43003457F58312D36C7B007A24797478491236
:104A5300CC2112CE7FD003D002D001D00012D1E5F9
:104A63009066B712D3A49068CDE0FEA3E07802C3AA
:104A730033CE33CED8F924C7F582EE344EF5831204
:104A8300D36C90675C12D3A47F357EFA7D8E7C3C19
:0F4A930090675812D38812CC2112E2F7900011CD
:104AA20012D3A47F357EFA7D8E7C3C90675812D358
:104AB2008812CC2112E2E190673B12D3A47F357EAB
:104AC200FA7D8E7C3C9055DD12D38812CC21900069
:104AD2000D12D3A490000D12D36C12E2F7904E7413
:104AE20012D3A490000D12D36C12E2E190677912F6
:104AF200D3A47F357EFA7D8E7CBC9055E512D38897
:104B020012CC2112E2F7904E6212D3A47F357EFAC4
:104B12007D8E7C3C9055E512D38812CC2112E2E1C5
:104B220090677112D3A47F007E007D007C409000CC
:104B32000D12D38812CC2112E2E17B297ABC79DBF7
:104B4200783A12CC217B227A92797F783F12CB304D
:104B52007B487A5179C7784512CC21C004C005C080
:104B620006C0077B007A00797A78449055E912D31F
:104B72006C12CD2AD003D002D001D00012CB3090DB
:104B82004E6A12D3A47F447E497D7E7C3F904E7450
:104B920012D38812CC2190677912D38812CD2A12AF
:104BA200E44190000D12D3A4904E7412D36C904E37
:104BB2006A12D38812CC21904EBA12D3A49067798C
:104BC20012D36C904E6A12D38812CC219067711264
:104BD200D38812CC21904EAE12D3A490677912D30F
:104BE2006C904E6A12D38812CC21904E6212D388F6
:104BF20012CC21904EB612D3A490000D12D36C1297
:104C0200E2E1C004C005C006C007904E6A12D36C30
:104C120012CE30D003D002D001D00012CC21904E5F
:104C22006212D38812CC217B407AED7998783812BF
:104C3200CC2190665C12D3A490000D12D36C12E2C8
:104C4200E1904E6A12D38812CC2190677112D388F8
:104C520012CC217B407AED7998783812CC2190667B
:054C62006412D3A4223E
:104C67009068CFEFF09065F512D38890655512D311
:104C77006C12CB2C90691C12D3A47F007E007D00A0
:104C87007C4090691C12D38812CC219065A312D363
:104C97008812CC2190678E12D38812CB309068D0BF
:104CA70012D3A49068D012D36CA804A905AA06ABA6
:104CB7000712CC21A804A905AA06AB077FCB7E184B
:104CC7007D897C5612CD2AC004C005C006C0079056
:104CD700694012D3B03EAAAAABD007D006D005D000
:104CE70004120A0A905EEB12D3A49068D012D36C18
:104CF700905EEB12D38812CC217B5B7A827998780D
:104D07003812CC219068D412D3A490673F12D36C89
:104D1700A804A905AA06AB0712CC21A804A905AACD
:104D270006AB077F007E007D807C3F12CB2C90690D
:104D37000412D3A490690412D36C12E1F19067476F
:104D470012D3A47B007A0079B4784390677E12D39C
:104D57006C12CD2A90677512D38812CB30906924D4
:104D670012D3A4905EEB12D3887F487E517DC77C17
:104D77004512CD2AC004C005C006C007906940127D
:104D8700D3B040600000D007D006D005D004120A87
:104D97000A7B337A33791F784112CC21C004C005CE
:104DA700C006C00790690412D36CA804A905AA0617
:104DB700AB0712CC21A804A905AA06AB07D007D0D8
:104DC70006D005D00412CD2A90690812D3A49069A1
:104DD7000812D36C90691C12D38812CC2190673BC0
:104DE70012D38812CC21A804A905AA06AB07900004
:104DF7000112D36C12CB2C905F8F12D3A47F357E18
:104E0700FA7D8E7C3C905F8F12D38812CC2112E200
:104E1700F790690012D3A47F357EFA7D8E7C3C9093
:104E27005F8F12D38812CC2112E2E19068FC12D373
:104E3700A490673B12D36CA804A905AA06AB071276
:104E4700CC217B007A007920784012CC217B007A34
:104E570000790078BF12CB30C004C005C006C00778
:104E670090690812D36C90691C12D38812CC21D098
:104E770003D002D001D00012CC21904E4A12D38821
:104E870012CB3090659F12D3A47F357EFA7D8E7C3E
:104E97003C90659F12D38812CC2112E2F7906910DB
:104EA70012D3A47F357EFA7D8E7C3C90659F12D30A
:104EB7008812CC2112E2E190690C12D3A490690008
:104EC70012D36C90691012D38812CC2190673B12D1
:104ED700D38812CC21C004C005C006C0079068FC67
:104EE70012D36C90690C12D38812CC21D003D00254
:104EF700D001D00012CB2C905F4712D3A490690049
:0F4F070012D36C90690C12D38812CC2190673BA7
:104F160012D38812CC21C004C005C006C007906811
:104F2600FC12D36C90691012D38812CC217B007AC4
:104F360000798078BF12CC21D003D002D001D000F6
:104F460012CB2C905F5712D3A49068FC12D36C90AE
:104F5600691012D38812CC2190673B12D38812CCE9
:104F660021C004C005C006C00790690012D36C902A
:104F7600690C12D38812CC21D003D002D001D00004
:104F860012CB30905F4B12D3A49068FC12D36C9076
:104F9600690C12D38812CC2190673B12D38812CCAD
:104FA60021C004C005C006C00790690012D36C90EA
:104FB600691012D38812CC217B007A00798078BFE1
:104FC60012CC21D003D002D001D00012CB30905F9A
:104FD6005B12D3A490001112D36C90691012D3887F
:104FE60012CC21905F4F12D3A490001112D36C9073
:104FF600690C12D38812CC21905F5F12D3A49069FA
:105006004012D3B04000000090691C12D36C120A03
:105016000A9065A312D38812CC21C004C005C0062D
:10502600C00790691C12D36C90678E12D38812CC7D
:105036002190692412D38812CB30D003D002D0013C
:10504600D00012CB3090692012D3A47FBD7E377D6D
:10505600867C3590692012D38812CB30120B639070
:10506600691412D3A490691412D38890692012D3BC
:105076006C12CB2C7BBD7A377986783512CB307B98
:10508600007A007980784312CC21904E4212D3A444
:1050960090691412D38890692012D36C12CB2C7BA2
:1050A600DB7A0F79C9784012CC21905F8B12D3A49A
:1050B6007F007E007D007C40905F8B12D38812CCEF
:1050C6002112E2F7C004C005C006C00790673F1270
:1050D600D36CA804A905AA06AB0712CC217B007ADB
:1050E600007900783F12CC21D003D002D001D00045
:1050F60012CC21C004C005C006C007905F8B12D336
:105106006C12E2F790673F12D38812CC21905F8B26
:1051160012D38812CB30D003D002D001D00012CBEC
:1051260030905F6F12D3A4905F6F12D36C12E2F7C8
:10513600904E3E12D3A4905F6F12D36C12E2E190B0
:10514600674312D3A490674312D36C90673F12D380
:105156008812CC21A804A905AA06AB077F007E0009
:105166007D807C3F12CB2C90001812D3A4904E3E2B
:0951760012D36C90673F12D3883C
:10517F0012CC21A804A905AA06AB07905F6F12D322
:10518F006C12CB2C90678A12D3A4905F8B12D388AA
:10519F0090678A12D36C12CB2C9068F812D3A4901C
:1051AF0068F812D36C12DFCC7BBD7A3779867835ED
:1051BF0012CDC360025039905F6F12D36CC004C020
:1051CF0005C006C00790001812D3889068F812D354
:1051DF006C12CD2AA804A905AA06AB07D007D006E2
:1051EF00D005D00412CB2C905F6F12D3A402512D97
:1051FF0090673F12D38890674312D36C12CB2C90D9
:10520F005EEB12D38812CC21904E5212D3A490672A
:10521F004712D36C905EEB12D38812CC21904E3E86
:10522F0012D38812CC21904E5612D3A4900018128C
:10523F00D36C905EEB12D38812CC2190608912D37D
:10524F00A49068D412D36C12CE30904E3E12D388F5
:10525F0012CC2190001812D38812CD2A90692812EF
:10526F00D3A490674712D36C9068D412D38812CC12
:10527F002190674312D38812CC2190001812D38843
:10528F0012CD2A90692C12D3A4905F5712D36C9031
:10529F004E5612D38812CC21C004C005C006C007D9
:1052AF00905F4712D36C904E5212D38812CC21D0FC
:1052BF0003D002D001D00012CB309068E412D3A4F7
:1052CF00905F5B12D36C904E5612D38812CC21C0D4
:1052DF0004C005C006C007905F4B12D36C904E52AE
:1052EF0012D38812CC21D003D002D001D00012CB20
:1052FF00309068E812D3A4905F5F12D36C904E5633
:10530F0012D38812CC21C004C005C006C007905F1D
:10531F004F12D36C904E5212D38812CC21D003D09F
:10532F0002D001D00012CB30904E6612D3A4905F02
:10533F005712D36C90692C12D38812CC21C004C0A1
:10534F0005C006C007905F4712D36C90692812D32F
:10535F008812CC21D003D002D001D00012CB3090D4
:10536F0068EC12D3A4905F5B12D36C90692C12D3AC
:10537F008812CC21C004C005C006C007905F4B1235
:10538F00D36C90692812D38812CC21D003D002D0CD
:09539F0001D00012CB309068F03F
:1053A80012D3A4905F5F12D36C90692C12D3881229
:1053B800CC21C004C005C006C007905F4F12D36C53
:1053C80090692812D38812CC21D003D002D001D002
:1053D8000012CB309068F412D3A47FB77E597D8039
:1053E8007C3F90655512D38812CC2190675C12D30C
:1053F8008812CB3090678612D3A490678612D36C3C
:10540800120B63A804A905AA06AB0790678612D3F6
:105418006C12CB2C7BDB7A0F79C9784012CC2190A7
:10542800678612D3A490678612D36C12E2F77B00CA
:105438007A00798078BF12CC21904E5A12D3A4906A
:10544800678612D36C12E2E190676412D3A4904E7F
:105458005A12D36C9068E812D38812CC21C004C0C9
:1054680005C006C00790676412D36C9068E412D335
:105478008812CC21D003D002D001D00012CB2C90BE
:1054880065A712D3A490676412D36C9068E812D30E
:105498008812CC21C004C005C006C007904E5A121D
:1054A800D36C9068E412D38812CC21D003D002D0F8
:1054B80001D00012CB309065AB12D3A4904E661287
:1054C800D36C9065C912D3A4904E5A12D36C9068CD
:1054D800F012D38812CC21C004C005C006C00790C2
:1054E800676412D36C9068EC12D38812CC21D00375
:1054F800D002D001D00012CB2C9068D812D3A4903F
:10550800676412D36C9068F012D38812CC21C0045F
:10551800C005C006C007904E5A12D36C9068EC12B2
:10552800D38812CC21D003D002D001D00012CB30C6
:105538009068DC12D3A49068F412D36C9068E012DF
:10554800D3A4904EAE12D3889065A712D36C12CB19
:105558002C904E7912D3A4904EB612D3889065AB96
:1055680012D36C12CB2C904E9112D3A4904EBA1237
:10557800D3889065C912D36C12CB2C904EA012D34D
:10558800A4904E9112D36C904E9112D38812CC21D4
:10559800C004C005C006C007904E7912D36C904E67
:1055A8007912D38812CC21D003D002D001D00012B6
:1055B800CB30C004C005C006C007904EA012D36C03
:1055C800904EA012D38812CC21D003D002D001D0A3
:0D55D8000012CB3012E1F1904E4612D3A428
:1055E500904E6212D36C904E9112D38812CC2190BA
:1055F500677912D38812CC21C004C005C006C00744
:1056050090677112D36C904E7912D38812CC219089
:10561500677912D38812CC21D003D002D001D000F3
:1056250012CB30C004C005C006C007904E7412D31B
:105635006C904EA012D38812CC21D003D002D00199
:10564500D00012CB30904EB212D3A490677112D312
:105655006C904E7912D38812CC21904E7412D38857
:1056650012CC217B007A00798078BF12CC21C0044E
:10567500C005C006C007904E6212D36C904E9112C1
:10568500D38812CC21904E7412D38812CC21A80451
:10569500A905AA06AB07D007D006D005D00412CBC2
:1056A5002CC004C005C006C00790677912D36C9062
:1056B5004EA012D38812CC21D003D002D001D00045
:1056C50012CB30904EA612D3A4904E6212D36C909A
:1056D5004E7912D38812CC21C004C005C006C0077C
:1056E50090677112D36C904E9112D38812CC21D051
:1056F50003D002D001D00012CB2C904EAA12D3A415
:10570500904E4612D388904EB212D36C12CD2A9089
:105715004E4E12D3A4904E4E12D36C904E4E12D3D1
:105725008812CC21A804A905AA06AB077F007E0034
:105735007D807C3F12CB2C12E1F190675412D3A4EB
:1057450090675412D388904E4E12D36C12CD2A1204
:10575500E4417B357AFA798E783C12CD2A906782BE
:1057650012D3A4904EA612D388904EAA12D36C12CF
:10577500CD2A12E4417B357AFA798E783C12CD2A0E
:1057850090676012D3A490608912D3889065C9127E
:10579500D36C12CD2A90675012D3A490675012D3C0
:1057A5006C90675012D38812CC21A804A905AA06CB
:1057B500AB077F007E007D807C3F12CB2C12E1F190
:1057C500A804A905AA06AB0790675012D36C12CDA1
:1057D5002A12E4417B337A337965784212CC2190E1
:1057E500000612D3A49065A712D3889065AB12D397
:1057F5006C12CD2A12E4417B337A337965784212F3
:10580500CC21904E7012D3A47F007E007D007C00D9
:105815009065A712D38812CDC3501A904E7012D33B
:10582500887F007E007D347C4312CB2C904E701215
:10583500D3A40259197F007E007D007C009065A7E6
:1058450012D38812CDC3602F402D7F007E007D00CE
:0B5855007C009065AB12D38812CDC31D
:10586000501A904E7012D36C7B007A00798078BF0A
:1058700012CC21904E7012D3A40259197F007E00E1
:105880007D007C009065A712D38812CDC3603040A4
:105890002E7F007E007D007C009065AB12D38812C5
:1058A000CDC3601B4019904E7012D3887F007E00DC
:1058B0007DB47C4312CB2C904E7012D3A4805A7FBF
:1058C000007E007D007C009065A712D38812CDC3B6
:1058D000701BFFFEFDFC9065AB12D38812CDC34058
:1058E0000C904E7012D3B043870000802C7F007E56
:1058F000007D007C009065A712D38812CDC370197B
:10590000FFFEFDFC9065AB12D38812CDC3500A9008
:105910004E7012D3B042B400007F007E007D347C14
:1059200043904E7012D38812CDC35019904E70120E
:10593000D36C7B007A00798078BF12CC21904E70B6
:1059400012D3A4802A7F007E007D347C43904E7069
:1059500012D38812CDC34017904E7012D3887F00A7
:105960007E007DB47C4312CB2C904E7012D3A47F6A
:10597000007E007D007C00904EA612D38812CDC31D
:10598000501A90676012D36C7B007A0079347843A8
:1059900012CB3090676012D3A4025A377F007E008A
:1059A0007D007C00904EA612D38812CDC3602E409D
:1059B0002C7F007E007D007C00904EAA12D38812BE
:1059C000CDC350197F007E007DB47C439067601288
:1059D000D38812CB3090676012D3A4805A7F007EA8
:1059E000007D007C00904EA612D38812CDC3701BA0
:1059F000FFFEFDFC904EAA12D38812CDC3400C903E
:105A0000676012D3B042B40000802C7F007E007D1E
:105A1000007C00904EA612D38812CDC37019FFFEF1
:105A2000FDFC904EAA12D38812CDC3500A90676035
:105A300012D3B04387000090666412D3889068DC6C
:105A400012D36C12CB2C904E9112D38812CC21C061
:105A500004C005C006C00790665C12D3889068D861
:105A600012D36C12CB2C904E7912D38812CC21D049
:105A700003D002D001D00012CB30C004C005C00654
:105A8000C007904EA012D36C9068E012D38812CC5D
:105A900021D003D002D001D00012CB30904E46125C
:105AA000D38812CD2A90691812D3A47F007E007D7E
:105AB000807CBF9065FD12D38812CC2190691812AA
:105AC000D38812CC217B207A7B7955784012CC2167
:105AD000905F6712D3A49065FAE020E403025BD7DD
:105AE0007B007A40791C7846905F6712D36C12CDA8
:105AF0002A12CE7F90693012D3A4905F6712D36CC4
:105B000012CE7F7B107A277900780012E6B5AC00C0
:105B1000AD01AE02AF0390693412D3A47F107E278B
:105B20007D007C0090693012D38812D200906938D1
:105B300012D3A47FC47E097D007C0090693412D307
:015B400088DC
:105B4100C312D341501290693812D36CE412CE4182
:105B5100905F6712D3A480527F4C7E1D7D007C0034
:105B610090693412D388C312D3414020906938120E
:105B7100D36CEF2410FFEE3427FEE43DFDE43CFC42
:105B8100E412CE41905F6712D3A4801E906938124F
:105B9100D36CEF2488FFEE3413FEE43DFDE43CFCBE
:105BA100E412CE41905F6712D3A47F007E007D0096
:105BB1007C0090691812D38812CDC36019401790E8
:105BC1005F6712D36C7B007A00798078BF12CC2199
:105BD100905F6712D3A47F007E247D747C49906519
:105BE100FD12D38812CC2112CE7FC004C005C0069D
:105BF100C007905F6712D36C12CE7FD003D002D062
:105C010001D00012D1E590655D12D38812D1E590E3
:105C110065F112D3A49065F112D388C000C001C010
:105C210002C0039068CFE0FF3395E0FEEF7802C336
:105C310033CE33CED8F924E6F582EE3456F583120D
:105C4100D36C7B007A247974784912CC2112CE7FEF
:105C5100D003D002D001D00012D1E59065F112D36A
:105C6100A49065F112D388C000C001C002C00390A6
:105C710068CFE0FF3395E0FEEF7802C333CE33CE39
:105C8100D8F92493F582EE345FF58312D36C12CEEA
:105C91007FD003D002D001D00012D1E59065F1127E
:105CA100D3A47F007E007D807CBF90660312D388E1
:105CB10012CC2190691812D38812CC217B207A7BD7
:105CC1007955784012CC2190655912D3A47F007E7A
:105CD100247D747C4990660312D38812CC2112CEA4
:105CE1007FC004C005C006C00790655912D36C126D
:105CF100CE7FA804A905AA06AB07D007D006D00518
:105D0100D00412D1F29066B712D3A49066B712D321
:105D110088C000C001C002C0039068CFE0FF339586
:105D2100E0FEEF7802C333CE33CED8F924D6F58224
:105D3100EE3457F58312D36C7B007A247974784959
:105D410012CC2112CE7FD003D002D001D00012D1CB
:105D5100E59066B712D3A490001CE0FCA3E0FDE43B
:105D610012CE46120B6BC004C005C006C007906579
:105D71005512D36C120B6BA804A905AA06AB07D068
:105D810007D006D005D00412CDC36039905F6B12E5
:105D9100D36C7B007A007980783F12CB30905F6BB7
:105DA10012D3A490001CE0FCA3E0FDE412CE467BDC
:105DB100007A007980783F12CB3012CE7F90001CA0
:065DC100EEF0A3EFF0225A
:105DC700905E73E4F0A3740DF0905C8A12D3B04335
:105DD7007F84129055F512D3B000012F689058C6F2
:105DE70012D3B0421DE9449059B612D3B04148933B
:105DF700619054ED12D3B042CAE17C90503712D370
:105E0700B03AA170FE905D8312D3B042E8998C90AE
:105E17005B9612D3B04371E0AA905AA612D3B0B4DE
:105E27009652E8904F4712D3B043D98F5C905127D1
:105E370012D3B04311E66690512B12D3B04311F938
:105E47009A90512F12D3B04311E66690513312D373
:105E5700B04311E6669065617404F090661FF09098
:105E670066BCE054FEF054FDFFF0FB9057D612D30A
:105E7700B0000000009056E612D3B000000000EB1F
:105E870044109066BCF078A17C607D017BFF7AB7F7
:105E970079427E007F0612D558905E75E4F0A374B0
:105EA7000DF0905C8E12D3B0437EBE349055F9123C
:105EB700D3B00001494D9058CA12D3B0432A3E22AD
:105EC7009059BA12D3B041587B179054F112D3B0FE
:105ED70042C5176690503B12D3B03D0F27A0905D87
:105EE7008712D3B04395F3EB905B9A12D3B04396E6
:105EF700D8BE905AAA12D3B033D6BF95904F4B1243
:105F0700D3B043D9966690513712D3B04311D99A7B
:105F170090513B12D3B04311E66690513F12D3B074
:105F27004311E66690514312D3B04311E66690657C
:105F3700627404F0906620F09066BEE054FEF05460
:105F4700FDF04410F09057DA12D3B0000000009033
:105F570056EA12D3B00000000078B57C607D017B63
:105F6700FF7AB779497E007F0612D558905E77E4AD
:105F7700F0A3740DF0905C9212D3B0437E8AC49064
:105F870055FD12D3B000012F9D9058CE12D3B043C8
:105F9700A1E9C79059BE12D3B04164A8C59054F582
:105FA70012D3B041FB78A190503F12D3B03D0FDD23
:105FB700A9905D8B12D3B04341FB3D905B9E12D3FA
:105FC700B0439555B5905AAE12D3B036A5C2479097
:105FD7004F4F12D3B043D9F47B90514712D3B043FC
:105FE70011DEB890514B12D3B04311D99A90514F4B
:105FF70012D3B04311E3D790515312D3B04311E8F2
:10600700F69065637404F0906621F09066C0E054E2
:10601700FEF054FDFFF0FB9057DE12D3B0000000F6
:10602700009056EE12D3B000000000EB44109066CB
:10603700C0F078C97C607D017BFF7AB779507E001C
:106047007F0612D558E4906668F0A304F0A304F025
:106057007F0374682FF582E43466F583EFF00FEF62
:10606700B43CEF906770743CF0904EA4E4F0A374D6
:036077003CF022D8
:10607A007BFF7AB779571208A37BFF7AB7795C124C
:10608A0008A37BFF7AB779861208A37BFF7AB779D0
:10609A00A21208A37BFF7AB779B91208A312E720E4
:1060AA00AE07EEC39431400BEED394335005EE2481
:0D60BA00D0FF22EE4420FFBF71DA7F71227B
:1060C700E49067DBF012607AEF24FE7003026173DD
:1060D7001470030262052492700302620B2470702D
:1060E700E47BFF7AB779CB1208A390E102E0448002
:1060F700F0E49067DBF030986E12E720EF24CE6073
:106107003324FD603B14601424FE601C2404703D9E
:10611700126D0B90E102E04420F08042126D019075
:10612700E102E04420F08036126D2990E102E0445C
:1061370020F0802A126D3390E102E04420F0801EA7
:1061470090E102E054F0F0E054DFF0801190E102BA
:10615700E054F0F0E054DFF09067DB7401F09067F3
:10616700DBE060030260CC126480808A7BFF7AB830
:106177007906905EEF12D36C90679512D3A412D86C
:10618700AB7B017A6779DC9068BB12D4347BFF7AEA
:10619700A979731209D39067DE12D3A49067DCE064
:1061A7007002A3E0600C9067DE12D36C905EEF1272
:1061B700D3A47BFF7AB8791A905C8612D36C906768
:1061C7009512D3A412D8AB7B017A6779DC9068BBB0
:1061D70012D4347BFF7AA979731209D39067DE1240
:1061E700D3A49067DCE07002A3E0600C9067DE1236
:1061F700D36C905C8612D3A412620C0260CC12623C
:05620700530260CC22EF
:10620C009054E8E04404F090E102E04420F07BFF7D
:10621C007AB279801208A3126A4990E102E0540F15
:10622C00601230980A12E72090688FEFF080051208
:10623C00648080E39054E8E054FBF090E102E05479
:07624C00DFF0E054F0F02246
:106253007BFF7AB8792E90608D12D36C906795127C
:10626300D3A4905F7312D36C90679912D3A49060F8
:106273009112D36C90679D12D3A4905F7712D36C65
:106283009067A112D3A490609512D36C9067A51266
:10629300D3A4905F7B12D36C9067A912D3A49060B0
:1062A3009912D36C9067AD12D3A4905F7F12D36C15
:1062B3009067B112D3A412D8AB7BFF7AB8796F90F1
:1062C300609D12D36C90679512D3A4905F8312D311
:1062D3006C90679912D3A412D8AB7BFF7AB8797FFD
:1062E3001208A312E7209067E8EFF0C3943140400F
:1062F300E0FFD394355039EF24CFF0E0FB25E025C0
:10630300E0248DF582E43460F58312D36C905EEF64
:1063130012D3A4EB25E025E02473F582E4345FF582
:106323008312D36C905C8612D3A412620C02625364
:106333009067E8E0442064736003026472A3F0A3EF
:10634300F0C39067EAE094059067E9E094004003A6
:106353000262537BFF7AB87996E0FEA3E0FF240143
:10636300906796F0E43E906795F0EF7802C333CEE2
:1063730033CED8F9248DF582EE3460F58312D36CD5
:1063830090679712D3A412D8AB7B017A6779E69012
:1063930068BB12D4347BFF7AA979731209D390674F
:1063A300E212D3A49067E6E07002A3E06032906744
:1063B300E212D36CC004C005C006C0079067E9E0D1
:1063C300FEA3E07802C333CE33CED8F9248DF58211
:1063D300EE3460F583D007D006D005D00412D3A4E1
:1063E3007BFF7AB879B69067E9E0FEA3E07802C351
:1063F30033CE33CED8F92473F582EE345FF58312AE
:10640300D36C90679512D3A412D8AB7B017A6779CA
:10641300E69068BB12D4347BFF7AA979731209D34F
:106423009067E212D3A49067E6E07002A3E06032C3
:106433009067E212D36CC004C005C006C007906722
:10644300E9E0FEA3E07802C333CE33CED8F9247358
:10645300F582EE345FF583D007D006D005D0041261
:10646300D3A49067E9E475F00112D19A02634490D2
:0D64730067E8E04420647160030262532278
:10648000E4FF120C7B9066B1E0FEA3E0FFC3E52DB4
:106490009FFFE52C9EFEEF253EF53EEE353DF53D9A
:1064A000A2E713F53DE53E13F53E9068FAE52CF0C2
:1064B000A3E52DF07F01120C7B906601E0FEA3E0C6
:1064C000FFC3E52D9FFFE52C9EFEEF252FF52FEE58
:1064D000352EF52EA2E713F52EE52F13F52F906834
:1064E000FCE52CF0A3E52DF0AC3DAD3EEC12CE4624
:1064F0009066B312D38812CD2A9068F212D3A4AC5E
:106500002EAD2FEC12CE4690660712D38812CD2AFC
:106510009068F612D3A49054E8E020E3457F007E13
:10652000007D347C439068F212D38812CDC3601B87
:1065300040199068F212D36C7B007A00793478436A
:1065400012CB2C9068F212D3A480179068F212D369
:106550006C7B007A007934784312CB309068F21269
:10656000D3A47BFF7AB879D39068FAE0FFA3E090D8
:106570006795CFF0A3EFF09068F212D36C90679715
:1065800012D3A49068FCE0FFA3E090679BCFF0A338
:10659000EFF09068F612D36C90679D12D3A412D8D6
:1065A000AB7BFF7AB5794390679512D4349068F24B
:1065B00012D36C90679812D3A49068F612D36C90A3
:1065C000679C12D3A47B017A6879CA12D8A57FC0D0
:0D65D0001205017B017A6879CA1208C12208
:1065DD007BFF7AB879FE1208A37BFF7AB9793E1258
:1065ED0008A312E7208F26E526442064736003027A
:1065FD00669D7BFF7AB9796D90659DE0FFA3E09074
:10660D006795CFF0A3EFF012D8AB7B017A6779DBFA
:10661D009068BB12D4347BFF7AA979731209D39099
:10662D0067DD12D3A49067DBE07002A3E0601190E8
:10663D0067DD12D36C12CE7F90659DEEF0A3EFF067
:10664D007BFF7AB97994906083E0FFA3E090679522
:10665D00CFF0A3EFF012D8AB7B017A6779DB9068AE
:10666D00BB12D4347BFF7AA979731209D39067DDFD
:10667D0012D3A49067DBE07002A3E0605B9067DD4E
:10668D0012D36C12CE7F906083EEF0A3EFF08048B2
:10669D00E5264420646D70407BFF7AB979B9120804
:1066AD00A37BFF7AB279801208A330980F12E720EE
:1066BD00EF44202492700302679480001267958046
:1066CD00E930980F12E720EF4420249270030267FF
:1066DD0094800012679580E97B017A6779DB906879
:1066ED004A12D4347BFF7ABA791D12099C9067DB6C
:1066FD00E07002A3E0600CEE3395E0FDFC9065EDDB
:10670D0012D3A47BFF7ABA793B1208A312E7208F2C
:10671D0026E5264420FFBF79099065FAE04402F092
:10672D00800ABF6E079065FAE054FDF07BFF7ABAE0
:10673D0079661208A312E720EF44202492600D24FD
:10674D00F570109065FAE04405F080079065FAE069
:10675D0054FBF07BFF7ABA79971208A312E720EF6A
:10676D0044202492601324FC701D9065FAE04408C7
:10677D00F090E102E04450F0229065FAE054F7F019
:08678D0090E102E054AFF0229C
:106795007F03120C7B7BFF7ABA79CA906795E52C4B
:0967A500F0A3E52DF012D8AB229F
:1067AE009068CAEFF09054E8E020E24B90E102E0EE
:1067BE0054F0F0904EC312D36C90673312D3A49062
:1067CE00676C12D3A4904EBE12D36C905C8612D31B
:1067DE008812CDC36019401790E000E030E00890B9
:1067EE00E102E04420F02290E102E054DFF022903A
:1067FE00E102E054DFF022904EBE12D36C905C8624
:10680E0012D38812CDC340030268E97F007E007D5B
:10681E00407CC0905C8612D38812CDC3405390E06A
:10682E0000E030E00990E102E04420F0800790E1C2
:10683E0002E054DFF09054E8E030E0357FCD7ECCBE
:10684E007DCC7C3D9065FD12D38812CDC360114086
:10685E000F9065FAE030E1089068CAE0FF123D92B1
:10686E009065F9E0FEA3E0FF30E20630E003123B54
:10687E00527F007E007D407CC0905C8612D38812D1
:10688E00CDC3502190E102E054DFF09065FAE02094
:10689E00E0139054E912D36C90673712D3A490652D
:1068AE00FAE04401F09054E8E030E424905F87125F
:1068BE00D36C905C8612D38812CDC350139068CAE5
:1068CE00E0FF123658905C8612D3B0C170000022E1
:1068DE0012086690E102E054F0F0229065F9E0A310
:1068EE0030E02B7FCD7ECC7DCC7C3D9065FD12D3F0
:1068FE008812CDC36011400F9065FAE030E1089028
:10690E0068CAE0FF123D929065F9E054FEF0906582
:10691E00F112D36C9054E912D3A490E102E044201A
:10692E00F09054E8E020E503026A459065E512D345
:10693E006C905C8612D38812CDC36010400E9065A9
:10694E00E512D36C905C8612D3A4801D9065E11283
:10695E00D36C905C8612D38812CDC3500C9065E137
:10696E0012D36C905C8612D3A49065D912D36C901E
:10697E0065DD12D38812CDC3604640449065DD12AA
:10698E00D36C905EEF12D38812CDC36011400F907E
:10699E0065DD12D36C905EEF12D3A4026A4590654A
:1069AE00D912D36C905EEF12D38812CDC34003027E
:1069BE006A459065D912D36C905EEF12D3A480779E
:1069CE009065D912D36C9065DD12D38812CDC35069
:1069DE00669065D912D36C905EEF12D38812CDC338
:1069EE0050237F007E007D347C43905EEF12D3886F
:1069FE0012CDC36010400E9065D912D36C905EEF2D
:106A0E0012D3A480329065DD12D36C905EEF12D358
:106A1E008812CDC36021401F7F007E007D347C43F1
:106A2E00905EEF12D38812CDC3500C9065DD12D359
:0B6A3E006C905EEF12D3A4126A492294
:106A4900E4FF120C7B9066B1E0FEA3E0FFC3E52DE5
:106A59009FFFE52C9EFEEF253EF53EEE353DF53DCB
:106A6900A2E713F53DE53E13F53E7F01120C7B903D
:106A79006601E0FEA3E0FFC3E52D9FFFE52C9EFE26
:106A8900EF252FF52FEE352EF52EA2E713F52EE57E
:106A99002F13F52FAC3DAD3EEC12CE469066B312E6
:106AA900D38812CD2A9068CC12D3A4AC2EAD2FEC8A
:106AB90012CE4690660712D38812CD2A9068D0125A
:106AC900D3A49054E8E020E3457F007E007D347C28
:106AD90043905EEF12D38812CDC350197F007E0018
:106AE9007D347C43905EEF12D38812CB309068D40A
:106AF90012D3A480257F007E007D347CC3905EEF95
:106B090012D38812CB309068D412D3A4800C905E33
:106B1900EF12D36C9068D412D3A4905C8612D36C14
:106B29009068D812D3A49065F9E0A330E52E906857
:106B3900D412D36C7B007A007934784312CB30902D
:106B490068D412D3A49068D812D3887F007E007DC0
:106B5900347C4312CB2C9068D812D3A49068D412F9
:106B6900D36C90660B12D38812CB309068D412D3B1
:106B7900A49068D812D36C90660F12D38812CB30C8
:106B89009068D812D3A47F007E007DB47C439068BE
:106B9900D412D38812CDC3601B40199068D412D384
:106BA9006C7B007A0079B4784312CB2C9068D412AC
:106BB900D3A4802A7F007E007D007C009068D412D7
:106BC900D38812CDC350179068D412D36C7B007A46
:106BD9000079B4784312CB309068D412D3A47F00E3
:106BE9007E007D347C439068D812D38812CDC3408F
:106BF9000C9068D812D3B043340000801F7F007E08
:106C0900007D007C009068D812D38812CDC3600241
:106C1900500A9068D812D3B0000000009068D412CE
:106C2900D3889068CC12D36C12CB2C12DFCCC00461
:106C3900C005C006C0077F007E007D407C4090668D
:106C49001312D38812CC21A804A905AA06AB07D030
:106C590007D006D005D00412CDC3500990E102E057
:106C69004480F0800790E102E0547FF09068D412EC
:106C7900D3889068CC12D36C12CB2C12DFCC9066DF
:106C89001312D38812CDC3501D9068CC12D36C90C7
:106C990068D412D38812CDC360074005126D0180F4
:106CA90008126D0B8003126D159068D812D3889065
:086CB90068D012D36C12CB2C41
:106CC10012DFCC90661712D38812CDC3502E906874
:106CD100D012D36C9068D812D38812CDC36006400D
:106CE10004126D29227F007E007D007C009068D80F
:106CF10012D38812CDC34007126D3322126D3D228B
:0A6D010090E102E054FC4402F0228D
:0A6D0B0090E102E054FC4401F02284
:106D1500904EC312D36C90676C12D3A490E102E03D
:046D250054FCF02208
:0A6D290090E102E054F34408F02268
:0A6D330090E102E054F34404F02262
:106D3D00904EC312D36C90673312D3A490E102E04E
:046D4D0054F3F022E9
:106D51007BFF7ABA79E49066B1E0FFA3E090679592
:106D6100CFF0A3EFF0900015E0FFA3E0906797CF7D
:106D7100F0A3EFF0906601E0FFA3E0906799CFF0F8
:106D8100A3EFF0906768E0FFA3E090679BCFF0A3CB
:106D9100EFF012D8AB7BFF7ABB791E120BD3906751
:106DA100DBEFF0BF010C9065F9E04440F0A3E0F0A7
:106DB100800D9067DBE070079065F9E054BFF07BD0
:106DC100FF7ABB794E120BD39067DBEFF064016061
:106DD100079067DBE070E822E4FF120C7B9066B15C
:106DE100E52CF0A3E52DF07F01120C7B906601E507
:106DF1002CF0A3E52DF07BFF7ABB7991120BD39098
:106E010067DBEFF0640160079067DBE070E822E484
:106E1100FF120C7B900015E52CF0A3E52DF07F010E
:106E2100120C7B906768E52CF0A3E52DF012052B81
:016E3100223E
:106E32007BFF7ABB79D39066B1E0FFA3E0906795C0
:106E4200CFF0A3EFF0900015E0FFA3E0906797CF9B
:106E5200F0A3EFF012D8AB7B017A6779DB9068BBC5
:106E620012D4347BFF7ABB79F81209D39067DD1212
:106E7200D3A49067DBE07002A3E060119067DD129B
:106E8200D36C12CE7F9066B1EEF0A3EFF07B017A65
:106E92006779DB9068BB12D4347BFF7ABC7911121C
:106EA20009D39067DD12D3A49067DBE07002A3E000
:106EB20060119067DD12D36C12CE7F900015EEF058
:106EC200A3EFF07BFF7ABC7929120BD3EFB4010C4C
:106ED2009065F9E04440F0A3E0F0800AEF7007907B
:106EE20065F9E054BFF07BFF7ABC7958906601E007
:106EF200FFA3E0906795CFF0A3EFF0906768E0FF03
:106F0200A3E0906797CFF0A3EFF012D8AB7B017AA2
:106F12006779DB9068BB12D4347BFF7ABC797F122D
:106F220009D39067DD12D3A49067DBE07002A3E07F
:106F320060119067DD12D36C12CE7F906601EEF085
:106F4200A3EFF07B017A6779DB9068BB12D4347BC4
:106F5200FF7ABC79981209D39067DD12D3A49067A7
:106F6200DBE07002A3E060119067DD12D36C12CEF9
:0D6F72007F906768EEF0A3EFF012052B2270
:106F7F007BFF7ABC79B01208A312E7209067E3EF8A
:106F8F00F04420647960030271719054E8E044107A
:106F9F00F07BFF7ABC79DC9055F112D36C9067953A
:106FAF0012D3A412D8AB7B017A6779DB9068BB123E
:106FBF00D4347BFF7AA979731209D39067DF12D388
:106FCF00A49067DBE07002A3E0600C9067DF12D340
:106FDF006C9055F112D3A47BFF7ABD7901904F3F8E
:106FEF0012D36C90679512D3A412D8AB7B017A673A
:106FFF0079DB9068BB12D4347BFF7AA979731209BD
:10700F00D39067DF12D3A49067DBE07002A3E06038
:10701F000C9067DF12D36C904F3F12D3A47BFF7A93
:10702F00BD79221208A312E7209067E3EFF0442006
:10703F00647960030271689065F9E04402F0A3E09F
:10704F00F07BFF7ABD794D9065CD12D36C9067952B
:10705F0012D3A412D8AB7B017A6779DB9068BB128D
:10706F00D4347BFF7AA979731209D39067DF12D3D7
:10707F00A49067DBE07002A3E0600C9067DF12D38F
:10708F006C9065CD12D3A47BFF7ABD796A9065D1E0
:10709F0012D36C90679512D3A412D8AB7B017A6789
:1070AF0079DB9068BB12D4347BFF7AA9797312090C
:1070BF00D39067DF12D3A49067DBE07002A3E06088
:1070CF000C9067DF12D36C9065D112D3A47BFF7A3B
:1070DF00BD798312D8AB7B017A6779E412091DEF72
:1070EF004E602F9067E4E04420249A601824F160EA
:1070FF000C240970189066637401F0801590666314
:10710F007402F0800D9066637404F08005E490665D
:10711F0063F07BFF7ABD799F12D8AB7B017A6779D9
:10712F00E412091DEF4E604B9067E4E04420249A6F
:10713F00601824F1600C240970189066627401F0D5
:10714F0080319066627402F080299066627404F058
:10715F008021E4906662F0801A9065F9E054FDF0AA
:10716F0080119067E3E04420FFBF6E079054E8E082
:10717F0054EFF07BFF7ABD79BB1208A312E7209082
:10718F0067E3EFF04420647960030272BD9054E826
:10719F00E04420F07BFF7ABD79E39065D912D36C80
:1071AF0090679512D3A412D8AB7B017A6779DB90E5
:0B71BF0068BB12D4347BFF7AA97973FF
:1071CA001209D39067DF12D3A49067DBE07002A3A1
:1071DA00E0600C9067DF12D36C9065D912D3A47B60
:1071EA00FF7ABE79089065DD12D36C90679512D349
:1071FA00A412D8AB7B017A6779DB9068BB12D434CE
:10720A007BFF7AA979731209D39067DF12D3A4900E
:10721A0067DBE07002A3E0600C9067DF12D36C902A
:10722A0065DD12D3A47BFF7ABE79299065E112D37A
:10723A006C90679512D3A412D8AB7B017A6779DB7D
:10724A009068BB12D4347BFF7AA979731209D39060
:10725A0067DF12D3A49067DBE07002A3E0600C90B2
:10726A0067DF12D36C9065E112D3A47BFF7ABE79F3
:10727A004A9065E512D36C90679512D3A412D8ABE5
:10728A007B017A6779DB9068BB12D4347BFF7AA9D9
:10729A0079731209D39067DF12D3A49067DBE07089
:1072AA0002A3E0601F9067DF12D36C9065E512D3EA
:1072BA00A480119067E3E04420FFBF6E079054E872
:1072CA00E054DFF07BFF7ABE796B1208A312E72045
:1072DA009067E3EFF044206479600302738C906551
:1072EA00F9E054F7F07BFF7ABE7993905D81E0FF75
:1072FA00A3E0906795CFF0A3EFF012D8AB7B017AA9
:10730A006779DB90684A12D4347BFF7AA9797312C1
:10731A00099C9067DDEEF0A3EFF09067DBE0700266
:10732A00A3E0600F9067DDE0FFA3E0905D81CFF0FE
:10733A00A3EFF07BFF7ABE79C29066A5E0FFA3E0D7
:10734A00906795CFF0A3EFF012D8AB7B017A6779FB
:10735A00DB90684A12D4347BFF7AA9797312099CAC
:10736A009067DDEEF0A3EFF09067DBE07002A3E038
:10737A0060249067DDE0FFA3E09066A5CFF0A3EF5D
:10738A00F0229067E3E04420FFBF6E0A9065F9E0BF
:07739A004408F0A3E0F0221B
:1073A1007BFF7ABE79F990661312D36C90679512C0
:1073B100D3A412D8AB7B017A6779DB9068BB12D476
:1073C100347BFF7AA979731209D39067DD12D3A4B4
:1073D1009067DBE07002A3E0600C9067DD12D36C74
:1073E10090661312D3A47BFF7ABF791B90661712A4
:1073F100D36C90679512D3A412D8AB7B017A6779CD
:10740100DB9068BB12D4347BFF7AA979731209D35C
:107411009067DD12D3A49067DBE07002A3E0600CFB
:107421009067DD12D36C90661712D3A47BFF7ABFED
:10743100793990660B12D36C90679512D3A412D848
:10744100AB7B017A6779DB9068BB12D4347BFF7A1E
:10745100A979731209D39067DD12D3A49067DBE099
:107461007002A3E0600C9067DD12D36C90660B1282
:10747100D3A47BFF7ABF795990660F12D36C9067C2
:107481009512D3A412D8AB7B017A6779DB9068BBE4
:1074910012D4347BFF7AA979731209D39067DD1274
:1074A100D3A49067DBE07002A3E0600C9067DD126B
:0974B100D36C90660F12D3A422E3
:1074BA0078DB7C677D017BFF7AC979C87E007F090A
:1074CA0012D55878E47C677D017BFF7AC979D17E31
:1074DA00007F0612D55878EA7C677D017BFF7AC95E
:1074EA0079D77E007F0F12D55878F97C677D017BAA
:1074FA00FF7AC979E67E007F0612D55878FF7C6745
:10750A007D017BFF7AC979EC7E007F1212D55890F3
:10751A0054E7E0FFA3E0906811CFF0A3EFF07BFF00
:10752A007AB779571208A37B017A4E797D906795CD
:10753A0012D4349055DD12D36C90679812D3A4906C
:10754A0055E112D36C90679C12D3A49055E912D3DB
:10755A006C9067A012D3A47BFF7ABF79A912D8AB2B
:10756A007BFF7ABF79E19066B1E0FFA3E09067956F
:10757A00CFF0A3EFF0900015E0FFA3E0906797CF5C
:10758A00F0A3EFF0906601E0FFA3E0906799CFF0D7
:10759A00A3EFF0906768E0FFA3E090679BCFF0A3AA
:1075AA00EFF012D8AB9065F9E0A330E6097BFF7AD9
:1075BA00C0791212D8AB7BFF7AB2798012D8AB7B32
:1075CA00FF7AC0791990661312D36C90679512D31B
:1075DA00A490661712D36C90679912D3A412D8ABF1
:1075EA007BFF7AC0794C90660B12D36C9067951228
:1075FA00D3A490660F12D36C90679912D3A412D8B1
:10760A00AB9054E8E020E4030276A07BFF7AC079CD
:10761A007F9055F112D36C90679512D3A4904F3F87
:10762A0012D36C90679912D3A412D8AB9065F9E083
:10763A00A330E1579065CD12D36C90679512D3A40D
:10764A009065D112D36C90679912D3A4906663E0C7
:10765A0075F003A424EAF582E43467F58312D3FDB6
:10766A0090679D12D434906662E075F003A424EA10
:10767A00F582E43467F58312D3FD9067A012D434FF
:10768A007BFF7AC079B212D8AB80147BFF7AC079BB
:10769A00EF1208A380097BFF7AC1790812D8AB9050
:1076AA0054E8E030E53B7BFF7AC179219065D91235
:1076BA00D36C90679512D3A49065DD12D36C906752
:0476CA009912D3A49A
:1076CE009065E112D36C90679D12D3A49065E5127C
:1076DE00D36C9067A112D3A412D8AB80097BFF7A2A
:1076EE00C1795C12D8AB7BFF7AC17975904EBE1210
:1076FE00D36C90679512D3A4905F8712D36C90676A
:10770E009912D3A4904F4312D36C90679D12D3A4B9
:10771E0012D8AB9065F9E0A330E30B7BFF7AC17909
:10772E00B71208A380397BFF7AC179D7905D81E0CB
:10773E00FFA3E0906795CFF0A3EFF012D8AB906661
:10774E00A5E0FEA3E0FFC3943DEE940050117BFF35
:10775E007AC27904906795EEF0A3EFF012D8AB9051
:10776E005D7AE075F003A424DBF582E43467F583DB
:10777E0012D3FD90679512D434E4FE906812E05453
:10778E00807807CEC313CE13D8F99067F975F0033E
:10779E0012D3E1EE75F003A42583F58312D3FD9089
:1077AE00679812D4347BFF7AC2793512D8AB905DCC
:1077BE007AE014601914604A2402706E9065FAE043
:1077CE0030E5677BFF7AC2794E1208A3805C906524
:1077DE00FBE030E00B7BFF7AC2795A1208A38010CF
:1077EE009065FBE030E1097BFF7AC279631208A352
:1077FE009054E8E030E6337BFF7AC2796C1208A32E
:10780E0080287BFF7AC27978900005E0906795F02A
:10781E0090000CE0906796F090000AE0FFA3E090D5
:10782E006797CFF0A3EFF012D8AB9065FCE075F040
:10783E0003A42402F582E43468F58312D3FD906725
:10784E009512D4347BFF7AC2798B12D8AB7BFF7A38
:10785E00C2798F90659DE0FFA3E0906795CFF0A36E
:10786E00EFF0906083E0FFA3E0906797CFF0A3EF77
:10787E00F012D8AB7BFF7AC279BF9065ED12D36C54
:10788E0090679512D3A412D8ABE4FE906812E05420
:10789E00087803CEC313CE13D8F99067E475F003BE
:1078AE0012D3E1EE75F003A42583F58312D3FD9078
:1078BE00679512D4347BFF7AC279DA12D8AB905620
:1078CE00E5E075F003A424FFF582E43467F5831236
:1078DE00D3FD90679512D4347BFF7AC279F212D819
:0E78EE00AB7BFF7AC3791712D8AB12E72022CA
:1078FC009067DBEEF0A3EFF0E49067EFF0A3F0906D
:10790C00681B12D3B03F80000090681F12D3B000E8
:10791C000000009067DCE0FF1247231245387BFF24
:10792C007AC37935906795E53FF0A3E540F0A3E580
:10793C002BF0A3E528F0A3E529F0A3E52AF0A3E5B5
:10794C0027F012D8AB7BFF7AC3795B1208A3E490C3
:10795C0067F6F09067F3F07B017A6779F112091DF5
:10796C009067F6E0FF9067F3E04F642F6003027AB4
:10797C00219067FFE0FF9067FCE04F643A600302E0
:10798C007A219067F1E0FB75F00AA4FFA3E07C007C
:10799C002FFFEC35F0CF245C9067E0F0EF340590CE
:1079AC0067DFF0EB64396007E475F06412D19A90EC
:1079BC0067F4E024D075F00AA4FFA3E024D02F9044
:1079CC0067E8F09067F7E024D075F00AA4FFA3E015
:1079DC0024D02F9067E9F09067FAE024D075F00A74
:1079EC00A4FFA3E024D02F9067EAF09067FDE02479
:1079FC00D075F00AA4FFA3E024D02F9067EBF09091
:107A0C006800E024D075F00AA4FFA3E024D02F90E6
:107A1C0067ECF080209067DFE53FF0A3E540F09045
:107A2C0067E8E52BF0A3E528F0A3E529F0A3E52A08
:107A3C00F0A3E527F09067DFE0FEA3E0FF9067E896
:107A4C00E0FDA3E0FBA3E090683BF09067EBE090D7
:107A5C00683CF09067ECE090683DF0127D937BFF02
:107A6C007AC3798490655512D36C90679512D3A420
:107A7C0012D8AB7BFF7AC379A21208A37B017A6878
:107A8C0079199068BB12D4347BFF7AC379AE120992
:107A9C00D390682B12D3A4906819E07002A3E06015
:107AAC000C90682B12D36C90681B12D3A47B017AB8
:107ABC006879199068BB12D4347BFF7AC379B912F8
:107ACC0009D390682F12D3A4906819E07002A3E038
:107ADC00600C90682F12D36C90681F12D3A490681E
:107AEC001B12D36C7B5E7A0B7936783A12CC2190D0
:107AFC00681B12D3A490681F12D36C7B417A2E7929
:107B0C0042783712CC2190681F12D3A490681F12B0
:107B1C00D36C90681B12D38812CB3090682312D38D
:107B2C00A47BFF7AC379EF90679512D4347AC3792A
:107B3C00F490679812D4347AC379F990679B12D475
:107B4C00347AC379FC90679E12D4347AC379FF904F
:0C7B5C0067A112D4347AC479059067A4A4
:107B680012D4347AC379C412D8ABE49067EEF0909B
:107B780067EEE0C394164003027D5830980B12E775
:107B880020E49067F0F0027D589067DCE0FF124C2B
:107B98006790655512D36C12CE7FAC06AD0790671F
:107BA800DDECF0A3EDF0EC12CE46A804A905AA0678
:107BB800AB0790655512D36C12CB2C90682712D363
:107BC800A47B017A6779E390683E12D4347A670916
:107BD80090684112D4347A6779E19067DDE0FCA3BC
:107BE800E0FDA3E0FEA3E0FF127EF27B017A677955
:107BF800E690683E12D4347A670990684112D4340A
:107C08007A6779E590682712D36C127FEE7F007E41
:107C1800007D807CBF90678212D38812CDC360023A
:107C28005003027CE07BFF7AC4790D9067E1E0FFA6
:107C3800A3E0906795CFF0A3EFF09067E3E090673B
:107C480097F09067E4E0906798F09067E5E09067B8
:107C580099F09067E6E090679AF09067E7E09067A0
:107C68009BF090676012D36C90679C12D3A49067C6
:107C78008212D36C9067A012D3A4904E4212D36C98
:107C88009067A412D3A4905F6712D36C9067A81270
:107C9800D3A412D8AB90683312D36C90678212D3F6
:107CA8008812CDC3600840069067EF7401F09067B2
:107CB800EEE004F090655512D36C90682312D388D7
:107CC80012CB3090655512D3A490678212D36C9072
:107CD800683312D3A4027B7790683312D36C906711
:107CE8008212D38812CDC350159067EFE0B4010E0D
:107CF8007BFF7AC4794C1208A3E49067EFF07F14F5
:107D08007E0B7D367C3A90682312D38812CDC360EF
:107D180019401790655512D36C90682312D38812B6
:107D2800CB3090655512D3A4801790655512D36C4B
:107D38007B147A0B7936783A12CB3090655512D38A
:107D4800A490678212D36C90683312D3A4027B7715
:107D58009067F0E06003027B2D7BFF7AC4795912AB
:107D680008A312E7209067EDEFF04420FF647160EC
:107D780019EF64736003027B2D9067F004F07BFFBA
:0B7D88007AB279801208A3027B2D2242
:107D9300906837EEF0A3EFF0906837E0FEA3E0FFC2
:107DA3001246C790001CEEF0A3EFF090683BE0FC96
:107DB300E412CE4B7B007A0079C0784112CD2A9031
:107DC300684212D3A490683CE0FCE412CE4B7B00E3
:107DD3007A0079B4784412CD2A90684612D3A490DD
:107DE300683DE0FCE412CE4B7B007AC079A878476B
:107DF30012CD2A90684A12D3A4904E6EE0FEA3E0FF
:107E0300FFC3906838E09FFF906837E09EFE90685C
:107E13003EF0A3EFF04E6075A3E4F0A304F0906886
:107E23003EE0FEA3E0FFA3E0FCA3E0FDD39FEC9EB6
:107E3300505BC3906838E09DFF906837E09CEF5437
:107E430003702490001CE0FCA3E0FDE412CE467B0B
:107E5300007A0079B7784312CB3012CE7F90001CA2
:107E6300EEF0A3EFF0800B90001C740175F06D121F
:107E7300D19AD3906841E09405906840E094005013
:107E83000C906840E475F00112D19A8091D3900070
:107E93001DE0948D90001CE0940140097BFF7AC49F
:107EA300797F1208A390001CE0FCA3E0FDE412CE4E
:107EB3004690655512D3A490655512D388C000C06F
:107EC30001C002C00390684612D36C90684212D37B
:107ED3008812CB3090684A12D38812CB30D003D0AB
:0F7EE30002D001D00012CB3090655512D3A422EB
:107EF200906837EEF0A3EFF0A3ECF0A3EDF0A3123D
:107F0200D4347F01904E6EE0FDA3E0906844CDF042
:107F1200A3EDF0E4906845E0540370047E01800212
:107F22007E00AF06906839E0FDA3E0906846CDF090
:107F3200A3EDF09068487401F0906848E0FEEF7598
:107F4200F00DA424AFF582E43465F583E5822EF5C5
:107F520082E43583F583E0F9FD906846E0FAA3E018
:107F6200FBD39DEA9400401EEED3940C5018E9FD19
:107F7200C3EB9D906847F0EA9400906846F09068E1
:107F820048E004F080B3906848E0FED3940C402EA1
:107F9200EED3940C409DEF600D90683974FE75F03D
:107FA2009212D19A800B90683974FE75F09312D1B7
:107FB2009A906844E475F00112D19A027F15906894
:107FC2003E12D3FDEE12D13E906847E0FF90684129
:107FD20012D3FDEF12D13E906844E0FEA3E0FF9081
:0C7FE200683B12D3FDEE8FF012D1C622D6
:107FEE0090683712D3A490683B12D4347F007E0081
:107FFE007DC07C4190683712D38812CC21906844A2
:10800E0012D3A490684412D36C12CE7F906848EFBE
:10801E00F090684412D36CC004C005C006C007902F
:10802E006848E0FCE412CE4BA804A905AA06AB07EB
:10803E00D007D006D005D00412CB2C90684412D3B2
:10804E00A47F007E007D707C4290684412D388121B
:10805E00CC2112CE7F906849EFF090684412D36C19
:10806E00C004C005C006C007906849E0FCE412CE0B
:10807E004B7B007A007970784212CD2AA804A905AC
:10808E00AA06AB07D007D006D005D00412CB2C9091
:10809E00684412D3A47F007E007D617C45906844C5
:1080AE0012D38812CC2112CE7F906848E0FE9068E1
:1080BE003B12D3FDEE12D13E906849E0FE90683E31
:1080CE0012D3FDEE12D13E90684112D3FDEF12D1C4
:0280DE003E2240
:1080E000E49067E1F0A3F01208287BFF7AC4799747
:1080F0001208A390676AE0FFA3E09067E3CFF0A3C4
:10810000EFF0C39067E4E0941F9067E3E0944E5073
:108110002A12E7209067E6EFF09067E3E0FCA3E027
:10812000241EF582EC3400F583EFF0641A600C90A5
:1081300067E3E475F00112D19A80C79067E3E0FE2F
:10814000A3E0FF90676AEEF0A3EFF0C3941EEE94F5
:108150004E40097BFF7AC479C31208A37BFF7AB231
:1081600079801208A31205C8E49067E3F0A3F0E455
:108170009067E5F09067E5E0FFC3944F504090674B
:10818000E3E475F00112D1B0FC741E25F0F582EC29
:108190003400F583E09067E6F0E0FE641A601FEEBD
:1081A000640D601AEE640A60159067E5E0FD04F066
:1081B00074372DF582E43468F583EEF080B690676D
:1081C000E6E0641A700302880F74372FF582E434F6
:1081D00068F583E4F0906837E0FF64206091EF6019
:1081E0008E7E007F14C006C0077F00C0079067E145
:1081F000E0FEA3E0FF7C007D1412D15074A12FF9A2
:1082000074603EFA7B01D005D007D00612D46F907F
:1082100067E1E0FEA3E0FF7C007D1412D15074A161
:108220002FF974603EA801FC7D017B017A687937E3
:108230007E007F0F12D558E49067E5F09067E5E087
:10824000C3944F50409067E3E475F00112D1B0FE43
:10825000741E25F0F582EE3400F583E09067E6F0B9
:10826000E0FF641A601FEF640D601AEF640A601586
:108270009067E5E0FE04F074E72EF582E43467F5DC
:1082800083EFF080B79067E7E06431600302816FAD
:108290009067E9E06441700302816F9067F9E02420
:1082A000D075F00AA4FFA3E0FD24D0FDE434FFCD97
:1082B0002FCD35F0FC9067E2E025E0FF9067E1E02C
:1082C00033FE74732FF582EE345EF583ECF0A3ED8C
:1082D000F0E49067E5F09067E5E0FFC3940C50216F
:1082E000E0FE24FBF582E43467F583E0FD74372E6D
:1082F000F582E43468F583EDF09067E5E004F08002
:10830000D574372FF582E43468F583E4F07B017A85
:1083100068793712DFD9C004C005C006C00790676E
:10832000E1E0FEA3E07802C333CE33CED8F9248A4D
:10833000F582EE345CF583D007D006D005D0041268
:10834000D3A4E49067E5F09067E5E0FFC3940A509A
:1083500021E0FE2408F582E43468F583E0FD7437FB
:108360002EF582E43468F583EDF09067E5E004F0E3
:1083700080D574372FF582E43468F583E4F07B010F
:108380007A68793712DFD9C004C005C006C00790EB
:1083900067E1E0FEA3E07802C333CE33CED8F92400
:1083A000A6F582EE345AF583D007D006D005D00466
:1083B00012D3A4E49067E5F09067E5E0C3944F50D2
:1083C000409067E3E475F00112D1B0FE741E25F011
:1083D000F582EE3400F583E09067E6F0E0FF641A82
:1083E000601FEF640D601AEF640A60159067E5E0A6
:1083F000FE04F074E72EF582E43467F583EFF08035
:10840000B79067E7E06432600302816FE49067E54C
:10841000F09067E5E0FFC394085021E0FE24EFF5FB
:1084200082E43467F583E0FD74372EF582E4346826
:10843000F583EDF09067E5E004F080D574372FF513
:1084400082E43468F583E4F07B017A68793712DFDF
:10845000D9C004C005C006C0079067E1E0FEA3E0F4
:108460007802C333CE33CED8F924EDF582EE3454FE
:10847000F583D007D006D005D00412D3A4E49067CA
:10848000E5F09067E5E0FFC394085021E0FE24F892
:10849000F582E43467F583E0FD74372EF582E43429
:1084A00068F583EDF09067E5E004F080D574372F30
:0F84B000F582E43468F583E4F07B017A6879376C
:1084BF0012DFD9C004C005C006C0079067E1E0FE17
:1084CF00A3E07802C333CE33CED8F92496F582EEEB
:1084DF00345BF583D007D006D005D00412D3A49017
:1084EF0067E57402F09067E5E0FFC394075021E061
:1084FF00FE24FFF582E43467F583E0FD74372EF533
:10850F0082E43468F583EDF09067E5E004F080D500
:10851F0074372FF582E43468F583E4F0906837748C
:10852F0030F0A3742EF07B017A68793712DFD9C04F
:10853F0004C005C006C0079067E1E0FEA3E0780223
:10854F00C333CE33CED8F92437F582EE3450F583CA
:10855F00D007D006D005D00412D3A4E49067E5F07D
:10856F009067E5E0FFC394085021E0FE2409F582EF
:10857F00E43468F583E0FD74372EF582E43468F552
:10858F0083EDF09067E5E004F080D574372FF58226
:10859F00E43468F583E4F07B017A68793712DFD928
:1085AF00C004C005C006C0079067E1E0FEA3E078F5
:1085BF0002C333CE33CED8F92483F582EE345DF582
:1085CF0083D007D006D005D00412D3A4E49067E57A
:1085DF00F09067E5E0FFC394085021E0FE2412F508
:1085EF0082E43468F583E0FD74372EF582E4346855
:1085FF00F583EDF09067E5E004F080D574372FF543
:10860F0082E43468F583E4F07B017A68793712DF0E
:10861F00D9C004C005C006C0079067E1E0FEA3E023
:10862F007802C333CE33CED8F924C6F582EE345850
:10863F00F583D007D006D005D00412D3A4E49067F9
:10864F00E5F09067E5E0FFC3940B5021E0FE241B9B
:10865F00F582E43468F583E0FD74372EF582E43457
:10866F0068F583EDF09067E5E004F080D574372F5F
:10867F00F582E43468F583E4F07B017A6879371288
:10868F00DFD9C004C005C006C0079067E1E0FEA3B4
:10869F00E07802C333CE33CED8F924B6F582EE3468
:1086AF0059F583D007D006D005D00412D3A4E49097
:1086BF0067E5F09067E5E0FFC394055021E0FE24E5
:1086CF0026F582E43468F583E0FD74372EF582E4F5
:1086DF003468F583EDF09067E5E004F080D57437EA
:1086EF002FF582E43468F583E4F07B017A687937FB
:1086FF0012E83FC004C005C006C0079067E1E0FE66
:10870F00A3E07802C333CE33CED8F9FBAA0624F503
:10871F00F582EA3455F583D007D006D005D0041280
:10872F00D3A474472BF582EA344FF58312D3B000EC
:10873F000000009067E2E0C4F8540FC868FB906730
:10874F00E1E0C454F048FA74332BF582EA3451F562
:10875F008312D3B000000000742F2BF582EA34513E
:10876F00F58312D3B0000000009067E2E0C4F85424
:10877F000FC868FB9067E1E0C454F048FA742B2BE4
:10878F00F582EA3451F58312D3B00000000074274C
:10879F002BF582EA3451F58312D3B000000000901C
:1087AF0067E1E0FEA3E0FF2401906796F0E43E90BE
:1087BF006795F07C007D1412D15074A12FF974606D
:1087CF003EFA7B0190679712D4347BFF7AC479DA33
:1087DF0012D8AB9067E1E475F00112D19A9067E17E
:1087EF00E0FEA3E0FF904EA4EEF0A3EFF0C3943CA5
:1087FF00EE9400500B9067E6E0641A600302816FFD
:04880F00128C2E2277
:108813007BFF7AB279801208A3E49067E2F0A3F0B9
:108823009067E1F09067E1E0FFC3943C50157468F2
:108833002FF582E43466F58374FFF09067E1E0047A
:10884300F080E1E49067E1F01288D4C3EF64809490
:10885300805011D39067E3E094009067E2E09400C6
:10886300405780619067E1E02468F582E43466F55F
:1088730083EFF03395E0FE7C007D1412D15074A198
:108883002FF974603EFA7B0190679512D434906798
:10889300E3E004906798F07BFF7AC479E912D8ABE0
:1088A3009067E2E475F00112D19AC39067E3E09414
:1088B3003C9067E2E09400500C9067E1E004F0E044
:1088C300C3943C40839067E3E0906770F0128B9F02
:0188D3002282
:1088D400E49067E6F0A3F07BFF7AB279801208A3F4
:1088E400E49067E4F0A3F09067E4E0FEA3E0FFC344
:1088F400943CEE940040030289BD904EA4E0FCA396
:10890400E0FDC3EF9DEE9C40030289BDEF4E601273
:10891400E49067E5E0540370097BFF7AB279801232
:1089240008A39067E4E0FCA3E0FD25E0FFEC33FE40
:1089340074BB2FF582EE3466F583A3E030E42FEDAB
:108944002401906796F0E43C906795F07E007F14D4
:1089540012D15074A12FF974603EFA7B019067978D
:1089640012D4347BFF7AC5790E12D8AB8034906769
:10897400E4E0FEA3E0FF2401906796F0E43E9067F4
:1089840095F07C007D1412D15074A12FF974603ECF
:10899400FA7B0190679712D4347BFF7AC5791A1257
:1089A400D8AB9067E6E475F00112D19A9067E4E4DD
:1089B40075F00112D19A0288EB7B017A6779E8900D
:1089C400684A12D4347BFF7AC5792612099CAD0714
:1089D400AC069067E6E0FEA3E0FFD3ED9FEC9E407B
:1089E400057EFF7FFF22D3ED9400EC6480948040E9
:1089F40029D3ED943CEC64809480501EED25E0FF77
:108A0400EC33FE74BA2FF582EE3466F583E044103D
:0F8A1400F0ED24FFFFEC34FFFE227EFF7FFF22F8
:108A23007BFF7AB279801208A3E4906843F0A3F045
:108A3300906843E0FEA3E0FFC3943CEE648094801F
:108A43004003028B0BE02468F582E43466F583E08F
:108A5300C3648094805003028AFE906770E0FDD364
:108A6300EF9D7480F86E984003028B0BEF4E601CF1
:108A7300906843E0FEA3E0FF7C007D0412D164ED27
:108A83004C70097BFF7AB279801208A390665BE091
:108A9300FF3395E0FE906843E0FCA3E0FDEFB505EE
:108AA3000CEEB50408906842742AF0800690684280
:108AB3007420F0ED2401906796F0E43C906795F004
:108AC300906842E0906797F0906844E02468F582EC
:108AD300E43466F583E0FF3395E0FE7C007D1412F9
:108AE300D15074A12FF974603EFA7B0190679812FC
:108AF300D4347BFF7AC5793112D8AB906843E475DF
:108B0300F00112D19A028A337BFF7AB2798012087C
:108B1300A3906668E0FF3395E0FE7C007D1412D1DC
:108B23005074A12FF974603EFA7B01C003C002C0E8
:108B3300017BFF7AC5793E9069E512D4349069E8E8
:108B4300E4F0A37407F0D001D002D00312E7A7EF3B
:108B5300700C7BFF7AC579461208A37FFF227B0145
:108B63007A68794590684A12D4347BFF7AC57926AE
:108B730012099CEF24FFFFEE34FFFE906770E0FDC7
:108B8300C3EF9D7480F86E9850D4C3EE64809480D4
:0C8B9300500474FFFEFF90665BEFF022C0
:108B9F00E4FF9069E2F09069E2E0FEC3943C502A52
:108BAF0074682EF582E43466F583E0FEC364809426
:108BBF0080400FAD070F74682DF582E43466F5839E
:108BCF00EEF09069E2E004F080CC9069E2EFF09073
:108BDF0069E2E0FFC3943C504574682FF582E4349A
:108BEF0066F58374FFF074682FF582E43466F583BD
:108BFF00E0FF3395E0FE7C007D1412D15074A12F5D
:108C0F00F974603EA801FC7D017BFF7AC579757E02
:0F8C1F00007F0212D5589069E2E004F080B12284
:108C2E00E4906888F0120828E490688FF0A3F09022
:108C3E006890E02468F582E43466F58374FFF09062
:108C4E00688FE475F00112D19A90688FE07004A3DA
:108C5E00E0643C70DA7BFF7AC579781208A39067DE
:108C6E006AE0FFA3E090688FCFF0A3EFF0C39068A7
:108C7E0090E0941F90688FE0944E502A12E7209057
:108C8E006891EFF090688FE0FCA3E0241EF582EC73
:108C9E003400F583EFF0641A600C90688FE475F081
:108CAE000112D19A80C7C3906890E0941F90688F8C
:108CBE00E0944E40097BFF7AC479C31208A37BFF70
:108CCE007AB279801208A390676AE0FEA3E0241EB0
:108CDE00F582EE3400F583E0641A7048906888F0EF
:108CEE00906888E0FF904EA4E0FCA3E0FDC3EF9DEA
:108CFE00E49C502C906888E02468F582E43466F594
:108D0E0083EFF0EF25E024BCF582E43466F583E0D2
:108D1E004410F0906888E004F0E0906770F080C036
:108D2E00128B9F2290676AE0FFA3E090688FCFF0CE
:108D3E00A3EFF0E4906887F0906887E0C3945050FA
:108D4E003B90688FE475F00112D1B0FE741E25F0D1
:108D5E00F582EE3400F583E0906891F0E0FF640A4E
:108D6E00601AEF641A6015906887E0FE04F0749242
:108D7E002EF582E43468F583EFF080BC906891E0C4
:108D8E00641A7003029396906887E0FF04F0749261
:108D9E002FF582E43468F583E4F0906892E0FF608A
:108DAE0092EF643B608DEF642060887BFF7AC5791B
:108DBE00A79067C512D4347B017A6879F69067C89C
:108DCE0012D4347A69790A9067CB12D4347A6979DD
:108DDE00469067CE12D4347A6979BE9067D112D498
:108DEE00347A6979C69067D412D4347A6979CE9080
:108DFE0067D712D4347A6979D69067DA12D4347A76
:108E0E006979DC9067DD12D4347A68799212DD3993
:108E1E007B017A6879F612E80E906889EFF0E4A388
:108E2E00F090688AE0FFFD904EA4E0FAA3E0FBC349
:108E3E00ED9BE49A4003028D41EF75F014A424A13A
:108E4E00F9746035F0FA7B01C002C0017A6879F6D8
:108E5E009069E512D434906889E0FF9069E8E4F0F7
:108E6E00A3EFF0D001D00212E7A7EF600302938DBB
:108E7E00906888E0C3943C400302938DE490688C24
:108E8E00F07B017A69790A12E80E90688BEFF07B1D
:108E9E00017A69790A7D2F12E823EA497003028F5D
:108EAE0089E4906887F090688BE0FF906887E0C354
:108EBE009F5043E0FF240AF582E43469F583E0FE17
:108ECE0074322FF582E43469F583EEF090688CE00D
:108EDE0004F0740A2FF582E43469F583E0B42F0EA2
:108EEE0074322FF582E43469F583E4F080089068DB
:018EFE0087EC
:108EFF00E004F080B07B017A69793212DFD9906893
:108F0F008AE025E025E02447F582E4344FF583120B
:108F1F00D3A4E4906887F090688CE0FF90688BE0B2
:108F2F00C39FFE906887E0FDC39E5023E0FEEF2EA7
:108F3F00240AF582E43469F583E0FF74322EF5825A
:108F4F00E43469F583EFF0906887E004F080C8742B
:108F5F00322DF582E43469F583E4F07B017A697987
:108F6F003212DFD990688AE025E025E024E6F58209
:108F7F00E43456F58312D3A480337B017A69790ADE
:108F8F0012DFD990688AE0FB25E025E02447F582BF
:108F9F00E4344FF58312D3A4EB25E025E024E6F566
:108FAF0082E43456F58312D3B000000000E49068D9
:108FBF008CF07B017A69794612E80E90688BEFF09E
:108FCF00E490688DF090688DE0C3940440030290A4
:108FDF00B8E4906887F090688BE0FF906887E0FEB8
:108FEF00C39F503D90688CE0FFEE2F2446F582E43E
:108FFF003469F583E0FF74AA2EF582E43469F583B2
:10900F00EFF074AA2EF582E43469F583E0FF642C47
:10901F006003EF7004E4F08008906887E004F0804C
:10902F00B57B017A6979AA12DFD990688AE075F069
:10903F001090512712D3E1C083C08290688DE0FB5E
:10904F00D082D08375F00412D3E112D3A490688C30
:10905F00E0FF906887E02F2446F582E43469F583BA
:10906F00E07033EB0490688EF090688EE0FFC3944D
:10907F0004503690688AE075F01090512712D3E1B2
:10908F0075F004EF12D3E112D3B000000000906826
:10909F008EE004F080D3906887E004FF90688CE046
:1090AF002FF0A3E004F0028FD4E490688CF07B01E2
:1090BF007A6979467D2F12E823EA49700302916796
:1090CF00E4906887F090688BE0FF906887E0FEC3BC
:1090DF009F501D90688CE004F074462EF582E434A6
:1090EF0069F583E0642F6008906887E004F080D50D
:1090FF00E4906887F090688CE0FF90688BE0C39FE6
:10910F00FE906887E0FDC39E5023E0FEEF2E2446BD
:10911F00F582E43469F583E0FF74AA2EF582E43416
:10912F0069F583EFF0906887E004F080C874AA2D8A
:10913F00F582E43469F583E4F07B017A6979AA1248
:10914F00DFD990688AE025E025E024D6F582E43463
:10915F0057F58312D3A4801890688AE025E025E0A4
:10916F0024D6F582E43457F58312D3B00000000003
:10917F009069BEE04420249D603024FD603E24F1C0
:10918F0060162409704890688AE02461F582E434FF
:10919F0065F5837401F0804590688AE02461F5825B
:1091AF00E43465F5837402F0803390688AE02461BB
:1091BF00F582E43465F5837403F0802190688AE0CA
:1091CF002461F582E43465F5837404F0800F9068B0
:1091DF008AE02461F582E43465F583E4F09069C692
:1091EF00E04420249D603024FD603E24F16016246D
:1091FF0009704890688AE0241FF582E43466F5838D
:10920F007401F0804590688AE0241FF582E434668B
:10921F00F5837402F0803390688AE0241FF582E4AE
:10922F003466F5837403F0802190688AE0241FF57B
:10923F0082E43466F5837404F0800F90688AE0242A
:01924F001FFF
:10925000F582E43466F583E4F09069CEE04420FFC3
:10926000BF631590688AE025E024BCF582E434668B
:10927000F583E054FEF08016BF6D1390688AE025F8
:10928000E024BCF582E43466F583E04401F09069A3
:10929000D6E04420FFBF6D1590688AE025E024BC2D
:1092A000F582E43466F583E04402F0801390688A26
:1092B000E025E024BCF582E43466F583E054FDF05B
:1092C0009069DCE04420FFBF691DA3E04420FEBE9E
:1092D000721590688AE025E024BCF582E43466F5D6
:1092E00083E04404F0801390688AE025E024BCF514
:1092F00082E43466F583E054FBF0BF6B1F9069DDB8
:10930000E04420FFBF721590688AE025E024BCF598
:1093100082E43466F583E04408F0801390688AE0C4
:1093200025E024BCF582E43466F583E054F7F09040
:10933000688AE0FF906888E02468F582E43466F586
:1093400083EFF0EF25E024BCF582E43466F583E09A
:109350004410F0EF75F014A424A1F9746035F0FA0C
:109360007B0190679512D434906888E004906798E8
:10937000F07BFF7AC579BF12D8ABE49069DCF0903E
:109380006888E004F0E0906770F0028D4190688A90
:0A939000E004F0028E2F128B9F22E2
:10939A00E490681AF0A3F0A3F0A3F0A3F0A3F012EC
:1093AA0008287BFF7AC579EF1208A390676AE0FF65
:1093BA00A3E0906818CFF0A3EFF0C3906819E09487
:1093CA001F906818E0944E502A12E720906821EF07
:1093DA00F0906818E0FCA3E0241EF582EC3400F556
:1093EA0083EFF0641A600C906818E475F00112D1EA
:1093FA009A80C790676AE0FFA3E0906818CFF0A34D
:10940A00EFF0E4906820F0906820E0FFC3943C50AD
:10941A003E906818E475F00112D1B0FC741E25F074
:10942A00F582EC3400F583E0906821F0E0FE641ADE
:10943A007003029C2CEE640A6015906820E0FD041B
:10944A00F074222DF582E43468F583EEF080B87466
:10945A00222FF582E43468F583E4F0906822E0B4C0
:10946A0031A07BFF7AC679239067C512D4347B0179
:10947A007A4E797D9067C812D4347A5579DD90672F
:10948A00CB12D4347A5579E19067CE12D4347A5516
:10949A0079E99067D112D4347A68799A9067D412AC
:1094AA00D4347A68791C9067D712D4347A687922CE
:1094BA0012DD3990689BE04420FFBF72099065FA7B
:1094CA00E04410F080079065FAE054EFF0BF610CB9
:1094DA009065F9E04410F0A3E0F080079065F9E0A8
:1094EA0054EFF090689AE04420FFBF73099054E863
:1094FA00E054F7F0800ABF6E079054E8E04408F0A1
:10950A007F007E007D007C009055E112D38812CD49
:10951A00C350197F007E007D807CBF9055E112D335
:10952A008812CC219055E512D3A480179055E112E8
:10953A00D3887F007E007DB47C4312CB2C9055E506
:10954A0012D3A490681CE0FEA3E0FFBE010ABF2C60
:10955A0007E49056E5F08046BE040BBFB00890566B
:10956A00E57401F08038BE090BBF60089056E574B7
:10957A0002F0802ABE120BBFC0089056E57403F0B1
:10958A00801CBE250BBF80089056E57404F0800E3F
:10959A00E4B5070AEEB44B069056E57405F0E4907C
:1095AA006820F0906820E0FFC3943C503E90681811
:1095BA00E475F00112D1B0FC741E25F0F582EC348A
:1095CA0000F583E0906821F0E0FE641A7003029CC3
:1095DA002CEE640A6015906820E0FD04F074222DD8
:1095EA00F582E43468F583EEF080B874222FF582B0
:1095FA00E43468F583E4F0906822E0B432A07BFF9B
:10960A007AC679399067C512D4347B017A6679B102
:10961A009067C812D4347A0079159067CB12D43483
:10962A007A6679019067CE12D4347A67796890673E
:10963A00D112D4347A6879729067D412D4347A68A1
:10964A00792212DD39906872E04420FFBF660C90DF
:10965A0065F9E04440F0A3E0F080079065F9E05432
:10966A00BFF012052BE4906820F0906820E0FFC359
:10967A00943C503E906818E475F00112D1B0FC7425
:0E968A001E25F0F582EC3400F583E090682197
:10969800F0E0FE641A7003029C2CEE640A601590D8
:1096A8006820E0FD04F074222DF582E43468F58327
:1096B800EEF080B874222FF582E43468F583E4F084
:1096C800906822E0B433A07BFF7AC6794C9067C5D6
:1096D80012D4347B017A6679139067C812D4347A2D
:1096E8006679179067CB12D4347A66790B9067CE77
:1096F80012D4347A66790F9067D112D4347A6879A3
:109708002212DD39E4906820F0906820E0FFC394CD
:109718003C503E906818E475F00112D1B0FC741EFC
:1097280025F0F582EC3400F583E0906821F0E0FE46
:10973800641A7003029C2CEE640A6015906820E09D
:10974800FD04F074222DF582E43468F583EEF08090
:10975800B874222FF582E43468F583E4F090682227
:10976800E0B434A07BFF7AC6795C9067C512D43424
:109778007B017A6879729067C812D4347A687986DE
:109788009067CB12D4347A0079059067CE12D4341E
:109798007A00790C9067D112D4347A68791A906774
:1097A800D412D4347A00790A9067D712D4347A68FC
:1097B800792212DD39906872E044202497604024B1
:1097C800F0601A240E7058E4905D7AF0906879E0A1
:1097D8006437704B9065FAE04420F08042905D7ADF
:1097E8007401F0906877E04420FFBF77099054E84F
:1097F800E054BFF080299054E8E04440F080209085
:109808005D7A7402F0906876E04420FFBF73099097
:1098180065FBE04410F080079065FBE054EFF090A2
:109828006878E024C8601B0470309065FBE0440150
:10983800F054FDF0904E95742EF0904E78741EF012
:10984800802C9065FBE054FEF04402F0904E957435
:1098580021F0904E787411F080149065FBE054FE6E
:10986800F054FDF0904E957401F0904E78F09068A9
:1098780086E04420FFBF66099054E8E04480F08009
:109888000ABF61079054E8E0547FF090681AE0FE40
:10989800A3E0FFBE040ABFB007E49065FCF080387F
:1098A800BE090BBF60089065FC7401F0802ABE12E7
:1098B8000BBFC0089065FC7402F0801CBE250BBF6E
:1098C80080089065FC7403F0800EE4B5070AEEB4D6
:1098D8004B069065FC7404F0C2CA9065FCE025E074
:1098E80024A7F582E43466F583E0FCA3E0FDECF5FB
:1098F800CBF5CDEDF5CAF5CCD2CAE4906820F0904E
:109908006820E0FFC3943C503E906818E475F0016D
:1099180012D1B0FC741E25F0F582EC3400F583E01A
:10992800906821F0E0FE641A7003029C2CEE640A31
:109938006015906820E0FD04F074222DF582E4346F
:1099480068F583EEF080B874222FF582E43468F568
:1099580083E4F0906822E0B435A07BFF7AC679747E
:109968009067C512D4347B017A6879729067C812FF
:10997800D4347A5579F19067CB12D4347A4F793F41
:109988009067CE12D4347A4E79BE9067D112D4340F
:109998007A5F79879067D412D4347A4F7943906785
:1099A800D712D4347A68792212DD39906872E0B41B
:1099B80031099054E8E04410F080079054E8E054EE
:1099C800EFF0906873E0906886F0E4A3F07B017A8A
:1099D80068798612E94DEF04900017F0906874E0FA
:1099E800906886F0E4A3F07B017A68798612E94DE5
:1099F800EF2402900017F0E4906820F0906820E0CF
:109A0800FFC3943C503E906818E475F00112D1B041
:109A1800FC741E25F0F582EC3400F583E090682193
:109A2800F0E0FE641A7003029C2CEE640A60159044
:109A38006820E0FD04F074222DF582E43468F58393
:109A4800EEF080B874222FF582E43468F583E4F0F0
:109A5800906822E0B436A07BFF7AC6798A9067C501
:109A680012D4347B017A68799A9067C812D4347A10
:109A78006579CD9067CB12D4347A6579D19067CE69
:109A880012D4347A6879729067D112D4347A6879AA
:109A9800869067D412D4347A5D79819067D712D4CE
:109AA800347A6679A59067DA12D4347A6879221202
:109AB800DD3990689AE0B4310C9065F9E04402F021
:109AC800A3E0F080079065F9E054FDF090689BE012
:109AD800B431099065F9E054F7F0800A9065F9E02F
:109AE8004408F0A3E0F0906872E04420249D601CD4
:109AF80024FD602024F1600C2409702090666274B3
:109B080001F0801D9066627402F0801590666274A0
:109B180003F0800D9066627404F08005E49066623C
:109B2800F0906886E04420249D601C24FD60202479
:109B3800F1600C240970209066637401F0801D9018
:109B480066637402F080159066637403F0800D906C
:109B580066637404F08005E4906663F0E49068201E
:109B6800F0906820E0FFC3943C503E906818E4757C
:109B7800F00112D1B0FC741E25F0F582EC3400F52A
:109B880083E0906821F0E0FE641A7003029C2CEEDA
:109B9800640A6015906820E0FD04F074222DF582B7
:109BA800E43468F583EEF080B874222FF582E4344B
:109BB80068F583E4F0906822E0B437A07BFF7AC6AA
:109BC80079A39067C512D4347B017A68797290675B
:109BD800C812D4347A6579D99067CB12D4347A65AF
:109BE80079DD9067CE12D4347A6579E19067D11225
:109BF800D4347A6579E59067D412D4347A687922B6
:109C080012DD39906872E0B431099054E8E04420DC
:109C1800F080079054E8E054DFF07BFF7AC679B60D
:0D9C28001208A3227BFF7AC679D81208A388
:019C3500220C
:109C36009054E7E04410FEA3E0FF9054E7EEF0A353
:109C4600EFF020E103029CD690665BE0FF3395E0DF
:109C5600FE74682FF582EE3466F583E0FF3395E0F7
:109C6600FEEF7802C333CE33CED8F924E6F582EE82
:109C76003456F58312D36C12CE7F7BA07A86790197
:109C8600780012D20090688712D3A490665BE0FF3A
:109C96003395E0FE74682FF582EE3466F583E0FFB7
:109CA6003395E0FEEF7802C333CE33CED8F924D60F
:109CB600F582EE3457F58312D36C12CE7F7BA07AF1
:109CC600867901780012D20090688B12D3A4801492
:109CD60090688B12D3B00000000090688712D3B052
:109CE600000000007BFF7AC679FC1208A37BFF7A8E
:109CF600C779131208A37F801205017BFF7AC77903
:109D0600521208C17FC01205017BFF7AC77964121F
:109D160008C17BFF7AC779761208A37B017A677937
:109D2600FB12091D7B017A6779FB12E80E9067DC4E
:109D3600EFF07BFF7AC779839067C512D4347B0135
:109D46007A68794B9067C812D4347A6879699067D3
:109D5600CB12D4347A6779FB12DD399067FBE0FFCA
:109D6600442012D449A1F63FA04A619D8C669F0209
:109D76006D9D8471A18F73A109740000A212905485
:109D8600E7E054EFF0229067FCE04420647560033E
:109D9600029E3A9067DBF09067DBE0FFC3940950C0
:109DA60021E0FE24FDF582E43467F583E0FD74DDF1
:109DB6002EF582E43467F583EDF09067DBE004F07E
:109DC60080D574DD2FF582E43467F583E4F07B01FA
:109DD6007A6779DD12E83F90688B12D38812D1E555
:109DE6009066B712D3A49066B712D36C7B0A7A003A
:109DF6007900780012D2009066B712D3A490665B01
:109E0600E0FF3395E0FE74682FF582EE3466F58345
:109E1600E0FF1240017FC01205017BFF7AC77989F6
:109E26001208C17FC31205017B017A6779DD12082A
:109E3600C1029D189067FCE0442064646003029EA2
:109E4600E89067DBF09067DBE0FFC394095021E000
:109E5600FE24FDF582E43467F583E0FD74DD2EF51E
:109E660082E43467F583EDF09067DBE004F080D59B
:109E760074DD2FF582E43467F583E4F07B017A67BD
:109E860079DD12E83F90688712D38812D1E5906594
:109E9600F112D3A49065F112D36C7B0A7A00790093
:109EA600780012D2009065F112D3A490665BE0FFB1
:109EB6003395E0FE74682FF582EE3466F583E0FF95
:089EC600123D927FC01205015C
:109ECE007BFF7AC7799B1208C17FC31205017B0104
:109EDE007A6779DD1208C1029D187BFF7AC779ADCA
:109EEE001208A37FC01205017BFF7AC779D512082D
:109EFE00C1029D189067FCE0442064756003029FC8
:109F0E0099A3E04420249D601C24FD602024F16070
:109F1E000C240970209066607401F08037906660A2
:109F2E007402F0802F9066607403F0802790666054
:109F3E007404F0801FE4906660F07FC01205017B10
:109F4E00FF7AC779E61208C17BFF7AC779F7120844
:109F5E00A3029D187FC01205017BFF7AC779641298
:109F6E0008C17FC01205017B017A6779FB1208C117
:109F7E0090665BE0FF3395E0FE74682FF582EE3459
:109F8E0066F583E0FF1242A1029D189067FCE04443
:109F9E00206464600302A030A3E04420249D601C72
:109FAE0024FD602024F1600C2409702090666174F9
:109FBE0001F080379066617402F0802F90666174B4
:109FCE0003F080279066617404F0801FE490666150
:109FDE00F07FC01205017BFF7AC879181208C17B89
:109FEE00FF7AC879291208A3029D187FC0120501B5
:109FFE007BFF7AC779641208C17FC01205017B010D
:10A00E007A6779FB1208C190665BE0FF3395E0FE3C
:10A01E0074682FF582EE3466F583E0FF1242A102DA
:10A02E009D187BFF7AC8794A1208A37FC0120501DA
:10A03E007BFF7AC879711208C1029D189067DCE027
:10A04E00C3940A501A7BFF7AC879821208A37FC084
:10A05E001205017BFF7AC879AA1208C1029D18E485
:10A06E009067DBF09067DBE0FFC394035021E0FEC6
:10A07E00244DF582E43468F583E0FD74DD2EF5821F
:10A08E00E43467F583EDF09067DBE004F080D5747F
:10A09E00DD2FF582E43467F583E4F07B017A67798E
:10A0AE00DD12DFD9905EEF12D3A4E49067DBF0905F
:10A0BE0067DBE0FFC394025021E0FE246BF582E4DF
:10A0CE003468F583E0FD74DD2EF582E43467F583A4
:10A0DE00EDF09067DBE004F080D574DD2FF582E4BF
:10A0EE003467F583E4F07B017A6779DD12DFD9906E
:10A0FE005C8612D3A412620C029D18E49067DBF00A
:10A10E009067DCE0FF9067DBE0FEC39F502074FC9D
:10A11E002EF582E43467F583E0FF74DD2EF582E4DC
:10A12E003467F583EFF09067DBE004F080D274DDE6
:10A13E002EF582E43467F583E4F07B017A6779DDEE
:10A14E0012E94DEF1490665BF0D36480948E501834
:10A15E00E0FF3395E0FE74682FF582EE3466F583EA
:10A16E00E0C364809480500C7BFF7AC879BC1208DF
:10A17E00A3029D189054E8E04404F0122B32029D85
:05A18E0018E49067DBFE
:10A19300F09067DCE0FF9067DBE0FEC39F50207424
:10A1A300FC2EF582E43467F583E0FF74DD2EF5823F
:10A1B300E43467F583EFF09067DBE004F080D2745A
:10A1C300DD2EF582E43467F583E4F07B017A677969
:10A1D300DD1208DF7FC01205017BFF7AC7796412A5
:10A1E30008C17FC01205017B017A6779DD1208C1BE
:10A1F300029D189067FCE04420FFBF610612648053
:10A20300029D187BFF7AC879CE1208A3029D187BA2
:10A21300FF7AC9790D1208A37FC01205017BFF7A6B
:0AA22300C979201208C1029D18221B
:10CAAE00ED7E09D3C2CF30CFFDD3C297C2CF1330A4
:10CABE00CFFD9297C2CFDEF630CFFDC2CF30CFFD85
:10CACE00EF702222EF7E09D3C2CF30CFFDD3C295B5
:10CADE00C2CF1330CFFD9295C2CFDEF630CFFDC25E
:10CAEE00CF30CFFD227EFA000000000000000000D3
:10CAFE000000000000000000000000DEEADFE62279
:10CB0E007EFA00000000000000000000000000009F
:0BCB1E00000000000000DEEADFE6225D
:10CB290002CEEBE86480F8E933E83360110460F081
:10CB3900ED33EC337009E8FCE9FDEAFEEBFF220472
:10CB490060DED3EB9FEA9EE99DE8C2E78CF0C2F76D
:10CB590095F0400CE8CCF8E9CDF9EACEFAEBCFFB39
:10CB690012CEB685D0F05804700320D5B3E804700E
:10CB7900075002B2D502CEF592D5EC0460F7E4CCA9
:10CB8900C0E0C398F8603B94186008400DD0E0FB02
:10CB990002CECDE4FBFAC9FC8028E830E406E4C9FA
:10CBA900FBE4CAFCE830E305E4C9CACBFCE8540756
:10CBB9006010F8C3E913F9EA13FAEB13FBEC13FC61
:10CBC900D8F130F52FC3E49CFCEF9BFFEE9AFEED04
:10CBD90099FDD0E0FBEF4E4D4C701222DB0302CEE3
:10CBE900F2EC2CFCEF33FFEE33FEED33FDED30E7D5
:10CBF900EB02CECDEF2BFFEE3AFEED39FDD0E0FB97
:10CC090050130BBB000302CEF5ED13FDEE13FEEF3F
:08CC190013FFEC13FC02CECD69
:10CC2100EC4D6011E8497017ED33EC3304600DE40D
:10CC3100FCFFFEFD22E933E8330470F802CEEB126B
:10CC4100CEB658046009E4CC24815006285009026C
:10CC5100CEF528400302CEF2C0E0EB4A7044B98021
:10CC610006D0E0FB02CEE1EF4E701CBD8008EBFF69
:10CC7100EAFEE9FD80EBE98DF0A4FEE5F002CD0AC4
:10CC8100E9CDF9EAFEEBFFEF89F0A4FCE5F0CE89EE
:10CC9100F0A42EFFE435F0CD89F0A42DFEE435F0AB
:10CCA1008067EF4E7005BD80D780C3EF8BF0A4ACD9
:10CCB100F0EE8BF0A42CFCE435F0F8EF8AF0A42C14
:10CCC100E5F038FCE433CB8DF0A42CFCE5F03BF827
:10CCD100EE8AF0A42CFCE5F038F8E433CF89F0A417
:10CCE1002CFCE5F038CF3400CE89F0A42FFFE5F01D
:10CCF1003EFEE433C98DF0A42EFEE5F039CD8AF075
:10CD0100A42FFFE5F03EFEE43DFD33D0E0FB5007EC
:10CD11000BBB000F02CEF5EC2CFCEF33FFEE33FE24
:06CD2100ED33FD02CECD52
:10CD270002CEF5EC5D046005E85904700302CEEB12
:10CD370012CEB6580460F6EC4860F2EC7004FDFEC3
:10CD4700FF22C82481C85007C398500602CEF29824
:10CD570050CEF582E9294B4A7005AB8202CEE175C8
:10CD6700F0007C1A7880C3EF9BEE9AED99400DC3D3
:10CD7700EF9BFFEE9AFEED99FDE842F0DC23ACF065
:10CD8700D0E0FFD0E0FED0E0FDAB8220E7101BEB48
:10CD970060BAEC2CFCEF33FFEE33FEED33FD02CE31
:10CDA700CDE803F830E705C0F075F000EF2FFFEE90
:0CCDB70033FEED33FD40B830E7C280AA27
:10CDC30074F8CC6480CCC86480C8F582046043C323
:10CDD300EB9FF5F0EA9E42F0E99D42F0E89C45F0B6
:10CDE30060305018E5825FFFE582F42B5582FB50DB
:10CDF300210ABA001D09B90019088016E5825BFBF8
:10CE0300E582F42F5582FF50090EBE00050DBD00CB
:10CE1300010CC3EB9FF5F0EA9E42F0E99D42F0E876
:0DCE23009C45F06007CC4820E701B3EC22ED
:10CE3000ED33EC33600A047003BD8004ECB2E7FC10
:01CE400022CF
:10CE410075F020800E75F010800575F0087D007E6C
:10CE5100007F003392D530D50312D31DEC3340103F
:10CE6100EF33FFEE33FEED33FDEC33FCD5F0ED2275
:0ECE7100E5F0247EA2D513CC92E7CDCEFF22B1
:10CE7F00EDD2E7CD33EC3392D524814006E4FFFEAB
:10CE8F00FDFC22FCE4CFCECDCC24E0501174FF800A
:10CE9F00EDC3CC13CCCD13CDCE13CECF13CF0470A7
:07CEAF00F030D5DE02D31DB7
:10D84000E5082495F582E43467F583E00508229025
:10D850006792300803906795E475F00112D40602D0
:10D86000D0F82001E97F2ED2018018EF540F2490C8
:10D87000D43440D4FF30050BEF24BFB41A0050035A
:10D880002461FFE50960021509050CE50C7002052D
:10D890000B30080E906792E475F00112D406EF0287
:10D8A000D13E02E6F97403D2088003E4C208F50809
:10D8B00090679212D434E4F509F50BF50CE5096094
:10D8C000077F2012D88380F5F50AC202C201C20385
:10D8D000C204C206C207C20912D84FFF700D300839
:10D8E000057F0012D894AF0CAE0B22B42563C2D5CD
:10D8F000C20512D84FFF24D0B40A00501E75F00A9A
:10D9000020D50DC509A42509F5097002D20480E0CF
:10D91000D201C50AA4250AF50A80D524CFB41A007D
:10D92000EF5004C2E5D20502DB7DD20280C2D201F3
:10D9300080BCD20380B8D2D580B6D20680B07F201A
:10D9400012D8832003077401B5090040F112D840B2
:10D95000FF12D88302D8BDD209D207809112D840D5
:10D96000FB12D840FA12D840F94A4B700679747A03
:10D97000DC7BFF200333E509602FAF0ABF00011FE6
:10D980007E008E8275830012D11160050EEE6F70DD
:10D99000F1C2D5EBC0E0EAC0E0E9C0E0EE12DBD9AD
:10D9A000D0E0F9D0E0FAD0E0FB12D0F8FF60A5EBB0
:10D9B000C0E0EAC0E0E9C0E012D883D0E02401F979
:10D9C000D0E03400FAD0E0FBE50A60DDD50ADA8069
:10D9D00083D203809E12DBBD60F7E50A12CEFFA959
:10D9E0000A600BE50A12DC61EF7003D50AF5EA3034
:10D9F000E702F404C3995079EAF4250A0430E701F8
:10DA0000E404F50A800D12DBBD60C6EA050A250AAA
:10DA100012CEFFEA9067C1F030E701E4250A04D591
:10DA20000A042006011412DBD9E4C0E012DC619084
:10DA300067C1E0601320E70714F012D86B8022045E
:10DA4000F0D0E014C0E07F0012D86BE50A60071246
:10DA5000D862150A800B30060312D862D0E002D8D3
:10DA6000BDD0E00480C412DBBD609EE50A0412CE86
:10DA7000FF9067C1EAF0E50A042006026001042471
:10DA80000412DBD974FF04C0E012DC6112D86BE52C
:10DA90000A200602600312D862D0E0B50AE87F458A
:10DAA00012D8759067C1E07F2B30E7047F2DF40416
:10DAB000C0E012D883D0E075F00A84C0F012D86CB0
:10DAC000D0E012D86C02D8BD791080027908C20764
:10DAD000C2098008D2D5790A8004790AC2D5E4FA4D
:10DAE000FDFEFF12D840FC7B0820021312D840FD37
:10DAF0007B1030010A12D840FE12D840FF7B20EC88
:10DB00003382D592D55013C3E43001069FFFE49EC3
:10DB1000FEE42002039DFDE49CFCE4CBF8C202EC91
:10DB2000700CCFCECDCCE824F8F870F38017C3EF9B
:10DB300033FFEE33FEED33FDEC33FCEB33FB99406A
:10DB400002FB0FD8E9EB300205F8D0E0C448B2027E
:10DB5000C0E00AEC4D4E4F78207B0070C2EAC0E076
:10DB600012DBDBD0F0D0E0200204C4C0E0C4B2027B
:10DB7000C0F012D86CD0F0D5F0EB02D8BD12D44969
:10DB8000D95D53DAC858D92E4CD92A42DACC4FDAAB
:10DB9000D444DAD449D94343DADA55DA0646DA66A8
:10DBA00045D9D547DC9750D9322DD9362ED9592BA6
:10DBB000D93A23D95720DC822A0000D95110010319
:10DBC000750A0612D840FC12D840FD12D840FE1249
:10DBD000D840FF9067BA02CF3C790AA2D52004143E
:10DBE000300609B910020404B9080104A2D52007BF
:10DBF000025001042003669203B509005032C0E0D0
:10DC00007F203004177F30A20372077206500D1276
:10DC1000DC30C203C207C2067F30800F300603E942
:10DC2000C0E012D883300603D0E0F9D0E0B509CEC9
:10DC30003006177F30B9100C12D8837F5830050793
:10DC40007F788003B9080312D8833003057F2D0243
:10DC5000D8837F202009F87F2B2007F322920380AE
:10DC6000CF7F00B40700500B24BAF582E43467F587
:10DC700083E0FF22286E756C6C29002D50434958B3
:10DC8000D20212D8403002F8C202780930D504D24C
:10DC900001780AF602D8EE12D8402403B4050040F9
:10DCA00001E490DC7B9312D874743A12D874D204D5
:06DCB00075090402DAC848
:10DCB600E50830040104F8232824C5F582E4346716
:10DCC600F583229067C23004039067C5E475F001BE
:10DCD60012D40602D0F860EAC50C7002150B14C502
:10DCE6000C200404FF02E7349067C274FFF5F002CB
:10DCF600D41DFF02E73CE5096006D509037F002233
:10DD0600050CE50C7002050B20040302E720906762
:10DD1600C212D3FD12D0F8FF60A89067C2E475F076
:10DD26000102D40612DD06EFC0E012DCF8D0E040B6
:10DD3600F380A3D2048002C2049067C212D434E4F2
:10DD4600F50AF508F50BF50C750900C203C201C208
:10DD560002C20512DCC9FF7005AF0A7E0022B42597
:10DD66003012DCC9FF24D0B40A00500C75F00AC585
:10DD760009A42509F50980E924CFB41A00EF500259
:10DD8600C2E502DF98D20280D8D20180D4D20580C3
:10DD9600D0EF12DCF8500512DD2A80ACEFC0E0129D
:10DDA600DD06D0E06F60A1EF606E12DCDC80AA7445
:10DDB60001C5096002F50912DD06EF605B20050E5C
:10DDC60012DCB6E475F00112D406EF12D13ED50985
:10DDD600E62005040508050A80C012DCFCEFC0E059
:10DDE60012DCF8D0E0500412DCDCE4FF20050E1251
:10DDF600DCB6E475F00112D406EF12D13EEF70DA0C
:10DE06002005040508050A8091E509600205091246
:10DE1600DD2A12DCFCEF70C6300404E412DCDCE51B
:10DE26000A600302DD5F7EFF7FFF22E509600205CF
:10DE36000912DD2AD207D20612DCFCEF3007026097
:10DE4600D7C0E012DCDCD0E0AC0DAD0EAE0FAF10EB
:10DE560012E5568C0D8D0E8E0F8F10500712DD06B3
:10DE6600C20680D4200510200602050A12DCB6126E
:10DE7600D3FD050812D35202DD4EEF12DCDC790821
:10DE8600803B12DD2A12DD06EF608DBF301B12DDEE
:10DE960006EF6084BF78028003BF58DE7910801DCC
:10DEA60012DD2A12DD06EF60E0790AEFB42D04D206
:10DEB600038019B42B02801412DCDC790AE50960B0
:10DEC600020509E9C0E012DD2AD0E0F9D206E4FC39
:10DED600FDFEFFE9C0E0ECC0E0EDC0E0EEC0E0EF23
:10DEE600C0E012DCFCEFF8D0E0FFD0E0FED0E0FDB1
:10DEF600D0E0FCD0F0E8604DB461004007B47B0090
:10DF06005002C2E524D0503DFA24F6500724F950B9
:10DF160034240AFAEAB5F000502BCFA9F0A42FFF5B
:10DF260092D5E9C5F0CEA4A2D53EFE92D5E9C5F0BC
:10DF3600CDA4A2D53DFD92D5E9C5F0CCA4A2D53C91
:0ADF4600FCC206808EE8C0E0200552
:10DF50002A200608050A30030312D31D12DCB6126C
:10DF6000D3FD050820010B20020DEE8FF012D1C663
:10DF7000800912D3528004EF12D13ED0E012DCDCD3
:10DF800002DD4E20051012DCB612D3FD0508E50BAC
:10DF9000850CF012D1C680E812D449DE0F53DEA200
:10DFA00058DD8F4CDD8B42DD8B48DE844FDEA6448E
:10DFB000DDB543DE8849DEC155DE3146DE3145DE62
:0CDFC0003147DD932ADF834E0000DD971F
:0DDFCC00ED33EC3360065004EC6480FC2261
:10DFD900D2079069E212D43412E015C0E0FF12E7CB
:10DFE9003CD0E040F312E556400122ECC0E0EDC020
:10DFF900E0EEC0E0EFC0E012E015D0F0AFF0D0F0F5
:10E00900AEF0D0F0ADF0D0F0ACF080D9E475F0010D
:09E019009069E212D40602D0F86D
:10E0220033DA929E35B16011377FE5FE392184895A
:10E032003AAEC3FF3C1D955B3D6358473E75FDF00C
:10E042003F3172183F800000C2D502CEF502CEEBFE
:10E05200BD80FA50F302CEF2ED33EC330460F17B73
:10E062003B7AAA79B8783F12CC21ED33EC3392D5C2
:10E07200247B5011A2D570DB500BED448024045058
:10E0820004A2D580CEEFFBEEFAEDF9ECF812CE7FCA
:10E09200EFF582F404FC12CE4B12CB30C08290E03A
:10E0A20022740912D050ED33CC33D0F092D525F042
:0AE0B200A2D57001C313CC13FD22A8
:10E0BC003E9248DA3ECCCCCD3F2AAAAB40000000C1
:10E0CC003F8000003F9837F03FB504F33FD744FC46
:10E0DC003E3172173EB172173F0515913EDE5BD98A
:10E0EC00D2018002C201EDD2E7F8CD33EC330470DB
:10E0FC000BBD800592D502CEF502CEEB40FBD314BE
:10E10C0060F2F5F07C3FEE7A00C39496C8948B4095
:10E11C00230AC89469C8941A401A0AC89468C89407
:10E12C001F40110AC8945AC89425400805F07A007B
:10E13C00CDC2E7CDC0F090694C12D3A4EA2323C022
:10E14C00E024CCF582E434E0F583C083C08212D3A2
:10E15C0094D082D08312CB30ECC0E0EDC0E0EEC0A6
:10E16C00E0EFC0E012D37890694C12D38812CB2C1C
:10E17C00D0E0FBD0E0FAD0E0F9D0E0B2E7F812CD75
:10E18C002A90694C12D3A490E0BC740312D0419035
:10E19C00694C12D38812CC21D0E0600F24D8F582C0
:10E1AC00E424E0F58312D39412CB3090694C12D353
:10E1BC00A4D0E0C3947FFDE49400FC12CE467B18FF
:10E1CC007A727931783F12CC2190694C12D3881233
:10E1DC00CB3030010B7BD97A5B79DE783E12CC21C7
:01E1EC002210
:10E1ED0002CEEB22EDA2E7D2E7F9EC3340F260F379
:10E1FD00B4FF08ED547F70E802CEF5F82481C2E03B
:10E20D00C0E0F40428FAC313FCED92E7FD90693CDD
:10E21D0012D3A4EEA2E7E9BA7F02C313340094002F
:10E22D00FA75F091A4E5F013F494FE8AF0A433E5A9
:10E23D00F033248CD313FDE492E7FE7F007C3F7511
:10E24D008302ECC0E0F8EDC0E0F9EEC0E0FAEFC0FB
:10E25D00E0FB8583F090693C12D36C85F08312CD81
:10E26D002AD0E0FBD0E0FAD0E0F9D0E0F812CB30C4
:10E27D00ED6480FD30E7011CD583C7ED33CC33F859
:0CE28D00D0E0A2E71328C313CC13FD223D
:10E299003A70FA83BCAAE9E43E81E0F8BF9DE9E659
:10E2A9003F80000039283C1ABB9969663DA335E3D4
:10E2B900BF255DE73FC90FDB418DDBCCC44936EE95
:10E2C90045C9913FC5B0F83D3F800000C317F534FB
:10E2D900452FFA73C60AFDDD12E3A204A2E19201F9
:10E2E9001420E01590E299740412D041803012E3B1
:10E2F900A230E102B20120E0EBA883A98290693C37
:10E3090012D3A48982888390E2AD740412D0418526
:10E3190082F090693C12D38885F08212CC21ED4CB1
:10E329006007300104EC6480FC2212E3A2C0E0A87B
:10E3390083A98290693C12D3A48982888390E2D10F
:10E34900740312D0418582F090693C12D38885F01C
:10E359008212CC2190693CE0CCF0A3E0CDF0A3E09F
:10E36900CEF0A3E0CFF090E2C1740312D041D08285
:10E379008582F090693C12D38885F082E58230E08D
:10E389000712CD2AB2018096EFCBFFEECAFEEDC986
:10E39900FDECC8FC12CD2A8085ED33EC547FCC33DB
:10E3A900920124605007D0E0D0E002CEEB7B837A63
:10E3B900F97922783E12CC21EDF933ECF833248136
:10E3C9005011EFFBEEFA12CE7F12CE41ECB2E7FC10
:10E3D90012CB30ED33EC33602F2403F8C313FCED7B
:10E3E90092E7FDE82481E4501FECF8EDF9EEFAEF2D
:10E3F900FB12CE7FEF04C2E0FCF58212CE4BECB2E9
:10E40900E7FC12CB30E58203FAED33EC33600714F5
:08E4190013FCED92E7FDEA227D
:10E42100BE1249253E4CCCCDBEAAAAAB3F8000000E
:10E431003E7ADBB03EED63383F24BC7D3F490FDBC4
:10E44100ED33ECC2E7CC339201B4FF13ED547F609E
:10E451000302CEEB7FDB7E0F7DC97C3F02E536C236
:10E4610002C3947F401E7007EDD2E794904015EFF0
:10E47100FBEEFAEDF9ECF87F007E007D807C3F1227
:10E48100CD2AD202ED33EC33248430E705E4C0E039
:10E49100806B04FAEDD2E754F0C333DAFD5407344C
:10E4A100002323C0E0CCC0E0F8EDC0E0F9EEC0E00D
:10E4B100FAEFC0E0FBE412CE4BEC24FEFC90693C89
:10E4C10012D3A412CC217B007A007980783F12CB41
:10E4D1003090693CE0B2E7CCF0A3E0CDF0A3E0CE10
:10E4E100F0A3E0CFF0D0E0FBD0E0FAD0E0F9D0E04B
:10E4F100F812CB3090693C12D38812CD2A90693C36
:10E5010012D3A490E421740312D04190693C12D338
:10E511008812CC21D0E0600F242DF582E434E4F59B
:10E521008312D39412CB3030020B7BDB7A0F79C983
:10E5310078BF12CB30ED33EC336006ECA20192E7E9
:02E54100FC22BA
:10CEB600E9D2E7C933E833F892D5EDD2E7CD33ECC2
:07CEC60033FC5002B2D5223B
:10CECD00EC30E7100FBF000C0EBE00080DBD0004C6
:10CEDD000BEB6014A2D5EB13FCED92E7FD2274FF72
:10CEED00FCFDFEFF22E480F8A2D574FF13FC7D80CB
:02CEFD0080F0C3
:10CEFF00F920E73624F950037907E4F42402FBE51F
:10CF0F0082158270021583DBF6E024FB501BE9606B
:10CF1F0014E4F0E582158270021583E004F0B40A80
:0DCF2F0008E4F0D9EE7401F00A22C2D52208
:10CF3C00ED33EC3392D5FA602AB4FF33EDC2E77BC4
:10CF4C00FF60067ACF7961E4227ACF796A20D50422
:10CF5C007ACF7965224E614E002B494E46002D4901
:10CF6C004E4600E47A08F0A3DAFC7B00740722C07A
:10CF7C0083C082ECC0E0EDC0E0EEC0E0EFC0E0EAC0
:10CF8C0075F010A4CAABF075F04DA42BFBE435F092
:10CF9C00FCEA2410FAEB34C5FBEC34D9FCEDC2E707
:10CFAC00FF75F056A4F42411C5F0F434C58FF0A429
:10CFBC002AE5F03BE43CF020E71412D0B8D0E0FFB7
:10CFCC00D0E0FED0E0FDD0E0FC12CD2A8014F404B9
:10CFDC0012D0B8D0E0FFD0E0FED0E0FDD0E0FC12E3
:10CFEC00CC21D082D083E0FAEDD2E7CD33EC3324E0
:10CFFC0082FBE4C3CF33CFCE33CECD33CD33DBF393
:10D00C007B0775F00A846004F0A31B0AE5F0F0A31B
:10D01C008FF0740AA4FFACF08EF0740AA42CFEAC52
:10D02C00F050010C8DF0740AA42CFDE435F0F0A343
:05D03C00DBDE74072299
:10E54300C208C209C20AC20BF9E4F511F512FCFDB7
:10E55300FEFFE91007EA200A0CB42D04D20AD322E5
:10E56300B42B02D32224D0504794095041240A30BB
:10E573000B15F88512F0740AA42872E74051C5F010
:10E58300704D85F012D322D209C0E0E4FBFA792062
:10E59300784112CC21ECF8EDF9EEFAEFFBD0E0FC78
:10E5A300E412CE4B12CB303008B41511D322240A17
:10E5B300200B20B4FE0720081AD208D32224EB60D4
:10E5C3000424E0700EA20A9208D20BC20AD322C31B
:10E5D30002CEEBE4300B0BE512300A02F404A2087E
:10E5E300920A3009EA251120D2E5A2E7920B5002E4
:10E5F300F404B4260050D8CCC0E0EDC0E0EEC0E097
:10E60300EFC0E0EC12D0B8D0E0FFD0E0FED0E0FDE8
:10E61300D0E0FC200B0512CC21800312CD2A300A56
:06E623000312CE30C322F9
:10D04100C0E0EFFBEEFAEDF9ECF812CC21D0E0F5FF
:10D05100F0EFFBEEFAEDF9ECF812D378A3E8C0E0BB
:10D06100E9C0E0EAC0E0EBC0E0C0F012CC2112D38D
:10D0710094A312CB30D0F0D0E0FBD0E0FAD0E0F9AD
:07D08100D0E0F8D5F0D72242
:10D088003F8000004120000042C80000447A0000B0
:10D09800461C400047C35000497424004B18968032
:10D0A8004CBEBC205A0E1BCA6753C21C749DC5AE29
:10D0B800FB60065407601C232312D0E6EB5438604B
:10D0C8000912D0D212D0E112CC21ECF8EDF9EEFA27
:10D0D800EFCB22EB12D0E180F1543803241C90D01E
:10D0E80088FE93FC0EEE93FD0EEE930ECE93FF2278
:0300000002E629EC
:0CE62900787FE4F6D8FD75814002E670B1
:10D0F800BB010689828A83E0225002E722BBFE0236
:09D10800E32289828A83E4932268
:10D11100BB010CE58229F582E5833AF583E02250D3
:10D1210006E92582F8E622BBFE06E92582F8E2221D
:0DD13100E58229F582E5833AF583E4932237
:10D13E00BB010689828A83F0225002F722BBFE01D0
:02D14E00F322CA
:10D15000EFF88DF0A4FFEDC5F0CEA42EFEEC88F024
:04D16000A42EFE22D9
:10D16400C2D5EC30E709B2D5E4C39DFDE49CFCEEE6
:10D1740030E715B2D5E4C39FFFE49EFE12D7D3C3B4
:10D18400E49DFDE49CFC800312D7D330D507C3E4AF
:06D194009FFFE49EFE2255
:10D19A00C5F0F8A3E028F0C5F0F8E5821582700220
:06D1AA001583E038F022BD
:10D1B000A3F8E0C5F025F0F0E58215827002158332
:06D1C000E0C838F0E8228F
:10D1C600BB010A89828A83F0E5F0A3F0225006F7B4
:0FD1D60009A7F01922BBFE06F3E5F009F31922B1
:0DD1E500EF2BFFEE3AFEED39FDEC38FC2299
:0ED1F200C3EF9BFFEE9AFEED99FDEC98FC2238
:10D20000E88FF0A4CC8BF0A42CFCE98EF0A42CFCCD
:10D210008AF0EDA42CFCEA8EF0A4CDA8F08BF0A44B
:10D220002DCC3825F0FDE98FF0A42CCD35F0FCEBAA
:10D230008EF0A4FEA9F0EB8FF0A4CFC5F02ECD396F
:0FD24000FEE43CFCEAA42DCE35F0FDE43CFC22DC
:10D24F0075F008758200EF2FFFEE33FECD33CDCC96
:10D25F0033CCC58233C5829BED9AEC99E582984019
:10D26F000CF582EE9BFEED9AFDEC99FC0FD5F0D6F6
:10D27F00E4CEFBE4CDFAE4CCF9A88222B800C1B920
:10D28F000059BA002DEC8BF084CFCECDFCE5F0CB5E
:10D29F00F97818EF2FFFEE33FEED33FDEC33FCEB97
:10D2AF0033FB10D703994004EB99FB0FD8E5E4F952
:10D2BF00FA227818EF2FFFEE33FEED33FDEC33FC3F
:10D2CF00C933C910D7059BE99A4007EC9BFCE99A33
:10D2DF00F90FD8E0E4C9FAE4CCFB2275F010EF2F78
:10D2EF00FFEE33FEED33FDCC33CCC833C810D70778
:10D2FF009BEC9AE899400AED9BFDEC9AFCE899F8B3
:0ED30F000FD5F0DAE4CDFBE4CCFAE4C8F92245
:10E6B500C2D5E830E70FB2D5E4C39BFBE49AFAE490
:10E6C50099F9E498F8EC30E717B2D512E6EB12D2D7
:10E6D5008BE4C39BFBE49AFAE499F9E498F8800388
:10E6E50012D28B30D50DE4C39FFFE49EFEE49DFD61
:04E6F500E49CFC2283
:0ED31D00C3E49FFFE49EFEE49DFDE49CFC2221
:10D32B00EB9FF5F0EA9E42F0E99D42F0EC6480C879
:06D33B0064809845F02219
:10D34100EB9FF5F0EA9E42F0E99D42F0E89C45F042
:01D3510022B9
:10D35200BB010789828A8302D3A45005E9F802D867
:0AD3620028BBFE05E9F802D83422CA
:0CD36C00E0FCA3E0FDA3E0FEA3E0FF2234
:10D37800E493FCA3E493FDA3E493FEA3E493FF22C8
:0CD38800E0F8A3E0F9A3E0FAA3E0FB2228
:10D39400E493F8A3E493F9A3E493FAA3E493FB22BC
:0CD3A400ECF0A3EDF0A3EEF0A3EFF022FC
:10D3B000A8828583F0D083D08212D3C712D3C7123C
:10D3C000D3C712D3C7E473E493A3C583C5F0C58361
:10D3D000C8C582C8F0A3C583C5F0C583C8C582C8C7
:01D3E000222A
:0CD3E100A42582F582E5F03583F5832257
:10D3ED00FAE6FB0808E6F925F0F618E6CA3AF62241
:09D3FD00E0FBA3E0FAA3E0F92231
:10D40600F8E0FBA3A3E0F925F0F0E58215827002AF
:07D416001583E0FA38F02253
:10D41D00F8E0FBA3A3E025F0F9F0E5821582700298
:07D42D001583E038FAF0223C
:09D43400EBF0A3EAF0A3E9F022F9
:0CD43D00E493FB740193FA740293F9224B
:10D44900D083D082F8E4937012740193700DA3A372
:10D4590093F8740193F5828883E473740293686086
:06D46900EFA3A3A380DF86
:10E6F900EFB40A07740D12E704740A309811A89947
:10E70900B8130CC2983098FDA899C298B811F63080
:07E7190099FDC299F5992258
:10E7200010000B12EA25BF0D027F0A02E6F990677E
:04E73000D7E0FF220D
:08E734009067D7EFF0D200223C
:10E73C00EFC394094006EFC3940E4004EFB42003DA
:05E74C00D38001C3228F
:10E75100C3EE6480948040028007C3E49FFFE49E7F
:02E76100FE2296
:10E763009068DB12D3A47F007E007D007C0090685C
:10E77300DBE0F8A3E0F9A3E0FAA3E0FBC312D32B99
:10E7830040109068DBE0FCA3E0FDA3E0FEA3E0FF04
:10E7930080119068DBE0FCA3E0FDA3E0FEA3E0FFB3
:04E7A30012D31D224E
:10E7A7009069E2EBF0A3EAF0A3E9F09069E5E0FBFA
:10E7B700A3E0FAA3E0F912D0F8FE9069E2E0FBA328
:10E7C700E0FAA3E0F912D0F8FD6E702AED600E9022
:10E7D70069E874FFF5F012D19A45F070037F0022C3
:10E7E7009069E3E475F00112D19A9069E6E475F057
:10E7F7000112D19A80B5D3EE6480F8ED6480984019
:07E80700037F01227FFF22C5
:10E80E00E4FFFE12D0F8600C0FEF70010E09E970F4
:05E81E00F20A80EF2268
:10E82300E94A4B70012212D0F8FF6D700122EF709C
:0CE8330004FBFAF92209E970ED0A80EA02
:10E83F0090688FEBF0A3EAF0A3E9F090688FE0FB0C
:10E84F00A3E0FAA3E0F912D0F8FF12E73C500C90C6
:10E85F006890E475F00112D19A80E0D20190688F30
:10E86F00E0FBA3E0FAA3E0F912D0F8FF642B6004F9
:10E87F00EFB42D1D90688FE0FBA3E475F00112D16A
:10E88F00B0A9F0FA12D0F8642D6003D38001C392BF
:10E89F000190689212D3B00000000090688FE0FBE7
:10E8AF00A3E0FAA3E0F912D0F8FF12EA2F506A7F23
:10E8BF000A7E007D007C00906892E0F8A3E0F9A347
:10E8CF00E0FAA3E0FB12D200C8ECC8EDC0E0EEC046
:10E8DF00E0EFC0E090688FE0FBA3E0FAA3E0F9124D
:10E8EF00D0F8FF3395E0FEEF24D0FFEE34FFFEE4C7
:10E8FF00FCFDD0E0FBD0E0FAD0E0F9EB2FFFEA3ED1
:10E90F00FEED39FDEC38FC90689212D3A49068901C
:10E91F00E475F00112D19A8082300110906892E074
:10E92F00FCA3E0FDA3E0FEA3E0FF8011906892E05E
:0EE93F00FCA3E0FDA3E0FEA3E0FF12D31D2227
:10E94D009068AEEBF0A3EAF0A3E9F09068AEE0FBBF
:10E95D00A3E0FAA3E0F912D0F8FF12E73C500C90B7
:10E96D0068AFE475F00112D19A80E0D2019068AEE3
:10E97D00E0FBA3E0FAA3E0F912D0F8FF642B6004EA
:10E98D00EFB42D1D9068AEE0FBA3E475F00112D13C
:10E99D00B0A9F0FA12D0F8642D6003D38001C392B0
:10E9AD0001E49068B1F0A3F09068AEE0FBA3E0FA4B
:10E9BD00A3E0F912D0F8FF12EA2F503F9068AEE0B5
:10E9CD00FBA3E0FAA3E0F912D0F8FF3395E0FEEFD8
:10E9DD0024D0FBEE34FFFA9068B1E0FEA3E0FF7C9B
:10E9ED00007D0A12D150EF2BF0EE3A9068B1F09005
:10E9FD0068AFE475F00112D19A80AD30010A9068CC
:10EA0D00B1E0FEA3E0FF800F9068B1E0FEA3E0FF50
:08EA1D00C3E49FFFE49EFE220A
:10D46F00EF4E6013EDBB011089828A83EF60010ECE
:10D47F00EDF0A3DFFCDEFA2289F05007F709DFFC9D
:0DD48F00A9F022BBFE06F309DFFCA9F02284
:10D49C00E709F608DFFA8046E709F208DFFA803E72
:10D4AC0088828C83E709F0A3DFFA8032E309F6085F
:10D4BC00DFFA806EE309F208DFFA806688828C83DB
:10D4CC00E309F0A3DFFA805A89828A83E0A3F60885
:10D4DC00DFFA804E89828A83E0A3F208DFFA804269
:10D4EC0080D280FA80C680D4805580F2802980104A
:10D4FC0080A680EA809A80A880DA80E280CA80299F
:10D50C0088848C8589828A83E493A30586F0A3059D
:10D51C0086DFF5DEF3800B89828A83E493A3F60819
:10D52C00DFF9ECFAA9F0EDFB2288848C8589828ADC
:10D53C0083E0A30586F0A30586DFF6DEF480E3899D
:10D54C00828A83E493A3F208DFF980D688F0ED2475
:10D55C0002B4040050CCF582EB2402B4040050C297
:10D56C0023234582F582EF4E60B8EF60010EE58211
:05D57C002390D4EC73C4
:10D58100E3F5F009E208B5F06D606B80F3E3F5F0C7
:10D5910009E608B5F060605E80F387F009E608B53A
:10D5A100F054605280F487F009E208B5F048604613
:10D5B10080F488828C8387F009E0A3B5F038603667
:10D5C10080F488828C8387F009E493A3B5F0276007
:10D5D1002580F388828C83E3F5F009E0A3B5F0168A
:10D5E100601480F388828C83E3F5F009E493A3B59A
:10D5F100F004600280F202D698808580E7808E80F8
:10D60100D28032801580628074809B80B5808B804F
:10D61100A180458066803002D6AE88848C8589825F
:10D621008A83E493F5F0A30586E493A30586B5F018
:10D6310066606480ED89828A83E493F5F0A3E20851
:10D64100B5F054605280F289828A83E0F5F0A3E656
:10D6510008B5F043604180F389828A83E0F5F0A345
:10D66100E208B5F032603080F389828A83E493F571
:10D67100F0A3E608B5F020601E80F2804988848C12
:10D681008589828A83E493F5F0A30586E0A3058664
:10D69100B5F004600280EE7F00F845F0600EE863AB
:10D6A100F0806480D395F01F40027F012288848C32
:10D6B1008589828A83E0F5F0A30586E0A30586B516
:10D6C100F0D560D380EF88848C8589828A83E0F5E8
:10D6D100F0A30586E493A30586B5F0BB60B980EE9F
:10D6E10088F0ED2402B4040050ADF582EB2402B4BD
:0DD6F100040050A3232345822390D5FA7333
:10D6FE00E709F60870FA8046E709F20870FA803EEC
:10D70E0088828C83E709F0A370FA8074E309F60827
:10D71E0070FA806CE309F20870FA806488828C8358
:10D72E00E309F0A370FA805889828A83E0A3F60891
:10D73E0070FA804C89828A83E0A3F20870FA8040E6
:10D74E0080D280FA80C680D4805180F280278010EB
:10D75E0080A680EA809A80A880DA80E280CA80273C
:10D76E0088848C8589828A83E493A30586F0A30539
:10D77E008670F5800B89828A83E493A3F60870F98C
:10D78E00ECFAA9F0EDFB2288848C8589828A83E0ED
:10D79E00A30586F0A3058670F680E589828A83E468
:10D7AE0093A3F20870F980D888F0ED2402B4040037
:10D7BE0050CEF582EB2402B4040050C423234582DC
:05D7CE002390D74E730B
:10E63500020003E493A3F8E493A34003F68001F2F8
:10E6450008DFF48029E493A3F85407240CC8C333E6
:10E65500C4540F4420C8834004F456800146F6DFB5
:10E66500E4800B010204081020408090C9FEE47E7E
:10E67500019360BCA3FF543F30E509541FFEE493AA
:10E68500A360010ECF54C025E060A840B8E493A371
:10E69500FAE493A3F8E493A3C8C582C8CAC583CA9C
:10E6A500F0A3C8C582C8CAC583CADFE9DEE780BE54
:01CAAD000088
:10D7D300BC000BBE0029EF8DF084FFADF022E4CC3A
:10D7E300F875F008EF2FFFEE33FEEC33FCEE9DEC03
:10D7F300984005FCEE9DFE0FD5F0E9E4CEFD22ED49
:10D80300F8F5F0EE8420D21CFEADF075F008EF2F92
:10D81300FFED33FD4007985006D5F0F222C398FD83
:05D823000FD5F0EA2220
:0CD82800ECF608EDF608EEF608EFF6222C
:0CD83400ECF208EDF208EEF208EFF22230
:0AEA25003098FDAF99C2987E0022E0
:10EA2F00EFC394304009EFC3943A5003D38001C32E
:01EA3F0022B4
:00000001FF
